:100000000C94F5110C941D120C941D120C941D12DD
:100010000C941D120C941D120C941D120C941D12A4
:100020000C941D120C941D120C9478180C9497705B
:100030000C9402750C94E4700C941D120C9403192A
:100040000C9466180C941D120C941D120C941D1225
:100050000C941D120C941D120C941D120C941D1264
:100060000C9485750C9449190C9443710C94CF75BC
:100070000C941D120C941D120C94076E0C941D12FE
:100080000C941D120C941D120C941D12E01AE41A0B
:10009000A91AAF1AB51AB51AB51AD81ADC1AE01A85
:1000A000E41AF11AF11AE81A282528252825282506
:1000B00052254925492549254925492549254925C7
:1000C00038253D253D251931233138318531C13160
:1000D0001E3229322C3285328932CA35DF357536E7
:1000E000F4376538FF36153CB839DE38E6384B3919
:1000F000BC3AA543A346A646AA46B046B446B9466E
:10010000BC4DCB4DD64DEC4DF34DFA4D094E204E26
:10011000394EF64E214F294F314F3D4F574F614FCA
:100120008B4FD84FE44F1F502E50385046505250EE
:10013000A6538E5F2656FE5CA6568E5F8E5FCE5B04
:100140008E5F635E8E5F8E5F6B55B653AA57436CAE
:10015000326C2C6C346C386C3C6C2F6C406C466C84
:10016000DB73DE73F57310741074F573F573F57645
:10017000F776FA76FF7610771F772D773777477700
:1001800057775C777277757779777B777D7782772A
:100190008677917795779D77A477A877AA77AE77BA
:1001A000B077B277B477B877BC77C177C677CB77BB
:1001B000D077D577204F6C642056657273696F6E67
:1001C00020454550524F4D202020434845434B2069
:1001D00053455454494E47532F43414C49420041E3
:1001E0006C61726D732044697361626C6564004573
:1001F0004550524F4D206C6F77206D656D004C4F10
:100200004144494E47000553746F70706564006D3A
:10021000537461636B206F666C6F770053776974FA
:100220006368205761726E696E671F506C656173F9
:1002300065205265736574205377697463686573CC
:10024000005468726F74746C65206E6F74206964FA
:100250006C651F5265736574207468726F74746C7A
:1002600065004D45535341474500707265737320D7
:10027000616E79204B657900507265737320616EF1
:1002800079206B657920746F20736B6970004F461D
:10029000464F4E20544873544825000000642810EF
:1002A0000703010000000001010102020202010136
:1002B00003002D2D2D2D0020414C455254000401EA
:1002C000221F25280904010203070809000102036F
:1002D00000020103030102000302010004527564DD
:1002E00020456C65205468722041696C20004F4E97
:1002F00020004F46460003544852525544454C4551
:1003000049443049443149443241494C47454154BC
:10031000524E4C31204C32204C33204C34204C3542
:10032000204C36204C37204C38204C39204C412072
:100330004C42204C4320454C80454C2D454C81522D
:10034000558052552D52558141498041492D414991
:100350008147458047452D474581504231504232C3
:10036000001B1E272D36394B4E636C7278878D9398
:100370009CB1B4C6C9D2D8E1E453706C6173680013
:1003800080400000000000000000000000000000AD
:10039000000000000000000000000000000000005D
:1003A000000000000000000000000000000000004D
:1003B000000000000000000000000000000000003D
:1003C0000000000000000000000000000080C0E00D
:1003D000E0F0F8F8FCFCFCF8F8F8F0400000000051
:1003E000008080800000000000000000000000008D
:1003F0000000000000000080C0C0E0E0E0F0F0F08D
:10040000E0C00000000000C0F8FFFF9F87838383E7
:1004100083838383838383838383838383838383AC
:10042000838383038380838383838383838383831F
:1004300083838383838383838383838383C3E373FC
:100440003F1F0000000080E0F0F8FCFEFFFFFFFF10
:100450007F3F1F1F0F0783C3E1E1E0E0C0000E1FD5
:100460003F7F7FFFF3E0E08000000000000000001D
:10047000000080F0FCFEFFFFFFFF7F3F0F03010144
:100480000100000080F0FEFFFFC7C1C1C1C1C1C1B2
:10049000C1C1C1C1C1C1C1C1C1C1C1C1C1C1C1C14C
:1004A00001C1F0FEFF3F0F070F0D0D0D1D191919AA
:1004B000193131313171616161E1C1C1C181000026
:1004C0000080E0F8FCFFFFFFFF2F170F038180C0C3
:1004D000E0F0F8FCFEFFFFFFFFFFFF7F01000000E0
:1004E0000000000001010307070E1E1C3870E0F039
:1004F000F8FEFFFF7F1F0F03000100000000000057
:1005000000000000000000000000000000000000EB
:1005100000000000000000000000000000000000DB
:1005200000000000000000000000000000000000CB
:1005300000000000000000000000000000000000BB
:100540007EFFFFFFFFFFFFFBF8FCFCFEFF7F3F1F6E
:100550000F07C3FFFFFFFFFFFF7F07000000000042
:10056000000000000000000000C0E0F8FEFFFF7F78
:100570001F0F1F3D7CF8F8F0E08000000000000035
:10058000000000000000000000000000000000006B
:10059000000000000000000000000000000000005B
:1005A000000000000000000000000000000000004B
:1005B000000000000000000000000000000000003B
:1005C000000001010101010307070703010000000A
:1005D000E0FCFFFFFFFFFF1F030000000000000022
:1005E00000000000C0F078DE2713090E07030000AA
:1005F00000000000000001030F7FFFFC7878F80086
:1006000000000000000000000000808080808080EA
:10061000808080008080008080000000000000005A
:1006200080808080808080808080808080808080CA
:1006300080800000000000000000000000000000BA
:100640000000000000000000000000000080F0FE3C
:10065000FFFFFFFF3F0F010000000000000000C08F
:10066000E0381E0F03000100000000000000000041
:100670000000000000000000000000000003030173
:10068000000000000000000000000E0E0202020246
:10069000020303000F0F000F0F08080808080808DE
:1006A0000F0F08080808080F0F000000000F0F00C8
:1006B000000000000000000000000000000000003A
:1006C0000000000000000000000000C0F8BFFFFFB5
:1006D000FF1F7F010000000000000000F0FCFF7F12
:1006E0007830000000000000000000000000000062
:1006F00000000000000000000000000000000000FA
:1007000000000000000000000000000000000000E9
:1007100000000000000000000000000000000000D9
:1007200000000000000000000000000000000000C9
:1007300000000000000000000000000000000000B9
:10074000000000000000000000301C070E0F070131
:100750000000000000000000000000000000000099
:100760000000000000000000000000000000000089
:100770000000000000000000000000000000000079
:10078000000000564552533A2056312E1F44415422
:10079000453A2030332E30312E323032311F544919
:1007A0004D453A2030303A30323A31351F205356D9
:1007B0004E3A20657239782D7076723832321F20A9
:1007C0004D4F443A202020202020003603064F4E73
:1007D000202020204F4646202020424F54482020F1
:1007E00056617269626C005653001E010153580035
:1007F0004E756D62657220566F6963652053770090
:100800005361666574792053776974636865730012
:10081000434F5059205452494D205B4D454E555D34
:10082000000D4F6E004C4F474943414C20535749F0
:100830005443484553003C010A436F756E7420448D
:100840006F776E436F756E74205570202000546969
:100850006D65721F54726967676572411F547269D2
:1008600067676572421F54696D65721F52657365D3
:100870007420537769746368000A506F776572005B
:1008800020547970651F204368616E731F20436F89
:10089000756E7472791F42696E641F52616E67656E
:1008A000003C02094C50342F4C5035202044534D0D
:1008B000326F6E6C792044534D322F44534D5800A3
:1008C00044534D20547970650004486967684C6F43
:1008D00077200000044E6F6E650006466C79736BDE
:1008E0007948756273616E4672736B7944486973B7
:1008F0006B792056327832202044534D20202044FA
:1009000065766F20205944373137204B4E20202008
:100910002053796D615820534C5420202043583186
:10092000302020434730323320426179616E674680
:1009300072736B795845536B7920204D543939784F
:10094000784D4A587120205368656E716946593355
:100950003236205346485353204A3650524F204691
:100960005137373720415353414E204672736B79CC
:1009700056484F4E5441494F706E4C727341464831
:10098000443253513258322020574B327830315153
:100990003330332020475730303820444D30303208
:1009A00020434142454C4C45534B31353048385F2C
:1009B000334420434F524F4E4143466C69652048B3
:1009C000697465632057464C59202042554753208F
:1009D000204255474D494E5472617861734E433100
:1009E0003730314530315820205639313153204786
:1009F00044303058205637363120204B463630367A
:100A00002052656470696E506F74656E735A5358E6
:100A1000202020466C797A6F6E5363616E65724652
:100A200072736B7952414648445352486F54542074
:100A300020465838313620426179616E5250656CDB
:100A40006B616E546967657220584B2020202058D6
:100A50004E5F444D504672736B58324672536B5220
:100A60003950524F50454C4C5231322020536B7903
:100A70006172740050726F746F636F6C1F54797081
:100A8000651F506F7765721F42696E6420202020B9
:100A9000204175746F62696E641F52616E676500F4
:100AA000660103504F534E454700506F6C617269A9
:100AB00074790050504D2046724C656E0D6D536533
:100AC00063000C52784E756D000434434820364361
:100AD000482038434820313043483132434831348C
:100AE00043483136434800137553000650504D209B
:100AF0002020584A5420202044534D32202050506A
:100B00004D31362050504D53494D4D554C54492090
:100B1000534255532020000A317374204368616E9C
:100B20001F50726F746F000444521F024578706F3B
:100B30001F1F015765696768741F1F44725377311F
:100B40001F447253773200034869204D6964204C7A
:100B50006F77006604042D2D2D2D31323020313277
:100B60003058313430203930202000537761736899
:100B700020547970651F436F6C6C6563746976658A
:100B80001F53776173682052696E671F454C45207B
:100B9000446972656374696F6E1F41494C204469F2
:100BA00072656374696F6E1F434F4C2044697265B0
:100BB0006374696F6E0052455441313233005404FE
:100BC00006457870202020457846696E6546696E36
:100BD0006520204D656469756D436F6172736500B2
:100BE0005472696D20496E631F5472696D2053778A
:100BF0001F48692E52657320536C6F772F44656CC4
:100C000061791F547261696E65721F42656570205B
:100C1000436E74005A01062020456E642043656EC1
:100C200074726500452E204C696D6974731F546899
:100C3000722E2044656661756C741F5468726F74FF
:100C4000746C6520726576657273651F5468726F87
:100C500074746C65204F70656E1F542D5472696DED
:100C60001F542D4578706F2D4472006607032D2D9B
:100C70002D503120503220503320475634475635BE
:100C8000475636475637004465666C742053771FC5
:100C9000437573746F6D53746B4E616D65731F4153
:100CA00075746F204C696D6974731F566F6C756D28
:100CB0006520436F6E74726F6C00566F69636520B8
:100CC000496E646578114D454E55000519F019FBC4
:100CD00019E819E219DB1997170B19CA19BF1991ED
:100CE000176F1BE517B619564100566F696365000B
:100CF0004D454E55204C4F4E470044656C6574651C
:100D000000566F6963652046696C65004E03072DC8
:100D10002D2D2D2D2D2D4861707469633148617022
:100D20007469633248617074696333000776603DAB
:100D300076616C20763D76616C20200007280D29B5
:100D400000506C617920536F757263651F4F6E2080
:100D50006E6F2054656C656D657472791F46696CA1
:100D6000655479706500536F757263651F46756EC3
:100D70006374696F6E1F56616C75651F5377697474
:100D800063681F526174651F48617074696300561F
:100D90006F69636520416C61726D00034D4F56456C
:100DA00020535449434B532F504F54530005534540
:100DB00054204D4944504F494E5400035B4D454E1D
:100DC000555D20544F20535441525400537469636D
:100DD0006B205248206465616462616E64005374E4
:100DE00069636B205256206465616462616E6400C1
:100DF000537469636B204C48206465616462616E62
:100E00006400537469636B204C56206465616462AE
:100E1000616E64006607044E4F4E45455854314597
:100E200058543250433020504732205042372050DF
:100E30004735204C2D575200454C45207377697437
:100E400063681F41494C207377697463681F50427F
:100E500031207377697463681F5042322073776959
:100E60007463681F50473220496E7075741F50427A
:100E70003720496E7075741F4C2D575220496E7083
:100E80007574004D27536F756E64205365726961E8
:100E90006C0042616E644761700043616C004D7587
:100EA0006C7469706C696572001802036F66662065
:100EB0002B3D203A3D00036D6F64650A2520737257
:100EC00063202073770007536C61766500124247F8
:100ED00000414E41000F504232000F504231005449
:100EE00072696D2D202B00204C6566741F52696756
:100EF00068741F0355701F20446F776E1F2045785C
:100F000069741F204D656E75004449414700496E64
:100F1000766572742054656C656D657472790053E2
:100F20007469636B5363726F6C6C00506F745363BE
:100F3000726F6C6C0053706C6173682073637265C0
:100F4000656E1F53706C617368204E616D65004162
:100F50006C61726D205761726E696E6700426174D8
:100F600074657279207761726E696E671F496E6170
:100F70006374697669747920616C61726D136D1F99
:100F80005468726F74746C65205761726E696E6715
:100F90001F537769746368205761726E696E671FAB
:100FA0004D656D6F7279205761726E696E6700438F
:100FB000726F73735472696D1F5468726F74746CBE
:100FC0006520726576657273651F456E61626C653A
:100FD0002050504D53494D1F4368616E6E656C2023
:100FE0004F726465721F4D6F6465002048617074B4
:100FF000696320537472656E6774680042040A4224
:10100000656570657220202020506953706B7220D6
:101010002020204265657072566F69636550695380
:10102000706B566F6963654D656761536F756E646C
:1010300020005406065175696574204E6F4B657922
:10104000207853686F727453686F7274204E6F7299
:101050006D20204C6F6E672020784C6F6E672000EB
:10106000566F6C756D651F4265657065721F536FB5
:10107000756E64204D6F64651F20537065616B65EC
:1010800072205069746368004C69676874207377D4
:10109000697463681F4261636B6C69676874206977
:1010A0006E766572741F4C69676874206F6666207F
:1010B00061667465721F4C69676874206F6E205397
:1010C000746B204D761F466C617368206F6E2062D2
:1010D00065657000436F6E747261737400FD17B4C0
:1010E00017D517E517CC17C017F517ED17AA17A2D4
:1010F00017DC170B4F7074696F6E00014E59000BAF
:1011000054656C656D2E000B565458202020000D40
:1011100052617465000B542D00064175746F49448B
:10112000466978644944000B467265712E000420BC
:10113000346368203563682036636820376368202D
:1011400038636820396368313063683131636831EE
:101150003263680022047C5E034578704578464619
:101160006E654D65644372730011544F541F0154F2
:101170004D45115453571F0153544B1153542500DF
:10118000035B4D454E555D20746F20726566726538
:10119000736800746D72314C6174206D61781275E2
:1011A000731F746D72314C6174206D696E127573AA
:1011B0001F746D7231204A69747465721275731FE1
:1011C000746D61696E126D73005354415400096669
:1011D000726565004D4F44454C53454C0020464DCB
:1011E000300A52455441004241434B555020444F30
:1011F0004E4500524553544F5245440053415649C1
:101200004E4700524553544F52494E47004C4F41B0
:1012100044494E4700526573746F72650020464D15
:10122000005377697463681F5472696D731F466158
:10123000646520496E1F46616465204F75740046E1
:101240004C204D4F44450052414E474520434845B0
:10125000434B20525353493A000642494E44494EAB
:1012600047004475706C69636174696E67206D6FC7
:1012700064656C0044454C455445204D4F44454CF5
:10128000004455504C4943415445204D4F44454C32
:101290000054656D706C61746573104D454E55005A
:1012A000202020202020202020202020202000443A
:1012B000454C455445204D49583F00436C6561728B
:1012C00020414C4C206D697865733F0003594553AC
:1012D0000B4E4F1F035B4D454E555D0B5B4558490B
:1012E000545D004D6178206D697865727320726578
:1012F0006163683A2033321F1F5072657373205B3D
:10130000455849545D20746F2061626F7274004EBD
:10131000020841646420202020204D756C7469709F
:101320006C795265706C616365200008446966667B
:1013300000114578706F0001557365204F7574700A
:1013400075742020200001536F757263651F01576B
:1013500065696768741F014F66667365741F01468F
:101360006978204F66667365741F01456E61626C13
:10137000654578706F44521F015472696D1F1F1FBD
:10138000015377697463681F014D6F6465731F01B2
:101390004D756C7470781F0144656C617920446FE1
:1013A000776E1F0144656C61792055701F01536C85
:1013B0006F772020446F776E1F01536C6F7720206A
:1013C00055700045444954204D495820004F500065
:1013D00054656D706C61746573005343092B0D2A5D
:1013E000122F00536F757263651F1F4F666673651A
:1013F000741F4D756C7469706C6965721F446976F1
:1014000069736F721F556E69741F5369676E1F444D
:101410006563696D616C731F4F6666736574204107
:1014200074005B2D3E5D00435600505245534554B9
:10143000006A01032D2D2D494E56005357522000AE
:101440003C0102313620382403034431364438202D
:101450004C525052394D3C0203416D654A61704512
:10146000757201084C523132202020204C5231320A
:101470005F366368000437345F5A03063931354DEF
:10148000487A3836384D487A3931355F38633836DE
:10149000385F3863040643485F31362043485F387D
:1014A000202045555F31362045555F382020436C5C
:1014B0006F6E656403043235304B314D2020324D60
:1014C00020204155544F01045834353058343230BF
:1014D0000003503338010752582020202020436C4D
:1014E0006F6E6554580006465A5F3431300003323F
:1014F00038300003413230010446617374536C6F1D
:1015000077010547445F563147445F56320105561F
:1015100039313153453131392002054530313220DE
:101520004530313520453031364801084275677302
:101530006D696E69427567733348202002064F70EB
:10154000745F46774F70744875624D696E696D615E
:101550000206434F525F5631434F525F5632464464
:101560005F563320030748385F3344202048323029
:10157000482020204832304D696E694833304D692B
:101580006E6907064341425F5633435F54454C45FD
:101590004D2D20202020202D20202020202D2020F7
:1015A0002020202D2020202020465F5341464555F5
:1015B0004E42494E440306513330332020435833C2
:1015C00035202043583130442043583130574405AA
:1015D00006574B32383031574B3234303157365F43
:1015E000355F3157365F365F3157365F48454C5768
:1015F0003648454C4902045132323251323432516C
:10160000323832030750574D4942555350504D49D7
:1016100042555350574D5342555350504D534255D8
:10162000530206484F4E5441494A4A5243583120CA
:10163000205835433146513737375F010546593316
:10164000323646593331390505574C48303858360B
:101650003030205838303020483236442045303140
:101660003020483236574804054D54202020483752
:10167000202020595A2020204C5320202046593821
:101680003035030543485F313643485F38204555C0
:101690005F313645555F38200106426179616E67DA
:1016A00048385333442002054347303233594438D5
:1016B000323948385F33440607475245454E2020AB
:1016C000424C5545202020444D30303720202D2DD0
:1016D0002D202020204A333031355F314A333031DC
:1016E000355F324D4B33333034310105534C542088
:1016F000205649535441010753594D415820205316
:10170000594D415835430106574C544F595346459E
:10171000494C554E040759443731372020534B5913
:10172000574C4B5253594D4158342058494E5855F7
:101730004E204E494855492020030744534D322D31
:10174000323244534D322D313144534D582D3232C3
:1017500044534D582D313101054869736B79484B1D
:101760003331300204483130374833303148353076
:10177000310406466C79736B7956397839202056D6
:1017800036783620205639313220204358323020E6
:1017900020566F696365004C2E53776974636865E2
:1017A000730044696167416E610044696167537702
:1017B00074636800417564696F486170746963009F
:1017C00043616C6962726174696F6E00436F6E741D
:1017D000726F6C7300416C61726D7300486172646A
:1017E000776172650047656E6572616C005665725F
:1017F00073696F6E00547261696E6572004469733B
:10180000706C617900802D814954524541475B4D90
:10181000454E555D205748454E20444F4E450045A6
:101820004449540053454C4543540053454C2F45BF
:1018300044495400434F5059004D4F5645004445CC
:101840004C455445004241434B555000524553547A
:101850004F5245004544495400494E5345525400A7
:10186000434F5059004D4F56450044454C45544553
:1018700000434C45415220414C4C001208120008D4
:101880001C0808081C080000082200490022080063
:1018900000000000227F22000000082200490022F0
:1018A00008000008220049002208000000227F22D0
:1018B0000000000000082200490022080000081C67
:1018C0000808081C08005343004756000546656594
:1018D0007420566F6C74734465675F434465675F3B
:1018E000466D41682020416D7073204D65747265AE
:1018F0005761747473465643466D416D5718242FD3
:101900002F0033383B4D697865720054656D706CFB
:101910006174657300014E595402062D2D2D2D2D35
:101920002D4E756D62657220417564696F540206B3
:101930004E6F202020204265666F72654166746597
:101940007220047349447873544852735255447357
:10195000454C457341494C734745417354524E01C0
:101960002B2A5266030420203130203130302035BC
:101970003030313030305A0306202032352D3820B7
:1019800032352D31363230302D31363530302D3143
:101990003648010546697273744C617374206601A0
:1019A00004506C61794D7574654261636B757000AC
:1019B00001524554410050726F746F636F6C004761
:1019C0006C6F62616C566172730053616665747905
:1019D00020537773004375727665004375727665A0
:1019E00073004D6F646573004578706F2F4472000B
:1019F00048656C69205365747570004C696D697435
:101A000073004D6F64656C2053656C656374004DA5
:101A10006F64656C205365747570004C617374203D
:101A20004D656E7500526164696F20536574757001
:101A300000537461746973746963730042656570FF
:101A400020636F756E74646F776E004D696E757488
:101A500065206265657000032D2D2D52746D4574EF
:101A60006D54746D41746D52454E527564456C658C
:101A700054687241696C503120503220503320003C
:101A80000420204F4E204F4646424F544820414CA0
:101A90004C4F4E434500072D2D2D2D202020763E06
:101AA00076616C2020763C76616C20207C767C3ED2
:101AB00076616C7C767C3C76616C414E44202020C3
:101AC000204F522020202020584F522020202076C6
:101AD000313D3D7632207631213D76322076313EE1
:101AE0007632202076313C763220204C6174636857
:101AF0002020462D466C6F702054696D654F6666D8
:101B000076603D76616C20004E616D650006576120
:101B1000726E31205761726E3220436865657020A5
:101B200052696E672020536369466920526F626F65
:101B3000742043686972702054616461202043728C
:101B400069636B74536972656E20416C6D436C6B95
:101B50005261746174615469636B202048617074D0
:101B60006331486170746332486170746333005448
:101B7000696D6572000354783D53777200204142CD
:101B8000434445464748494A4B4C4D4E4F505152AD
:101B9000535455565758595A61626364656667686D
:101BA000696A6B6C6D6E6F7071727374757677782D
:101BB000797A303132333435363738395F2D2E006B
:101BC000FEFFFDF6F7F8F9FAFBFC042D2D2D2D5440
:101BD000494D3154494D3242415454477672314750
:101BE000767232477672334776723447767235476B
:101BF0007672364776723700032D2D2D783E307879
:101C00003C307C787C663E30663C307C667C633160
:101C10002063322063332063342063352063362011
:101C20006337206338206339206331306331316397
:101C3000313263313363313463313563313663318B
:101C400037000450312020503220205033202048CB
:101C5000414C4646554C4C4359433143594332431A
:101C600059433350504D3150504D3250504D3350F8
:101C7000504D3450504D3550504D3650504D3750DA
:101C8000504D3843483120434832204348332043A5
:101C900048342043483520434836204348372043C2
:101CA0004838204348392043483130434831314394
:101CB0004831324348313343483134434831354366
:101CC000483136535743484756312047563220470C
:101CD000563320475634204756352047563620473E
:101CE000563720544849530067656E7772697465AA
:101CF000206572726F7200454550524F4D20466FFD
:101D0000726D617474696E6700426164204545704C
:101D1000726F6D204461746100434845434B204D10
:101D20004F44454C2054494D455253004348454388
:101D30004B204D49582F445220534F555243455341
:101D4000004D4F44454C2020202020004D452020B0
:101D500020202020202000454550524F4D206F76F6
:101D60006572666C6F7700E2AEA1A6A4A2C02F25B3
:101D7000AF000000000000000000000000000000B4
:101D800000000000000000000B07000000C0C0C001
:101D9000C0C0C0C000000000000000000000000043
:101DA000000000000006060000000080E0781E062B
:101DB000181E0701000000F8FC8EC66EFCF8070F25
:101DC0001D181C0F07080CFEFE00000018181F1F2E
:101DD0001818000C0E86C6EE7C381E1F1B1918182A
:101DE0001806C6C6C6EEFC38181818181D0F07C00E
:101DF000E0B0988CFEFE01010101011F1F7E7E668E
:101E000066E6C686060C18181C0F07F8FCE666E6A0
:101E1000CC88070F1C181C0F07060606C6E67E1E98
:101E2000001C1F0300000038FCEEC6EEFC38070F54
:101E30001D181D0F0778FCCE86CEFCF8040C1D196A
:101E40001D0F0700000030300000000000030300F9
:101E500000E0F89C869CF8E01F1F0101011F1FFE97
:101E6000FEC6C6EEFC381F1F18181D0F07F8FC0E23
:101E7000060E0C08070F1C181C0C04FEFE060E1C98
:101E8000F8F01F1F181C0E0703FEFEC6C6C6060686
:101E90001F1F1818181818FEFEC6C6C606061F1FF4
:101EA0000000000000F8FC0E06CECCC8070F1C187E
:101EB000181F0FFEFEC0C0C0FEFE1F1F0000001F47
:101EC0001F0606FEFE06060018181F1F1818000041
:101ED000060606FEFE060E1E18181F0F00FEFEF078
:101EE000381C0E061F1F03070E1C18FEFE00000004
:101EF00000001F1F1818181818FEFC187018FCFE98
:101F00001F1F0000001F1FFEFC70C080FEFE1F1F71
:101F10000000030F1FF8FC0E060EFCF8070F1C183C
:101F20001C0F07FEFEC6C6EE7C381F1F0000000017
:101F300000F8FC0E060EFCF8070F1C1B1E0F1BFE04
:101F4000FE86C6EE7C381F1F03070E1C18387CEE79
:101F5000C6C68E0C0C1C18181D0F070606FEFE06C2
:101F6000060000001F1F000000FEFE000000FEFE35
:101F7000070F1C181C0F07FEFE000000FEFE0107E5
:101F80000E180E0701FEFE008000FEFE1F0F060366
:101F9000060F1F1E3EF0E0F03E1E1E1F0301031F32
:101FA0001E7EFEC0C0FE7E0000001F1F0000000657
:101FB00086C6E6F67E3E1F1F1B1918181800000083
:101FC00000000000181818181818180060606060E9
:101FD000E0C0060F1F1B1B1F1FFEFEE060E0C0805D
:101FE0001F1F1C181C0F07C0E0E06060E0C00F1F3F
:101FF0001C18181C0C80C0E060E0FEFE070F1C18C7
:102000001C1F1FC0E0606060E0C00F1F1B1B1B1B7C
:1020100001C0F8FCCEC60E0C001F1F00000000C05F
:10202000E0703070E0C003C7CECCEE7F3FFEFEC054
:10203000E0E0C0801F1F0100001F1F000060E6E6F7
:1020400000000000181F1F180000000000E3E3005C
:10205000307060607F3F00FEFEC0E07038181F1FC8
:1020600003070E1C18000006FEFE00000000181FEB
:102070001F1800E0E060C060E0C01F1F0001001FEB
:102080001FE0E0C0E0E0C0801F1F0100001F1F80B4
:10209000C0E060E0C080070F1C181C0F07E0F07064
:1020A0003070F0E0FFFF0E0C0E0F07E0F0703070A4
:1020B000F0E0070F0E0C0EFFFFE0E0C06060E0E014
:1020C0001F1F0000000000C0E06060606060191B1E
:1020D0001B1B1B1F0E6060FEFE60600000000F1FD8
:1020E000181C0CE0E0000000E0E0070F1C1C0E1FB5
:1020F0001FE0E0000000E0E001070E180E0701E01D
:10210000E0000000E0E00F1F180E181F0F60E080D5
:102110000080E060181C0703071C18E0E0000000C6
:10212000E0E007CFCECCEC7F3F6060606060E0E035
:102130001C1E1E1B1B191900000000000000006F70
:10214000000007000700147F147F14242A7F2A123E
:10215000231308646236495522500005030000002D
:102160001C2241000041221C0014083E08140808EB
:102170003E080800503000000808080808006060A9
:1021800000002010080402003E49453E0000427F46
:102190004000625149460041494936001814127FF7
:1021A0000027454539003E494932000179050300C1
:1021B00036494936000649291E000036360000001F
:1021C0005636000008142241141414141441221429
:1021D0000800020151090600060909067E090909DD
:1021E0007E7F494949363E414141227F4141221C7F
:1021F0007F494949417F090909013E4149497A7F9F
:102200000808087F00417F41002040413F017F08CE
:102210001422417F404040407F020C027F7F04082F
:10222000107F3E4141413E7F090909063E4151214F
:102230005E7F09192946264949493201017F01017A
:102240003F4040403F1F2040201F3F4030403F6301
:102250001408146307087008076151494543007F5B
:1022600041410002040810200041417F00040201A6
:1022700002044040404040080408100820545454D0
:10228000787F484444383844444420384444487FA4
:102290003854545418087E0901020C5252523E7FA1
:1022A0000804047800447D40002040443D007F1035
:1022B00028440000417F40007C041804787C080416
:1022C000047838444444387C14141408081414184E
:1022D0007C7C080404084854545420043F444020A3
:1022E0003C4040207C1C2040201C3C4020403C4482
:1022F000281028440C5050503C4464544C4400086E
:1023000036410000007F0000004136080008082226
:102310001C08081C22080804027F020410207F20E9
:10232000101830180C06010204081020408040806C
:102330000804201002019CCE003264E2F1003264F5
:10234000645A505A6450463C46649C141E465A5384
:102350006572766F2054657374283829005365724E
:10236000766F205465737428313629004779726F6F
:102370002053657475700048656C692053657475E9
:102380007000456C65766F6E5C44656C74610056D8
:102390002D5461696C00537469636B7920542D432B
:1023A000757400542D4375740053696D706C65200D
:1023B000342D434800A923A32396238F2382237718
:1023C000236C235D234F230000891112239B3224A9
:1023D00046AD573665BF74488CC19D5AAFD3BE6CAD
:1023E000CAE5DB7EE9F7F800DA7911241FBECFEFEA
:1023F000D0E1DEBFCDBF11E0A0E0B1E0ECE9F5EF48
:1024000002C005900D92A231B107D9F71EE0A2E1FA
:10241000B1E001C01D92A336B107E1F713E2CAEEA5
:10242000D3E204C02297FE010E94977AC83ED107EA
:10243000C9F70E9481780C94CC7A0C940000E0914A
:10244000790694E0E99FF0011124E80FF11DE453AF
:10245000FD4F84918F5F0895F8948091560D90916F
:10246000570D78940895E82FF0E0EE55FD4F8491D4
:1024700008952AE0829FC001112485599D4F089537
:1024800090917B0691708091C20586FB882780F928
:10249000892708950F93022F24FF03C00F7E9DE22A
:1024A00001C094E2411104C024E042EB52E00EC0AE
:1024B0004530A0F49091C20594FF0BC0006194E0F8
:1024C000499FA00111244057594F24E00E94BA6748
:1024D0000DC02FEF240F4CED52E006C0941730F0E2
:1024E0002BEF240F42E45CE10E94DE670F91089518
:1024F000442311F04C5E01C040E0CCCFCF93DF937A
:10250000EAE8F1E08091A406108291E0918381FFD6
:102510000AC092E2928393E29383EF01259694E2BC
:10252000948345E005C0EF01239692E0928341E059
:1025300082FF0AC09FE1988390E29983FE0133965F
:1025400091E29A83486004C0FE01319693E098833B
:1025500094E0908395E0918396E0928384FF0AC093
:1025600095E2938396E29483EF01269697E2958312
:10257000406104C0EF01249697E0938385FF0AC071
:1025800098E2988399E29983DE0113969AE29A83FE
:10259000406204C0DE01119698E0988399E09C9314
:1025A000FD0186FD02C0319604C032969BE2ED012A
:1025B000998387FF03C08CE280833196DF018AE034
:1025C0008D938F5F8631E1F78487CF018E579140DD
:1025D00080935C0127E1258750E099270196252FFC
:1025E00030E08217930754F0F901E657FE4FE0817F
:1025F000F0E0E35AFE4F50835F5FF1CF8091A80671
:1026000080FF0AC0909164009B7F9093640090913A
:10261000650094609093650081FF02C0BF98C79ADF
:1026200082FF02C0A498AC9A40935B01DF91CF91E6
:10263000089587FF03C0819591E001C090E0E82FE5
:10264000FF27E7FDF095E35AFE4F808191118195B8
:10265000089587FF03C0819591E001C090E0E82FC5
:10266000FF27E7FDF095E657FE4F80819111819598
:1026700008950F931F93CF93DF93D62FC42F022F6C
:1026800016E0180F442339F0463141F04A3E81F4F8
:1026900042EF52E005C043EB52E002C04EEE52E082
:1026A0006D2F812FDF91CF911F910F910C94F067C7
:1026B00047FF04C041E20E942D67C1952FEF2C0F08
:1026C000273114F026EF2C0F46EF52E06D2F812FAB
:1026D0000E94DE67DF91CF911F910F9108950F93B4
:1026E0001F93CF93DF93D82F162FC42F022F4D3275
:1026F00034F04DE682E18D0F0E942D67CC52202FE1
:102700004C2F612F8AEF8D0FDF91CF911F910F9189
:10271000B0CFDF92EF92FF920F931F93CF93DF938F
:10272000D82F162FF42E27FF03C0EBE0F2E002C0F3
:10273000E6E0F2E0C281D3802370E22E81E08217CE
:1027400018F1C4306CF483E0C802A0011124425790
:102750005D4F0F2D23E0612F8D2F0E94BA6718C0A7
:10276000CD5F0F2D2C2F48EF5BE1612F8D2F0E9445
:10277000DE67C0310CF4D6502F2D45E2612F82E187
:102780008D0F0E942D6704C082E028130AC004C088
:10279000E11007C0C13029F42F2D4D2D612F8D2F51
:1027A0009EDFDF91CF911F910F91FF90EF90DF900F
:1027B0000895873038F4E82FF0E0EE0FFF1FE15D59
:1027C000F74F24C08C3050F18431C0F4482F50E0D2
:1027D000DA01AA0FBB1FA45FBE4F2D913C9180313F
:1027E00048F4FA01EE0FFF1FE15BF94F8081918100
:1027F000281B390BC901880F991F0895843248F4AA
:10280000E82FF0E0EE0FFF1FE951F84F8081918132
:1028100008958E3218F484520C94D72480E090E00E
:1028200008950E947D78882311F0A895FACF109220
:10283000860D08951F93CF93DF93EC01162F0E940E
:10284000E466BE0188E10E94156812FF04C067E1DA
:1028500082E10E94EA7710FD11C011FF06C068E70F
:1028600072E080E30E94156806C04AE652E068E321
:102870008CE10E942B6847EB52E002C042E652E036
:1028800024E060E086E1DF91CF911F910C94F06726
:1028900061E0D0DF0C942F6B90917906917082E00B
:1028A000891B0E946E3F2091C20525FF05C00F962F
:1028B0004F9728F080E0089581319C4FDCF781E04C
:1028C00008950F93262F00E046EF52E060E10E944A
:1028D000DE670F9108950F931F93CF93DF93C6E1A7
:1028E00010E08C2F0E940D6C110F182BC150CE30B0
:1028F000C1F78091A40682FF12C08FE10E94F86C9C
:1029000024E0829FE0011124137CC12B84E00E940B
:10291000F86C20E1829FC00111241C2F182B85E246
:102920000E94F86C082F88E20E94F86C94E0899F5E
:10293000E0011124C02B82E20E94F86C20E1829F0A
:10294000C00111248C2B982F8827812BDF91CF91E8
:102950001F910F91089520910005482F50E0FA0132
:10296000EA5DFC4DE49190915B01E923F1F0811166
:102970000CC08091A40682FD0EC025FF02C082E03B
:10298000089524FB882780F90895833049F0209129
:102990001206823019F422952F7004C0853011F48C
:1029A00026952695822F8370089530E04150510975
:1029B00002C0359527954A95E2F7922F833018F09B
:1029C000969596959695892F817090FDD8CF08950C
:1029D00070E0882399F090E0019725E0289FF001AE
:1029E000299FF00D1124E60FF71FEE0FFF1FEA5E7F
:1029F000FA4F808191818B509E4F0895FB01ED5CD1
:102A0000FB4F8081992787FD909508951F93CF9361
:102A1000DF93D82F162FC4E0DD2391F0612F8D2F87
:102A2000D7DF9C01253F81E0380764F08BE0820FFF
:102A30008D1710F08CE0820FC15029F0D82FECCF09
:102A4000C0E001C0CD2F8C2FDF91CF911F91089551
:102A5000CF93C62FDBDF6C2FCF91BACF83382FEF08
:102A6000920714F483E89FEF8E37910514F08DE7F9
:102A700090E008950F931F93CF93DF93182F062FA5
:102A8000EA01882311F0C2DF182FCE01E7DFAC0185
:102A9000602F70E01123A9F0212F30E0215031097F
:102AA00085E0829FF001839FF00D1124E60FF71F50
:102AB000EE0FFF1FEA5EFA4F455F5140518340839E
:102AC00004C0FB01ED5CFB4F808386E0DF91CF917A
:102AD0001F910F910C940961AF92BF92CF92DF9238
:102AE000EF92FF920F931F93CF93DF938C017B01A3
:102AF0006A01A22EB09011029B2D9F7D943439F073
:102B000080910D08882309F498C0933479F4B19921
:102B100006C080913D01E801C80FD11D02C0E80147
:102B2000219683E10E94E07785E010C0953419F08A
:102B3000923409F088C0B19983C080913D01E801C9
:102B4000C81BD10984E10E94E07784E00E940D6CEB
:102B5000811168C0E114F104F9F481E0C816D104D0
:102B6000D9F480E6B81619F08EE2B81211C01092AE
:102B70000D08C1E00115110509F0C0E0D0E08B2D72
:102B80000E94196D8EE2B81206C01092440803C06C
:102B9000C170DD2701C0B12C40914001509141012D
:102BA000C41BD50B80914408813071F440911A0206
:102BB000B19905C084E14802A001112403C0552742
:102BC00047FD5095C40FD51FCC16DD0644F48B2D60
:102BD0000E94196D83E10E94E077E6010AC0CE15DC
:102BE000DF053CF48B2D0E94196D84E10E94E07793
:102BF000E701C017D10749F1B19903C08FEF809366
:102C0000C106209751F48B2D0E94096D17FF02C059
:102C100083E101C084E10E94E0778A2D83700E94E5
:102C2000096113C0CC27DD27C01BD10B85E00E94B2
:102C3000196D84E00E94196D8DCF953421F47BCFFE
:102C4000E80121977FCFE80185CFCE01DF91CF91B9
:102C50001F910F91FF90EF90DF90CF90BF90AF90BA
:102C60000895552747FD5095772767FD709599275B
:102C700087FD909531CF20910608F3CF462F209104
:102C8000060860E0EECF462F50E02091060860E095
:102C900070E022CF90914901911103C0811106C0CB
:102CA0000895811103C08FEF890F01C080E08093E8
:102CB00049018EEB809348010895E0914901F0E0CD
:102CC000EE0FFF1FE15BFE4F918380838FEB8093BC
:102CD0004801089580917D062AEF829FC00111244A
:102CE000880F991F20913A0130913B01281739072D
:102CF00020F490933B0180933A010895ECE2FEE0CA
:102D000037A1303180F420A541E0420F40A7DF0118
:102D1000A20FB11DA20FB11D8D939C93403108F0FD
:102D200010A63F5F37A3089590E08C5F9E4FE6CFDB
:102D300090E0E4CF80931C0290E04097DFCF0F93A8
:102D40001F93CF93DF93EC018091840681FF07C12D
:102D50008091920686FF89C012E001E00E94F56D25
:102D60008F3F2FEF920781F029A9211104C08F31E5
:102D7000A9F709ABF3CF213011F419ABEFCF223013
:102D800069F78AAB19AAEACF8EA1813041F53FA13C
:102D9000332309F452C029A5FE01E20FF11DE20F11
:102DA000F11D808191812F5F203108F020E029A75B
:102DB00031503FA32091CC0121FDE0C097FD02C01E
:102DC00021E101C028E22BA32FE12AA722E02BA7B3
:102DD0008CA79DA718AA84E08FA72EA32EC08111CF
:102DE00006C08091550D8D3340F186E025C08230BC
:102DF00021F19AA99078833049F4992329F08BA185
:102E000081508BA3811119C084E016C0843021F455
:102E1000992399F083E00EC0853039F48BA181505D
:102E20008BA381110AC081E007C0863031F4992359
:102E300021F084E18BA385E08EA38EA1823009F47A
:102E40009DC08BA98F5F8BAB8A3008F497C01BAAFB
:102E50008DE18AA781E08BA798A1911101C080E044
:102E60008CA718AA83E08FA789C098A189A199236C
:102E700011F0846001C08B7F89A38EA1813081F520
:102E8000C79A2FA1222349F189A531E0380F39A72C
:102E9000FE01E80FF11DE80FF11D808191819DA3D6
:102EA0008CA3303108F019A621502FA32091CC011A
:102EB00021FD64C097FD02C021E101C028E22BA3DF
:102EC00029A12C7F97FD226029A389A18BBBC798DC
:102ED0008FE18AA382E08EA351C089A18BBB4DC034
:102EE00081110CC0C79A89A1836089A38BBB809193
:102EF000550D8D3308F441C086E02FC0823009F4AF
:102F00003DC089A18BBBC79ABF9800C0000000C01C
:102F100086B38078BF9A9EA1933049F4882329F024
:102F20008BA181508BA3811128C084E016C09430FE
:102F300021F4882311F183E00EC0953039F48BA180
:102F400081508BA3811119C081E007C09630A9F48C
:102F5000882399F084E18BA385E08EA30EC0809135
:102F6000A80681FD0BC08091810686FB882780F929
:102F700098A1981711F0C79A01C0C798DF91CF9117
:102F80001F910F9108959091790690FD02C093E0F2
:102F90008927E82FF0E0E35CF74FE081E7FDE95F88
:102FA000E595E595E5951E1624F0EE2321F0E195D3
:102FB00002C080E801C080E0E83008F0E7E0F0E01F
:102FC000E556FD4FE491EE2319F099E090935901F5
:102FD0008E2B0895853030F46FEF680F80911107C4
:102FE00037DD24C08D3080F4E82FF0E0EE0FFF1FB6
:102FF000ED5DF74F8081918197FD079653E09595A0
:1030000087955A95E1F712C08D3170F4E82FF0E002
:10301000EE0FFF1FEB50F84F808191816AE070E066
:103020000E94447ACB0102C080E090E017CD482F87
:10303000833021F0882321F0E82F03C0E0E001C0B5
:10304000E3E0F0E0EE0FFF1FED5EFE4F8081918127
:10305000443080F42091930630E002C035952795E6
:103060004A95E2F720FF06C020E038E0A901481B9E
:10307000590BCA0108951F93CF93DF9310E0C0E866
:10308000D0E0812FD4DFC80FD91F1F5F1430C9F7DC
:103090008D2F90E0DF91CF911F910895E3E1F1E052
:1030A00040E0842F806487B9369A3699FECF24B1E8
:1030B00035B1369A3699FECF84B195B1820F931F00
:1030C000819391934F5F483061F7089578941F92F0
:1030D0000F920FB60F9211248F93809112018F5F80
:1030E000809312018F910F900FBE0F901F90189533
:1030F00078941F920F920FB60F9211242F938F93F3
:103100009F93CF93DF93EF93FF93F89487B78F7BD1
:1031100087BF78942091D0018091D201909184064C
:10312000882369F0222359F090FF07C08091620E36
:10313000820F8093620E87FF02C01B9A01C01B980A
:1031400091FF50C08091920686FF22C0ECE2FEE023
:1031500087A5882309F446C080911002811142C0DE
:1031600080919B0085FF0DC080A991E0980F90ABE6
:10317000EF01C80FD11D8AA580939C0087A58150BF
:1031800087A787A581112EC086A1823059F526C058
:1031900080913F09811126C0ECE2FEE086A18230D9
:1031A00009F583A1882311F081501BC021A1C79A82
:1031B00082A180FD09C02D7F84A195A196FD22608A
:1031C000880F991F95A384A381E082278BBB81A3DD
:1031D000C79882A1815082A3811104C083E086A395
:1031E00085E083A3F89487B7806487BF7894FF91C4
:1031F000EF91DF91CF919F918F912F910F900FBE03
:103200000F901F90189578941F920F920FB60F92FF
:1032100011242F933F934F935F936F937F938F93DB
:103220009F93AF93BF93EF93FF9381B7845681BF72
:103230008EEC91E00E9427760E94286D80918F0D80
:10324000826080938F0DE2E0F1E08081815011F087
:10325000808304C084E6808381E081838281815001
:1032600011F0828305C08AE0828383818160838339
:10327000FF91EF91BF91AF919F918F917F916F914E
:103280005F914F913F912F910F900FBE0F901F9024
:10329000189578941F920F920FB60F9211242F93C6
:1032A0003F934F935F936F937F938F939F93AF93CE
:1032B000BF93EF93FF932091800030918100F894A9
:1032C00080917D008F7D80937D0078948091BE06F3
:1032D0009091BF06A901481B590BCA019695879585
:1032E0003093BF062093BE06409123019C01215AD2
:1032F0003F402F3D3E4230F12FEF240F283028F57C
:103300009C012152334027373540F0F424E62093C6
:103310001B02E42FF0E0EE0FFF1FEE5DFE4F9C015D
:103320002C5D354050917F06565F529FC001539FE0
:10333000900D11246AE070E00E94447A71836083EA
:103340004F5F03C041E001C040E040932301F89487
:1033500080917D00806280937D007894FF91EF9151
:10336000BF91AF919F918F917F916F915F914F919D
:103370003F912F910F900FBE0F901F90189592ECD8
:10338000980F81E0973008F080E00895FC0180817B
:10339000882359F0843218F085520C940625815008
:1033A00008DA40E060E00C94F27708959C0155E063
:1033B000359527955A95E1F7280F391FAC01440F31
:1033C000452F441F550B241B350B892F990F990B43
:1033D0008595820F931F08959DE7980F9B3F88F076
:1033E0008E57E82FF0E0EE0FFF1FE85FFA4F808165
:1033F00086171CF46083862F0895481714F44083C1
:10340000842F089544E66CE9E7CF982F80916202FB
:1034100084FF03C081E0923009F080E0089549E222
:10342000840290011124359527953595279587FDC0
:10343000815C86FB880F880B80F9A901481B510924
:1034400087FD5395CA0108954F925F926F927F92C4
:103450008F929F92AF92BF92CF92DF92EF92FF92A4
:103460000F931F93CF93DF93782E642E882309F454
:10347000D7C086E1781621F09AEE791203C0D2C047
:1034800081E0D6C0872D992787FD909597FF03C0CF
:10349000919581959109873191056CF00E944D6C51
:1034A000982F81E017141CF49111C2C0BBC099235E
:1034B00009F4BEC0B7C0872D87FD81958A3040F4DE
:1034C000825F0E940D6C17140CF4B2C091E0A6C08C
:1034D0008A50E82EF12C6701CC0CDD1CE601CE0DE4
:1034E000DF1DC955DB4F8A818F7009F49BC094E0C2
:1034F000961530F4F701E455F94F908191708BC027
:10350000588049800E943312811107C08FEF850DCA
:1035100050D98C01898183DF0EC0823041F48FEF56
:10352000850D47D98C018981815043D904C080E041
:1035300090E000E010E02A812F70822E912CF4019F
:103540003197EE30F10508F071C0EA5BFF4F0C9443
:10355000957A17FF35C011950195110931C017FFF4
:1035600033C01195019511092FC001E0060D402FC0
:1035700060E0852D69DF182F402F60E0842D64DF27
:103580002A812F70253061F4112309F44FC088235C
:1035900009F44CC08A8182958F7059F591E031C051
:1035A000263019F41111F6CFF2CF982F91271EC0B3
:1035B00008171907D9F5EECF0817190759F736C0BC
:1035C000801791073CF332C0081719071CF32EC06F
:1035D000F601EC54FE4F91819095991F9927991F00
:1035E00005C0F701E455F94F908191709111D2CF48
:1035F00008C089300CF08F5F41E0460D60E024DFA9
:10360000982F2A812F7030E02C30310524F4F701F7
:10361000E455F94F908317143CF081E0892708C0E6
:10362000862F06C080E004C0892F02C090E0E9CF59
:10363000DF91CF911F910F91FF90EF90DF90CF908E
:10364000BF90AF909F908F907F906F905F904F90C2
:10365000089540E060E0F8CE80916606FADF8111BF
:1036600013C080913A0190913B01892B69F410922B
:103670004C0E8091550D9091C006981749F080939B
:10368000C0068CE29EE05BCB81E080934C0EF1CFD4
:103690000895CF9320914E02222331F0909350024F
:1036A00080934F02CF91089564E0C4D80E942F6B9D
:1036B00089E10E94FD6AB5D8C1E00E947D78882327
:1036C00011F0CF91AEC880918F0D833019F4A89579
:1036D00010928F0DC0934C0EBFDFEFCFE0914901E8
:1036E000E43018F08FE092E0D4CF2FEB2093480124
:1036F000EF5FE0934901F0E0EE0FFF1FE15BFE4F4B
:103700009183808308958091780680FD16C0C6DC81
:10371000C3D8811112C066E081E492E08BD80E9488
:103720002F6B7FD8BBDC98DFA895B6D8811105C078
:103730000E947D788823B1F374C80895FF920F9397
:103740001F93CF93DF938091780681FD3FC08091D6
:1037500000059091A40692FD0CC0982F98739830A4
:1037600041F0903131F0903221F0877C8860809375
:103770000005C0E011E06C2F62608CE192E05AD845
:10378000D2E0C0E000E08C2FE6D8F82E8C2FCDD709
:103790008F1531F04C2F60E18D2F0E94623501E0D2
:1037A000CF5FDB5EC63079F70E942F6B002371F08C
:1037B0000E947D7881110AC0112331F032D8C4E013
:1037C0004BDFA89510E0D7CFC0E0FACFDF91CF91C3
:1037D0001F910F91FF90089581117CDA80913A0139
:1037E00090913B01009709F0019720913901222324
:1037F00061F0209185064AEF249F90011124220F49
:10380000331F8217930708F4C90190933B018093FB
:103810003A0122CF1F93CF93DF93CEE1D5E090E022
:10382000888111E0190F882329F013DF882311F014
:10383000812F05C0912F2A96143091F780E0DF91F7
:10384000CF911F9108958F929F92AF92BF92CF9286
:10385000DF92EF92FF920F931F93CF93DF93EC01D0
:10386000A62EB12C6501CC0CDD1CF601E35EFD4FEC
:10387000008111818981882309F457C08D809E8041
:10388000888181500E94D9137C018981853038F468
:10389000833050F4813079F0823091F039C0853036
:1038A000A1F0863071F134C0F7FE03C0F194E194C9
:1038B000F108833029F481E08E149F043CF125C087
:1038C00081E0E814F90414F120C0888158DD8823D0
:1038D00069F08AE09701829F7001839FF00C1124A8
:1038E000F4018E9F40018F9F900C1124E818F90875
:1038F000FFE1EF0EF11C81E02FE3E216F10430F05E
:1039000004C081E0E814F90409F080E0E82EF12C0D
:103910008A81811104C0EF2829F081E01BC099DE63
:103920008111F9CF00E010E014C08A81882331F0C2
:1039300090DE81110BC00FEF1FEF0CC08B81843024
:1039400040F09C81907681E029F403C080E091E012
:1039500002C080E090E0892BF501E35DFD4F5F013F
:10396000F080209105019B8121FD2EC0933059F4F8
:103970008A810E94F86CF81689F1FF24F394F80EFE
:1039800000E010E02CC0813041F4F11003C0292F79
:103990002D7FB1F0913089F421C0F1E0FF120CC00D
:1039A0008FEF890F823040F480E000E010E0923029
:1039B000B1F462E0F62E13C080E0913219F40CC02D
:1039C00000E010E0F82E0BC0FF24F394913209F0D0
:1039D000F12C0FEF1FEF03C00FEF1FEFF12CF501DC
:1039E00080838C8187FD03C0F1100AC07BC0888171
:1039F0008532D0F3855263D7882309F473C0F4CF9E
:103A000017FF04C08B81833028F46CC001151105A9
:103A100009F055C08C818076803211F4CE01B6DC7D
:103A20008C81877059F1813021F52F81822F988503
:103A30008C3FF1E09F0740F040E050E060E070E034
:103A400084E0820FC2D60DC0853F21E0920748F086
:103A5000FC01EE0FFF1FE25EFE4F8081992787FD7C
:103A600090952F2D30E021503109820F931F46D9B8
:103A700005C060E070E08F810E94E5778C818076E0
:103A8000803411F4CE0182DC8C81282F287181F0E2
:103A9000869586958695837090E0029724F028316C
:103AA00021F48FE003C08DE001C08EE00E94E0773A
:103AB0008B8183508E31A0F00FEF1FEF13C01016D3
:103AC000110684F40F5F1F4F8B813AE0839FC00182
:103AD00011244397081719072CF000E010E002C0EA
:103AE00001E010E0F601E35EFD4F11830083DF91FA
:103AF000CF911F910F91FF90EF90DF90CF90BF90EB
:103B0000AF909F908F9008951F93CF93DF93CAEC4F
:103B1000D5E010E0612FCE0196DE29961F5F1830A8
:103B2000C9F7DF91CF911F9108959F92AF92BF92F5
:103B3000CF92DF92EF92FF920F931F93CF93DF9379
:103B4000109243088091120102B7909112018913DB
:103B5000F9CF10E0182BA2DA8EE587B91BBA8FE1F6
:103B60008ABB00C099B38FEF8ABBE2E1F2E08781A4
:103B7000882311F080E202C0892F807E8483292F60
:103B8000207C8081281759F08074880F90783181CB
:103B9000891711F0315001C03F5F3183208382814A
:103BA0009381891711F0838381838091560D9091C1
:103BB000BB06282F291B2093B3018093BB0680915D
:103BC0001002811106C060E085EE97E00E949149E5
:103BD00001C0A8958091B301882309F4DAC2C4E337
:103BE000D1E080910B08882319F0815080930B0855
:103BF00042DA2B813C818217930741F09C838B83AF
:103C00001A82198281E0809339012CC060917A0672
:103C1000665F41F180913C01823320F188818F5FA2
:103C200088838031F8F089819A8101969A8389830B
:103C3000188247E751E0649F9001659F300D112481
:103C40002817390778F48F719927019759F48091D3
:103C5000CC018D7F8093CC0186E06CD86DE280E151
:103C60000E94EA770E948C330E94A73280911B0247
:103C7000882319F0815080931B020E94E466D09043
:103C8000860D1092860D809110028111B2C14D2DCA
:103C90004F70A42E5AEFA50EC0916302C43021F0DC
:103CA000C33019F4C4E001C0C8E087E08A1508F405
:103CB00095C08D2D807F803209F490C08A2D869525
:103CC0000E941F129091920690FD04C0CC24CA94C9
:103CD000C80E03C0E4E0CE2EC81A6C2D80911107E7
:103CE0000E940615B82E6C2D0E9428157C01C1116A
:103CF0000CC0EC0197FF04C0CC27DD27C81BD90BF3
:103D0000D595C795D595C795CF5F92E0C9120FC0DD
:103D10008091620280FD02C0912C03C0992493948B
:103D2000C2E00E944012882319F0C19501C0912C75
:103D3000DD27C7FDD095A0FE03C0CE0DDF1D04C05A
:103D4000F701EC1BFD0BEF01209721F08D2F8F2544
:103D500087FF11C091100FC0EF2869F040E050E0DC
:103D60006C2D8B2D0E943A158D2D0E94196D86E1C8
:103D70000E94E07757C39E0124583F4F293F3105E9
:103D800048F4AE016C2D8B2D0E943A156C2FC7FFA5
:103D900018C016C01C161D061CF44DE750E002C0EA
:103DA00043E85FEF6C2D8B2D0E943A15CE018358AE
:103DB0009F4F8B3F910508F035C36C2F1C160CF4F8
:103DC000619567FD6D5F65956595772767FD7095D2
:103DD000645C7F4F85E10E94E57724C38D2D8F7B46
:103DE00071F48091C106B19919C38F3F31F08F5F93
:103DF000883C19F48FEF6DEBD62E8093C106EEE36D
:103E0000F1E080913B0890913C0820813181281B92
:103E1000390B37FF02C0215E3F4F55E0359527959E
:103E20005A95E1F72115310561F024813581281B70
:103E3000390B37FF02C02F5F3F4F35952795918390
:103E400080839583848380917B0685FD04C0809167
:103E50000908882311F020E030E033832283C2E197
:103E6000D2E02D818981821B8F3F09F480E087FD9C
:103E70008F5F85958887982F990F920F9D838D2945
:103E8000ABDCF0909106F7E0FF0EE0914901F0E025
:103E9000EE0FFF1FE15BFE4F208131812757374432
:103EA00009F040C08091660881113CC0288522231A
:103EB00071F08E81332727FD3095F901E80FF11D50
:103EC00087FDFA95CF010E942E158E831886E0910A
:103ED000CD048E2F807E31F1E295E695E770F0E01B
:103EE000E430F10554F4EE0FFF1FEB5CF74F208137
:103EF00031813C5F60E078E00CC0EE0FFF1FEA5FAD
:103F0000FA4F2081332727FD309523583F4F6AEF22
:103F100070E047E0429FC001439F900D11240E9432
:103F2000307AF62E80911C02F81619F08F2D0E941F
:103F30009A168091810687FF3BC080915A018823A1
:103F4000B9F1809159018823A9F18091BA0687FDC2
:103F500003C08F5F8093BA0682E015D8982F9F77B1
:103F600089F02091BA06921728F51092BA06D1105E
:103F700021C0D82ED094DD1CDD24DD1C83E68D19F4
:103F8000D82E18C083E00E94C317982F9F7791F016
:103F90002091BA06921770F41092BA06D1100AC096
:103FA000D82ED094DD1CDD24DD1CF4E6DF0E02C02B
:103FB0001092590181E080935A01E0901802FF2489
:103FC000E7FCF094C9E0D5E08881882369F085306A
:103FD00029F000D8992787FD909501C0C7010E945C
:103FE0002E15FE0131978083229625E0C731D20736
:103FF00059F780914F0290915002009711F160E0C3
:104000000E941A140E947D789091B9069923A9F014
:10401000913021F4811139C082E005C0923031F431
:10402000882399F183E08093B9062FC081112DC0B8
:104030001092500210924F0228C0882369F381E049
:10404000F2CF1092B906C0914801CC2331F0109202
:10405000480187E10E94E077DC2E84E180933D01F6
:10406000D092110280914108882319F081508093E9
:104070004108E0914901F0E0EE0FFF1FE15BFE4FC8
:104080000190F081E02D8D2D09950E942F6BC0913C
:1040900065008EEC91E00E941376882311F084E194
:1040A00005C08091610E882321F081508093610EBC
:1040B00006C080916300869581708093600E809128
:1040C000600E80934D02882309F4AAC18091810675
:1040D00085FDA6C1CF7EC09365008091550D8F717F
:1040E000823009F054C08091210190912201AC01ED
:1040F000F4E0440F551FFA95E1F797FD0796BC01D0
:10410000E3E075956795EA95E1F720916506332719
:1041100027FD30952A5F3F4F629FC001639F900D3E
:10412000729F900D1124840F951F20917B0626FD10
:1041300005C0609100017091010102C060EF70E064
:104140000E94307A80913C01680F711D6F5F7F4F34
:104150007595679560933C018091B806805F809368
:10416000B806811114C080916406681780F4623328
:1041700070F06EE281E10E94EA7780917B0683FF16
:1041800006C082E390E090933B0180933A01109245
:1041900039018EE587B9369A3699FECF84B195B14B
:1041A000909301018093000180918F0D833019F469
:1041B000A89510928F0D2091120182B79091120153
:1041C0002913F9CF90E0922B801B910B20910801CD
:1041D000309109012817390720F490930901809341
:1041E000080180910501882309F40AC18091BC0669
:1041F0009091BD0601969093BD068093BC06809178
:10420000CD048F7120E1F22EF81AF7E1FF1508F4C2
:1042100069C00F2D10E0E801CC0FDD1FC253DB4F4A
:104220004FE04F1528F4E801CC0FDD1FCE5CDA4FCC
:104230008881D82ED294D694D694B3E0DB22E9803C
:1042400053E0D51651F09AEF9E1538F4EE2DF0E0BC
:10425000EE0FFF1FE85EFC4FE0808F7309F440C053
:10426000F8D9C82E809105010B5C1D4F81FD36C029
:10427000D0FC0AC0F8018081811106C0CC2021F059
:104280008E2D90E00E947E168FEF8D0D823078F497
:10429000F8018081813011F5C11020C0F2E0DF12F9
:1042A00001C0E3948E2D90E00E947E1617C023E09B
:1042B000D21214C0F8018081811110C0CC2071F09D
:1042C000898187FF0AC09091840690FF02C0809583
:1042D00001C081E00E94E07701C098D3F801C0825C
:1042E000F39493CF07EA14E0ECEAAE2EE6E0BE2E9C
:1042F000F4EBCF2EF1E0DF2EE12CF12CF8019280CF
:10430000892D8F700E9433128330D9F5F601C08158
:10431000D181209771F4F801C081C7FD06C0C09516
:10432000FAE0CF02E00111241BC0DD27C7FDD095C4
:1043300017C0D7FF14C0219699F4F701E855FB4F39
:10434000C081C7FD06C0CF5F2AE0C202E001112490
:1043500006C0DD27C7FDD095C095D09501C0219737
:10436000892D807F59F0892D82958F7089300CF0CE
:104370008F5F6FD9811102C0CFEFDFEFF601D183DC
:10438000C083F501C081F80182818F708C3071F497
:1043900080815FD9811109C0F701E855FB4F808109
:1043A00058D9882319F0C0E001C0C1E0F80182812A
:1043B0008F708D3091F480814CD9882359F0C1FDE4
:1043C0000CC0F701E855FB4F808143D9882321F0C9
:1043D000C3E003C0CD7F01C0C2E0F501C1935F011E
:1043E0000D5F1F4FF3E0EF0EF11C22E0C20ED11C57
:1043F00044E2E416F10409F081CF86DB1092050156
:1044000080910301882381F010920301809159016A
:10441000882351F081508093590106C080E0EDCC93
:10442000C06159CED12CDDCCDF91CF911F910F917E
:10443000FF90EF90DF90CF90BF90AF909F90089546
:10444000282F30E0883058F02850310949E0429F49
:10445000C001439F900D1124815A9B4F089545E060
:10446000429FC001439F900D1124895C9B4F08958A
:10447000813641F40E94196D81E00E944A1681E75D
:1044800090E52CD963EE72E180E10C941568CF932E
:10449000C82F80918D0D80FF03C069E572E102C0D5
:1044A00067E472E188E10E941568C13641F481E653
:1044B0000E94196D10928D0D80E00E944A16809125
:1044C000550D811103C081E00E94E077CF910895DE
:1044D0001F93CF93DF93182FD62FC42F662329F075
:1044E0006FE0842F0E943E16C82F809162024C2FED
:1044F00083FF02C0440FD06250E02D2F612F80E671
:104500000E94186A8C2FDF91CF911F910895FF921E
:104510000F931F93CF93DF93182FF62E0AE08AE0B4
:10452000189FE0011124C559DD4F2FE130E0211B18
:104530003109029FA001039F500D1124BE01CE013D
:104540000A960E94A47AFF2049F0BE016A507109C0
:104550004AE050E0CE010E94A47A0DC0FE01119203
:104560000A95E9F78091E0088883898384E68A8345
:104570008F8188608F831093E20882E0DF91CF9172
:104580001F910F91FF900C940961AF92BF92CF924F
:10459000DF92EF92FF920F931F93CF93DF93EC0183
:1045A000C62ED42E88E068130AC0FE013E964591BF
:1045B000549160E085E40E942B6808E001C007E0A8
:1045C00010E07801EE0CFF1C98E0A92EB12CFE0142
:1045D000659174918A2D0E941568BC1448F4FE01FF
:1045E000EE0DFF1D459154916A2D85E40E942B68C4
:1045F000B394229688E0A80E87E0B812E8CF4FE384
:1046000060E083E40E94CB68DD20A1F087E06D2D9F
:104610008D1540F4601B660F660F660F20E04BE3BC
:1046200085E406C0660F660F660F20E042E480E076
:104630000E945168DF91CF911F910F91FF90EF90F1
:10464000DF90CF90BF90AF900895E3E6F8E08F3B06
:1046500019F49091630803C08E3B29F49081915026
:1046600090934B0110829281992321F091819F7741
:104670009083128290819923B1F0813219F08E38A3
:1046800009F04AC020910D08211109C09150909362
:104690004B0110820E94196D87E10E94E077109211
:1046A0000D0880E0089590914B01843681F4292F04
:1046B00030E0683031F070E026173707FCF427E06F
:1046C00004C027303105D4F428E0920F17C0853696
:1046D00029F4292F30E06830A1F418C0803611F099
:1046E0008E3261F49F5F9083906891830E94196D70
:1046F000109211021092E40790E080E090934B0139
:10470000089527303105D4F327E004C0283031055F
:10471000ACF328E0921BF2CF0895873028F4E82FFD
:10472000F0E0EB53FD4F84910895282F30E0F9011C
:10473000EA5DFC4DE49190915B01E92331F0F901D0
:10474000E254FD4F84910C94F86CE7DF0E94F86C02
:10475000882311F080E0089582E008950F9344309B
:1047600051F4909160029F70913029F44BE354E131
:104770000F910C94F067022F242F4AEC5BE10E940A
:10478000DE670F9108959C01220F331F280F391FF8
:104790009595879595958795280F391F95958795B8
:1047A0009595879595958795820F931F08954296C5
:1047B00043E7489F9001499F300D1124C901E6E06D
:1047C00095958795EA95E1F70895CF92DF92EF925C
:1047D000FF920F931F93CF93DF937B018A01D090B9
:1047E000430895E09D1508F45FC091E09D0D9093FE
:1047F0004308EBE08E9FE0011124CC56DA4F88810C
:10480000882349F081500E94D9139C01442737FD29
:104810004095542F03C020E030E0A901D092430816
:10482000DE80FD2DF870CF2ED3FC0AC089819A81DD
:10483000AA2797FDA095BA2F280F391F4A1F5B1F83
:10484000AB81B0E011960E94027A2C8130E02F5F9C
:104850003F4F442737FD4095542F0E94797ACC2052
:1048600051F089819A81AA2797FDA095BA2F280F28
:10487000391F4A1F5B1FD0FE07C0509540953095E9
:1048800021953F4F4F4F5F4FE114F10419F08D8197
:10489000F70180830115110529F08E8186958370BB
:1048A000F8018083C90102C080E090E0DF91CF91E0
:1048B0001F910F91FF90EF90DF90CF90089581E0CE
:1048C0000895FF920F931F93CF93DF93F82E062F37
:1048D000EA018091670281FF03C060E075E002C0D9
:1048E00060E074E0AE01D7FF04C0442755274C1B9D
:1048F0005D0B89E1849FF001859FF00D1124CF01AC
:104900009E5F0E94447A162F6A310CF019E125E56A
:1049100043E3602F87EE8F0D0E948E6845E06EEFB7
:10492000600F8F2D0E94CB681C161D0614F4F394A3
:1049300001C0F11A61E0600F412F8F2D0E94C968FC
:104940006FEF600F412F8F2DDF91CF911F910F914E
:10495000FF900C94C9689C0197FF04C0222733275D
:10496000281B390B2130310511F447E201C046E222
:1049700060E00C94F277E82FF0E0E054F44EE4911C
:10498000862F992787FD90952AE02E0F273070F00B
:10499000BC0163587F4FEE5FE23038F42AE0269F77
:1049A000C001279F900D11240895CB010895E82F91
:1049B000F0E0E054F44EE491E03F29F1ED3F4CF497
:1049C000EE0FFF0BE45EFA4F8081992787FD9095EB
:1049D0000895ED3FA1F0BCF0EF3F09F0A4F48E2F55
:1049E000992787FD909502962FE0289FF001299F37
:1049F000F00D1124EB5BF74F83859485089580912A
:104A00003C0190E0089580E090E00895CF92DF921D
:104A1000EF92FF92CF93DF9300D0CDB7DEB7F82EA1
:104A20001A821982C4DFEF2DF0E0E054F44E249195
:104A3000422F552747FD5095652F752F415F5F4FDA
:104A40004F30510578F54C5A5F4FFA010C94957A26
:104A5000AE014F5F5F4FBE016E5F7F4F8FE0820FF1
:104A6000B4DEEA81F0E0E350F74EE491EA831AC045
:104A700024E22A8321E0298315C06CE370E00E94C0
:104A8000447A6B017C01CB0166DFC70125E32A83F1
:104A900009C0E22FEE0FFF0BE45EFA4F80819927E9
:104AA00087FD90954A8169810E94F2770F900F905F
:104AB000DF91CF91FF90EF90DF90CF9008950F930B
:104AC0009FE0499FF0011124EB5BF74F438554852C
:104AD000022F0E94566A0F9108958F929F92AF9273
:104AE000BF92CF92DF92EF92FF920F931F93CF93DB
:104AF000DF9300D0CDB7DEB7F82ED62EC22EB32E60
:104B0000102F80E28A83E42FFF27E7FDF095E05421
:104B1000F44EA4908E2D8170982EE0FE20C0AFE060
:104B2000AA0DA43008F08CC08BE0A89FD0011124FE
:104B3000FD01E556FA4F8081882309F481C0AF0159
:104B400000E124E08F2D0E94BA6712FD03C008E146
:104B50000F0D06C00CE10F0D88EFD80E01C00F2D10
:104B60008E2D8870882EE3FC1F7B81EFA8160CF435
:104B70003DC084EF8A152CF482E08A0D8230F8F073
:104B800035C0AE014F5F5F4FBE016E5F7F4F8FE05C
:104B90008A0D1BDE2981213011F4106203C02230FE
:104BA00009F41063E7FE02C08C2D9B2DEA81F0E032
:104BB000EB50F74EE491EA83C82EB92E17C012FDD0
:104BC00002C08CEF01C082E0800F9110865F1770E9
:104BD000012F212F4C2D5B2D6D2D83500E94566A85
:104BE0008AEFF80EE3E3EA0DEA830AC0882071F148
:104BF0008DE38F0D212F4C2D5B2D6D2D0E94186A9A
:104C00008E2D867069F0E2FE04C08AE08F0D1B7F56
:104C100002C08091420D212F4A816D2D0E942D6787
:104C20008A810F900F90DF91CF911F910F91FF908C
:104C3000EF90DF90CF90BF90AF909F908F900895AE
:104C40004F5F20E06D2D8F2D89DD7FCF802FD2CF5C
:104C50000F931F93CF93DF93C82FD62F042F122FBC
:104C600049EC58E10E94F06740E3400F212F6D2F7F
:104C70008CE08C0FDF91CF911F910F910C942D67D9
:104C8000EF920F931F93CF93DF93C42F122F2E2DEC
:104C9000DE2DD3709DE7940F9B3F80F043E84C0FCF
:104CA0008251D6DFDD2359F122E042E850E06EE781
:104CB00070E08C2F90E00E946C150CC0552747FDCA
:104CC00050950E94186ADD23D1F0402F612F8C2F60
:104CD0000E943B16C82F809111028D3B81F48DE715
:104CE0008C0F8B3F40F0EC2FF0E0EE0FFF1FE45FE6
:104CF000FB4FC08101C0CEE782E00E9409618C2F8A
:104D0000DF91CF911F910F91EF900895EF920F9344
:104D1000E22E0DE723E8B4DF0F91EF900895CF93D3
:104D2000DF939EE0899FE0011124C550DC4F8C8504
:104D30000E94291B882339F08D850E94291B81112F
:104D400004C081E003C080E001C082E0DF91CF9128
:104D5000089590911A0281E0191624F0911101C072
:104D600080E0819510921A02089521E0AC0160E084
:104D700080E00C94F0670F931F93CF93C62F0E948F
:104D8000186AB8018C2FCF911F910F910C94156860
:104D9000FF920F931F93CF93DF93182FC42FD22F1F
:104DA0006115710591F0FB018491AB014E5F5F4F7E
:104DB0003196F490222319F00091070801C000E019
:104DC0002C2F612F0E94DE6714C0442329F042E893
:104DD000682F87E60E94B867DD2311F004E601C062
:104DE00000E027E047E0612F86E60E94C76AFF24C3
:104DF000F394DD23A1F080910508882321F08091B0
:104E00000D08882361F0209106084F2D60E08C2F5B
:104E1000DF91CF911F910F91FF900C9431168C2F41
:104E2000DF91CF911F910F91FF900895E09149017B
:104E3000F0E0E65BFE4F91E03081231390E0292FF4
:104E4000A7CF982F862F242F492F60E070E0EECF58
:104E50001F93CF93DF93D82FC62F122FBA018C2F19
:104E60000E941568412F6C2F8D2FDF91CF911F91DC
:104E7000E8CFCF93C1E09C2F981B892FE9DFC81B97
:104E80008C2FCF910895CF93C1E09C2F981B892F31
:104E9000D8DFC81B8C2FCF910895982F862F242FF1
:104EA000492F61E374E174CF0F93909160029F707A
:104EB00021E0913009F020E000E045E75BE10E944D
:104EC000DE670F9108954115510519F0805F0C942C
:104ED000186A42EF52E00C94F067FF920F931F9311
:104EE000CF93DF93182F062FC091E407E09149017B
:104EF000F0E0E65BFE4FD081A0913708B091380812
:104F00004091390850913A08EEE3F1E0268137816B
:104F10002A1B3B0B37FF02C0215C3F4F96E03595C3
:104F200027959A95E1F7922F20930A0820853185DD
:104F3000241B350B37FF02C0215C3F4F86E03595BF
:104F400027958A95E1F7822F20930808992311F07D
:104F5000B783A683882311F0518740878091090881
:104F6000811104C080917B0685FF06C010920A085B
:104F7000109208081092090880910A08811108C04F
:104F800080910808811104C082819381892B11F0DE
:104F90000E946A16F090E5080F3F09F449C080911D
:104FA0004408811129C08091DE08882319F01092ED
:104FB000DE08CF2DCEDE181644F4CF1510F4CF5FE7
:104FC000A9F4D01788F4DF5F10C0882379F0C111ED
:104FD00009C0DD2311F0D15001C0D02F81E08093B2
:104FE000DE0804C0C15002C0D0E0C0E01E3271F43F
:104FF00081E0809344080AC0813041F41E3221F0E0
:1050000080910D08811102C0109244088091E3073D
:10501000B1990BC08F3F19F08F5F8D3338F091E05D
:1050200090930D089093440801C080E08093E307BB
:10503000F092050840910D08411129C0809108089F
:10504000882391F0D81BD7FDD0E0802F90E02D2F42
:10505000332727FD3095281739070CF0D02FFC1681
:1050600008F4CF2D10920808DD2389F080910A08FA
:10507000882369F0C81BC7FDC0E08F2D90E02C2F5E
:10508000332727FD3095281739070CF0CF2D103620
:1050900079F190F4123409F464C028F41132D1F19A
:1050A0001E3231F178C0143409F43FC008F466C0F0
:1050B000153409F448C06FC0153609F446C040F4F1
:1050C000133609F45EC098F5123609F44CC063C07B
:1050D0001E38E9F01F3B39F0113809F05CC010921E
:1050E0000D0881E01FC010920D08D0E0C0E053C051
:1050F0000F3F09F450C081E0411180E080930D081A
:10510000882309F448C081E08093440844C08EE8B5
:105110000E94196D80910D08882319F010920D08D6
:105120003AC080E00E944A1636C0CF15A1F1FF2098
:1051300091F1411130C0CF1510F4CF5F01C0C0E034
:105140001092110228C0CC2331F1FF2021F141112E
:1051500022C0CC2319F0FF24FA94FC0E1092110205
:105160000BC0D017C1F0411116C0D01710F4DF5F8B
:1051700001C0D0E0FC1678F4CF2D0DC0DD2359F02E
:1051800021C0411108C0DD2311F00FEF0D0FFC16F7
:1051900008F4CF2DD02F20910D0821110AC031E045
:1051A0008091400190914101892B09F430E0832FD7
:1051B00001C081E080930C08222311F082E005C039
:1051C00081E003C04111E7CFE0CF80930708109240
:1051D000E508C093E407E0914901F0E0E65BFE4F8B
:1051E000D0838D2FDF91CF911F910F91FF90089564
:1051F000AF92BF92CF92DF92EF92FF920F931F93E5
:10520000CF93DF93C82F8FEB99E1AFDD6AE08C2F4E
:1052100064DEC82EB090E40786E0CE3211F0C036CE
:1052200071F48C1578F489EF8C0D8093E6088C2F3F
:105230000E94196D87E69DE40E946E1B5EC08C156E
:1052400008F45BC081E08093E508E12CF12C18E0C4
:1052500069EC78E1812F0E941568AE2C41E34E0D78
:10526000612F8CE00E94B867E701CC0FDD1FC85F9B
:10527000DA4FD12CCA1005C0BD1003C00091070839
:1052800001C000E080910D08882309F482C0D1108C
:1052900017C0002329F06CE189810E943E168983A2
:1052A00029812D3018F447E55AE105C02D31C8F4A5
:1052B0002D5F42E45CE1612F8CE30E94DE6711C048
:1052C000002331F04DE763E888810E943B16888314
:1052D0004881552747FD5095202F612F8CE60E946D
:1052E000186AD39482E0D812C5CF185F8FEFE81AFE
:1052F000F80A103409F0ACCF41C089EFC80E04E9B8
:1053000015E021E3E22E38E0F32E6AED73E18F2DF4
:105310000E9415684E2D6F2D8CE00E94B867E80141
:1053200020E048816F2D88E10E944A1249815A810C
:105330006F2D8BE40E94466A4B8150E04F5F5F4FB8
:105340006F2D80E60E94466A4C8150E04F5F5F4FB0
:105350006F2D8EE70E94466A88E0F80EE394055FA1
:105360001F4F88E2F812D1CF6C2D660F660F660FC3
:10537000685F20E04EE780E00E945168DF91CF91A6
:105380001F910F91FF90EF90DF90CF90BF90AF9063
:105390000895D1109DCF84CF1F93CF93DF93C82F53
:1053A000D62F142F27E147E160E285EF8C0F0E9492
:1053B000BC6A43E06AE28C2F0E94CB6843E06BE258
:1053C0008FEF8C0F0E94C968812F69EF0E94237AAA
:1053D000382F375D8D2F67E00E94237A8C0F25E0F0
:1053E00045E0632F8250DF91CF911F910C949C6A0E
:1053F000CF92DF92EF92FF920F931F93CF93DF93A1
:10540000CDE3D8E0498168818AE2C6DF4A816B81B9
:1054100086E5C2DFCFE2D8E028965AE3F52E0DE507
:1054200010E067E3C62E899199919C5FB8010E94B4
:10543000447ADD24D394D60EEC2CE61A4D2D6E2D35
:105440008F2D0E94CB684D2D6E2D81E08F0D0E9417
:10545000CB684D2D6E2D82E08F0D0E94CB6885E0CC
:10546000F80E89E4F812DFCFDF91CF911F910F91F1
:10547000FF90EF90DF90CF90089542E254E168E30F
:1054800088E60C942B680F931F93CF93DF93D82F4C
:10549000162FC42F022F47FF08C041E28AEF8D0F5D
:1054A0000E942D6786E08C1BC82F2C2F48EF5BE1F4
:1054B000612F8D2F0E94DE67DF91CF911F910F9199
:1054C00008950F931F93CF93DF93162F042FC62FAA
:1054D000D0E0AE014F5F5F4F202F682F86E60E941D
:1054E000186A002329F06FEFCE010E944316182F8F
:1054F000812FDF91CF911F910F9108950F93CF933B
:10550000DF93C42FD02FD27001FF03C00E946F130E
:1055100002C00E94391300FF41C0DD23B9F1CD3232
:1055200074F084ED8C0F0E94191320915C0130E01F
:10553000280F311D87FD3A952150310907C08C2F66
:105540000E941913282F332727FD309580915C0185
:10555000482F440F4250C1E06C2F681B822F0E94DD
:105560003B1690915C01482F552747FD5095292FF8
:1055700030E0421753073CF0C91B8C0F0E942913DF
:10558000CCE2C80F0BC00E94291307C040915C01F8
:10559000642F61958C2F0E943B16C82F8C2FDF91B2
:1055A000CF910F910895FF920F931F93CF93DF93A5
:1055B000182FF62EEA01022F4981453249F4298538
:1055C00022952695277042E459E10E94DE6711C0BA
:1055D00020610E944A1289818551803150F48F8167
:1055E00086FF07C0202F4DEC53E16F2D812F0E94C5
:1055F000F067DF91CF911F910F91FF9008958091F7
:10560000A103882329F088E392E20E946E1B81E0C7
:105610000895CF93DF93C82F88E00E9415686CEC43
:1056200072E188E20E941568C13671F028F4CE322A
:1056300069F0C03659F012C0CE3831F0CF3B71F46A
:1056400080E00E94E0770AC0D2E001C0D1E08C2F58
:105650000E94196D81E00E944A1601C0D0E08D2F92
:10566000DF91CF910895CF939091E1079F3F19F477
:105670006BEB72E102C06FEA72E1CBDF813019F0AF
:10568000823019F127C0C091E107CF3F19F40E9481
:105690007E6E1BC08C2F0E9439122FE130E02C1B34
:1056A0003109CAE0C29FA001C39F500D1124BC0163
:1056B000665F7F4F0E94A47AE1EAF3E0DF011D926A
:1056C000CA95E9F782E00E94096181E790E5CF91F0
:1056D0000C946E1BCF9108950F93CF93C82F4FE07A
:1056E0006AE678E08091DE070E944F6000E12AE0E0
:1056F0004AE658E060E181E00E94BA674FE360E16A
:1057000082E40E94B8678091DF07882319F061E87E
:1057100072E102C064E772E18C2F7BDF813019F007
:105720008230F9F024C08091DF078823A9F082E657
:1057300092E10E9448148091DE070E9497608823BE
:1057400039F087E10E94E07782E08093DF0709C0AB
:1057500080E00E94E07705C08091DE078F5F0E94A5
:105760008B648FE49CE2CF910F910C946E1BCF91D0
:105770000F910895DF92EF92FF920F931F93CF93B3
:10578000DF93EC01062FD42EF62E18E0E12CFF203B
:10579000B9F0F0FE0EC02D2D40EA52E1612F82E1FA
:1057A0000E94EB67AE01612F88E10E942B68E394B1
:1057B000185FF694FE01849121968111FBCFE7CF0B
:1057C000CD2DCC0FCD0DCC0F2AEF210F4C2F67E044
:1057D00082E10E94BC6A44EF4C0F60916708660F3B
:1057E000660F660F685F20E088E10E945168B1DAB9
:1057F000282FC6E6D8E099818B81882351F030911B
:10580000550D36FF08C081508B83811104C018826A
:105810001CC08FEF8B8380911102813681F028F4B8
:10582000803249F08E3239F012C08336C9F088F0E8
:105830008E3829F00CC018821B8281E01AC00E94A9
:10584000196D1092110218821B8282E012C012168A
:105850002CF4EA949E1530F49F5F04C0222339F0A3
:10586000911191508B81882311F08FEF8B83998355
:1058700080E0909167089F5F20E000FF02C0915098
:1058800021F006952F5F2830C1F720936808DF913B
:10589000CF911F910F91FF90EF90DF900895DF92CD
:1058A000EF92FF920F931F93CF93DF93C82F84ED56
:1058B00091E15BDAF0904B0180916608811103C0A1
:1058C0006FE08C2F0ADB6EEC71E180E00E941568BE
:1058D0000E94B163AC0160E086E60E94466A1091C6
:1058E0004B018091DF07823021F41092DA08109288
:1058F000DF0780910E0891E0980F191728F41230F5
:1059000068F08FEF810F0BC094E0980F911738F477
:105910008CEF810F8B3018F08AE001C080E080931B
:105920000E08082FD0E1EE24E3941013E12CDD24BF
:10593000D394D00E2E2D4D2D6D2F82E10E94486AFA
:1059400080916206081305C04AE26D2F81E00E9433
:10595000B8674FE06AE678E0802F0E944F60EE2043
:1059600031F08091DA08882311F001E101C000E1F3
:105970002FE04AE658E06D2F88E10E94BA67D85FB1
:10598000D03411F00D2DCFCF80916608882309F413
:1059900076C080916206811302C0D9E501C0DEE7BE
:1059A000812F0E948060811101C0D6E98091840618
:1059B00082FFDF734AE06D2F8FE198E1DBDE8130FB
:1059C00009F09AC0D0916808D11105C086E593E529
:1059D0000E945D1691C09FEF9D0F923060F510936D
:1059E000620680938B0D8C2F0E94196DA8950E94E2
:1059F0000562A895812F0E941462A89580910501E7
:105A000082608093050181E00E940961A8950E944F
:105A100005620E94831B0E949E1B80915B020E9474
:105A200094160E94717580916608823079F2D230A6
:105A300009F053C0CBCFD53031F48C2F0E94196DB3
:105A40001092DF0704C0D33049F48093DF0710932E
:105A5000DE078CE69BE20E946E1B4EC0D63019F426
:105A600080936E0804C0D73039F410926E081093FA
:105A7000720880ED90E3EFCF8093DA083DC0C63620
:105A800038F4C43688F4C036B1F0C13641F034C0C1
:105A9000C13819F1CF3B29F1CE3671F50CC0809198
:105AA000DA08882349F10DC080916206811709F454
:105AB0008DCF82E00AC010920D088091DA08882309
:105AC00019F01092DA0818C081E0809366088C2FD4
:105AD0000E94196D109267080FC081E00E944A165B
:105AE0000BC01092DA0810926608809162068093CB
:105AF0004B0181E00E945B618091DA088823F9F014
:105B0000CF2DDD27C7FDD095212F30E0C217D30759
:105B1000B1F061E0610F81E08F0D0E946A64209115
:105B20006206121303C0F092620606C030E0C2178C
:105B3000D30729F41093620681E00E940961DF9186
:105B4000CF911F910F91FF90EF90DF900895CF922A
:105B5000DF92EF92FF92CF93DF93FC01EB019C0168
:105B6000DC010E94E3799B01AC01DE010E94F8791F
:105B7000272F382F492F5527DF010E94F8796B0115
:105B80007C018CE0F694E794D794C7948A95D1F77A
:105B900024E630E02C1B3D0B0E94E3796E5C7F4FC6
:105BA0008F4F9F4F6C0D7D1D8E1D9F1D24E630E095
:105BB00040E050E00E94577AC901DF91CF91FF90F9
:105BC000EF90DF90CF9008951F93CF93DF936115EF
:105BD000710519F1192F111F1127111F19F0919536
:105BE0008195910977FF0FC0719561957109C0E0AA
:105BF000D4E09E01281B390BC901A9DF9E01281B97
:105C0000390BC90101C0A3DF112329F02227332753
:105C1000281B390B01C09C01C901DF91CF911F9155
:105C20000895EF920F93CF93DF93382F862F642F31
:105C3000922F332319F02091070801C020E0C09172
:105C4000E3084EE0C49FE0011124C550DC4F9336B9
:105C500029F4032F4C8552DC8C8726C0923629F418
:105C6000032F4D854BDC8D871FC0E02FF0E0E90F3F
:105C7000F11DE90FF11DEE0FFF1FEE0DF11DEC0FF1
:105C8000FD1FEF01011107C0E22E04E62CE9488157
:105C90000E94402608C048814C59E22E04E620E0CC
:105CA0000E94402684568883DF91CF910F91EF9018
:105CB000089590E0E92FF0E0E358F44EE491E817FE
:105CC00021F0EE2321F09F5FF5CF892F089580E02A
:105CD0000895823430F4E82FF0E0E358F44E8491D4
:105CE000089580E20895DF92EF92FF920F931F9341
:105CF000CF93DF93F82E162FEA01E22ED02E68E024
:105D00007BE1812F0E94156800E12E2DAE01612FED
:105D100082E40E94BA67DD2099F18F2D880F8F0DE4
:105D2000880F20910D0846E0612F8E5B0E9451681C
:105D30004E2D440F4E0D440F4C5F6FEF610F29E065
:105D400080E40E94BC6A80910D088823C9F0CF0DC1
:105D5000D11D88818111ADDF2D2D41E460E00E94CD
:105D60003116B7DF488150E0282F332727FD3095C3
:105D70004217530729F08883809106080E94096121
:105D8000DF91CF911F910F91FF90EF90DF900895D9
:105D9000FF920F931F93CF93DF93C82FD62FF42E2C
:105DA000122F622F842F0E94E814FC01E53F81E04E
:105DB000F80774F09BE09E0F9F1510F09CE09E0F7B
:105DC00040E3490F202F6D2F8C2F0E942D6707C0B5
:105DD000212F40EB59E16D2F8C2F0E94DE67DF9160
:105DE000CF911F910F91FF9008954F925F926F9204
:105DF0007F928F929F92AF92BF92CF92DF92EF925B
:105E0000FF920F931F93CF93DF93182FC091E60853
:105E10002AE0C29FE0011124CA5EDA4F8FE392E1CB
:105E20000E94B52664E0812F58D8A82E4091E6083C
:105E30004F5C60E080E30E94B86748E0B42E10E059
:105E400053E0952E66E0862E75E0772EA11203C0F2
:105E50006090070801C0612C1130C1F038F0123099
:105E600009F465C0143009F493C076C061E272E1B0
:105E70008B2D0E94156801E0611001C000E0262D05
:105E800048856B2D80E33ADB888792C06110909241
:105E9000E5083CE3432E512C8091E407851511F071
:105EA00000E001C0062D4091E6084F5F252D6B2DC7
:105EB000842D6EDF6620A1F18091E407851130C04A
:105EC00080910C08882361F17E01E50CF11CE50C42
:105ED000F11CF701C080D180FBE0CF1AFEEFDF0A92
:105EE00024EFC21621E0D20624F424EFC22EDD24D2
:105EF000D39422E048EF51E064EF71E0C6010E94C4
:105F00006C158C159D0561F0843FE1E09E0711F44E
:105F100080E090E0AC01455F5140F7015183408340
:105F20005394F6E04F0E24E05212B6CF41C06620E3
:105F300051F089856FE08F700E943E168F709985B1
:105F4000907F982B998749854F70262D206285E098
:105F5000489FA001112417C0662061F089856FE079
:105F600082958F700E943E168295807F99859F70E2
:105F7000982B9987498542954F70262D2062E5E040
:105F80004E9FA00111246B2D86E60E94186A10C056
:105F900061107092E5084091E608849EA0011124EA
:105FA00044585A4F062D26E06B2D8091E4079BDE66
:105FB0001F5FF8E0BF0E153009F048CFDF91CF9199
:105FC0001F910F91FF90EF90DF90CF90BF90AF9017
:105FD0009F908F907F906F905F904F9008951F9348
:105FE000CF93DF93C82FD62F142F4EE152E10E949A
:105FF0002B6840E3410F6D2F8CE08C0FDF91CF9128
:106000001F910C94B8679F92AF92BF92CF92DF928C
:10601000EF92FF920F931F93CF93DF93C82F82EEDF
:1060200099E10E94B52663E08C2F0E946D27982E7F
:10603000C03611F0CE3649F49092E6088C2F0E94BB
:10604000196D85EF9EE20E946E1B6DED71E180E19E
:106050000E941568E6E1CE2EE5E0DE2EFCE7EF2E8D
:10606000F5E0FF2E18E1B12CAA24A394B910A12CBD
:10607000E6018985882331F02A2D4AE2612F89E7DC
:106080000E942D67B3944B2D612F86E0A8DF2A2D47
:106090004885612F88E10E943913DCE3C0E00A2DB6
:1060A0002C2F4B2D612F8D2F73DECF5FDA5FC43025
:1060B000B1F700E126E0A701612F8AE50E94BA67E7
:1060C0008AE0C80ED11C185F86E0E80EF11C84E05F
:1060D000B812CACF0E940A1C682F660F660F660F9F
:1060E000615F29E04AE180E0DF91CF911F910F913C
:1060F000FF90EF90DF90CF90BF90AF909F900C9467
:10610000BC6A1F93CF93DF93162FEC01112329F064
:1061100089910E94EE6D1150F9CFDF91CF911F91BF
:106120000895CF93C82F0E94F56D8F3F21F08C13F7
:10613000FACF81E001C080E0CF910895CF93C82FBE
:1061400081E00E94EE6D80E00E94EE6D8C2FCF9179
:106150000C94EE6DEAE6F8E01382128282E0818709
:1061600084E40C94EE6D0F932091700830917108C7
:1061700042E3429FC001439F900D112462EF71E002
:106180000E94307A062F28E044E660E38EE00E9409
:10619000C76A0F910895AC0168E184E20C942B6802
:1061A0009F92AF92BF92CF92DF92EF92FF920F93A6
:1061B0001F93CF93DF93D82ECAE6D8E08C8181114C
:1061C00003C085E192E102C089EA99E10E94B52607
:1061D000A89521E6D21671F08FEBD81219C00E9453
:1061E000DC6D19861982E0914901F0E0E65BFE4F13
:1061F00010820EC08AE50E94EE6D809162060E94B8
:10620000146289E0898710920D0881E60E94196D59
:10621000E0914901F0E0E65BFE4FA080498550E047
:106220004A30510508F07EC1FA01ED59FF4F0C9438
:10623000957A8BE10E94EE6D8BE10E94EE6D1882E3
:106240001B8281E09CC08B81853030F48EE369DF56
:106250008B818F5F8B8366C18C81882339F01D828F
:1062600087E0898782E40E94EE6D5CC173DF5AC1CA
:1062700027E08A2D622F0E94177A829F202D1124F9
:1062800029838DE092E187DF1CE00AE00E94F56D32
:106290008F3F09F447C12091DB083091DC082F5F64
:1062A0003F4F3093DC082093DB08833009F467C04C
:1062B0008D3009F480E02A819881FE01129FE00D63
:1062C000F11D1124E90FF11D8287811116C09B81F8
:1062D0008981981750F081E0820F8A83883028F0F6
:1062E00088E50E94EE6D83E04AC08EE40E94EE6D68
:1062F0008B818F5F8B831882C9CF81E0890F8B30B0
:1063000010F48883C3CF0883C1CF8A81982E883048
:1063100010F0B7E09B2E6981680F61508D2D0E94AF
:106320006D278981A81A8A2D873008F09FCF7E01BA
:106330009AE0E90EF11C00E010E0A8E0CA2EBB24B0
:10634000A7FCB094091598F421E0A016B10609F055
:1063500020E02061A7016C2D8CE00E94F06728E00E
:10636000C20E0F5F1F4F8CE0E80EF11CEBCF90E6E2
:10637000D912D8C082E50E94EE6D1D8284E0898723
:10638000D1C083E092E107DF8D81811120C01F829F
:106390001E8282E7C6DE882309F44EC08DE0CEDE81
:1063A0008A2D90E02981821B91092CE0289FF00121
:1063B000299FF00D11243A96EC0FFD1F84EE838780
:1063C00083E084876DE0CF019CDE188263C081305A
:1063D00099F50E94F56D8F3F2FEF920769F1988133
:1063E00021E0290F2883FE01E90FF11D82878881B2
:1063F0008F3078F38E819F8104EE13E0081B190B18
:106400000D30110510F00CE010E0A80167E778E00E
:106410008F5A9D4F0E949B7A8E819F81800F911F82
:106420009F838E83843E934008F488C085E08987EB
:1064300085E60E94EE6D188296DE74C08CEF91E1C5
:10644000AADE88850E940A60882309F46BC086E072
:1064500096CF83EF91E15BC089EA99E19CDE8D8163
:1064600081111AC01F821E8282E65BDE882321F31F
:1064700088850E9482608DE061DE6AE081E592E0BD
:1064800040DE8BE00E94EE6D84EE0E94EE6D83E0B4
:106490000E94EE6D81E02FC0813049F483E641DE39
:1064A000882351F282E08D831F821E82C5CF823005
:1064B000D1F48E819F81843E934028F083E00E9436
:1064C000EE6D84E018C08CE039DE8E819F816CE037
:1064D0008F5A9D4F16DE83E08D838E819F810C96AF
:1064E0009F838E83A9CF833041F484E61ADE88230C
:1064F00009F4A2CF82E08D839FCF86E012DE88234D
:1065000009F49ACF88E0898797CF87EE91E143DE3F
:1065100009C08AE706DE882329F00E94E66D80E044
:106520000E944A16DF91CF911F910F91FF90EF903B
:10653000DF90CF90BF90AF909F9008958EE679CF77
:1065400021E0411101C020E0405D0C942D670E94C4
:106550002C122091D8083091D908AC01421B530B62
:106560009A01283E334088F09093D9088093D80848
:10657000809160028F70823041F485E10E94291B76
:10658000882319F087E00C94E07708950F9300E0DA
:1065900020E00E94566A0F9108951F93CF93DF93D6
:1065A000182F89EC91E10E94B526163628F414368E
:1065B00030F4113659F00FC01E3841F00CC08091F4
:1065C000D70891E089278093D70805C01092D70893
:1065D00080E00E944A168091D708882309F43FC0C2
:1065E000C6E0D1E0103641F48FEF888319821B8218
:1065F0001A8287E10E94E07763E971E188E00E94F6
:1066000015684981469550E068E086E60E94466A32
:106610004881469550E060E186E60E94466A4981DD
:106620008881481B469550E068E186E60E94466AEC
:106630008A819B8129E1289FA001299F500D112467
:10664000569547955695479520E360E286E60E9469
:10665000186A60E871E188E30E94156829C0C5E402
:10666000D8E069E671E180E00E9415684091D907A1
:106670005091DA0768E08AE289DF4D815E8168E047
:106680008EE484DF4F81588560E18AE27FDF4985AF
:106690005A85C4E056954795CA95E1F760E18EE4C6
:1066A00075DF4091D7075091D80760E08EE46EDF28
:1066B000DF91CF911F910895CF93DF93282F30E082
:1066C00095E0899FE0011124CA5FDD4F4C818FE086
:1066D000829FF001839FF00D1124EB5BF74F9881AF
:1066E000898195878687442311F090E080E0938725
:1066F000848710861782168215821286118611826F
:106700001082DF91CF9108951092DA071092D90785
:1067100080E0D2CF81E0D0CF5F926F927F928F9254
:106720009F92AF92BF92CF92DF92EF92FF920F9320
:106730001F93CF93DF9307ED17E0F8018F01868158
:106740008F5F868375E4A72E78E0B72EEAE0EE2E01
:10675000E2E0FE2E812C55245394E501811003C004
:106760008091C00502C08091C105882309F48DC1C4
:106770008D324CF08C520E94291B9C81891709F4A0
:1067800084C18C8302C00E94291B882309F47DC127
:10679000811002C0B9DF01C0BDDF66246394F70138
:1067A00032979080F701319770808EEF890D82309B
:1067B00028F4C0903308D090340802C0C12CD12CEA
:1067C00080914208882319F0C12C6CEFD62EF3E09B
:1067D000F91548F4E92DF0E0EE0FFF1FE352F84FF2
:1067E000C080D18002C0992059F12CE2271504F510
:1067F000F8018481958128813981822B932B2B810B
:10680000822B2681822B2A81822B892B09F41A82E2
:1068100084ED870D0E94291B882341F09A819111F4
:1068200005C091E02B81211190E09B838A8308C0F1
:10683000772029F0872D0E94291B8B8301C05B8262
:106840008B81882379F061100DC0FCEFDF1AD7FE31
:1068500003C02FE3C20ED11C46E0D594C7944A95DD
:10686000E1F701C0C12C888199818C0D911D99831C
:1068700088830E942C12F801C480D5808C199D0950
:106880008436910508F46AC0668170E08881998138
:106890000E94447A462F99838883F80181100DC0A5
:1068A000208131812F5F3F4F3183208322813381CB
:1068B0002F5F3F4F3383228307C01682F4E6CF0E4B
:1068C000D11CF801D582C482442331F02F81388550
:1068D0002F5F3F4F38872F83611009C02B81222300
:1068E00031F02D813E812F5F3F4F3E832D837727EF
:1068F0007595679589859A85680F791F7A87698765
:10690000F7013497808191819C878B879920E1F0F2
:10691000F1E09F1209C0711004C0F8016281738117
:106920000EC06D817E810BC0F2E09F1203C06F81AB
:10693000788505C024E0769567952A95E1F79C0156
:10694000261B370B3C872B87F7012081222331F050
:106950002B853C85821B930B9C878B878394FFE060
:10696000AF0EB11C25E0E20EF11C32E08312F5CE31
:1069700005E418E0F8018F01F0900A028091060208
:1069800090910702C385D485258536852C173D0750
:1069900009F47DC0D687C5872381222309F477C0F7
:1069A000FF2021F09C012C1B3D0BE90120917B066F
:1069B00022FF2DC0892B59F1CE31D10519F469E29E
:1069C00089E10BC0C431D10519F46AE28AE105C03E
:1069D000CA30D10529F46BE28BE10E94EA770AC044
:1069E000C630D1052CF4D7FD05C06C2F8CE1F5CF56
:1069F00080E001C081E090917B0693FF08C088236E
:106A000031F082E390E090933B0180933A01D7FF0D
:106A100005C0FF2019F0F801C385D4856CE370E050
:106A2000CE010E94447A40917B0641FF1AC0892B17
:106A3000C1F44091840641FF07C06115710539F02A
:106A4000CB010E94AB2403C080E00E94E0778091DC
:106A50007B0683FF06C082E390E090933B01809326
:106A60003A01F801838594850A960A9780F48CE1AF
:106A70000E94E07780917B0683FF09C082E390E06B
:106A800090933B0180933A0102C0612C88CEDF9144
:106A9000CF911F910F91FF90EF90DF90CF90BF901B
:106AA000AF909F908F907F906F905F9008950F931D
:106AB00004E12AE041E552E0682F88E10E94BA67CC
:106AC0000F9108950F931F93CF93DF93C82FD62F65
:106AD0004730E8F4242F30E0F901EA5DFC4DE49101
:106AE00080915B01E82399F0F901E254FD4F149184
:106AF000812F0E94F86C482F50E0410F511D242F28
:106B0000483010F027EF240F215000E009C0842FF7
:106B10000E948D23182F0E94291B2FEF210F082F71
:106B200046EF52E06D2F8C2F0E94DE67DF91CF91F0
:106B30001F910F9108956F927F928F929F92AF92C3
:106B4000BF92CF92DF92EF92FF920F931F93CF935A
:106B5000DF9391E0909306089091CC0190FF02C0E2
:106B600064E001C063E00E942523F82E6091E708ED
:106B700061500E946D27E82ED090070800916308AD
:106B800010E00C30110508F019C7F801E359FF4F68
:106B90000C94957A85E29AE10E94B5268091CC0109
:106BA00080FF02C06BE001C06AE06093E70841E04B
:106BB0004E0D67508DED90E10E94C522FFC68DEF0E
:106BC00097E10E94B52686E08093E708EE2011F059
:106BD000C0E001C0CD2D4091630650E004ED10E10E
:106BE0002C2F68E086E70E94BB26CC2351F04DE2B3
:106BF0006AE0809163060E943B16809363060E94C0
:106C00000A6B68E870E180E10E94156881E0E81293
:106C10000CC040915C01642F6195809166060E94D2
:106C20003B16809366062D2D01C020E0409166063C
:106C300060E180E60E9439138091810642E068E1BC
:106C400086FB882780F90E9421279091810680FB8E
:106C500096F990938106C0917D0693E0E91207C0F2
:106C600068E78C2F0E943E16C82F2D2D01C020E012
:106C7000E5E0CE9FA001112460E286E60E94632732
:106C8000CC2329F043E760E288E70E94B867C0930D
:106C90007D06C0918506F4E0EF1206C068E78C2FF0
:106CA0000E943E16C82F01C0D12C85E0C89FA001CC
:106CB00011242D2D68E286E60E946327CC2329F05B
:106CC00043E768E288E70E94B867C0938506809131
:106CD0007B0645E060E383FB882780F90E9421273B
:106CE00090917B0680FB93F987C084EB97E10E942B
:106CF000B52686E08093E70860E670E188E00E94B0
:106D00001568C0919106C95FE11008C0DD2DD064FF
:106D100067E08C2F0E943E16C82F01C0D0E44C2F94
:106D200050E02D2F68E086E60E94186AC750C09395
:106D3000910640917806469546954695477021E024
:106D400062E370E180E10E9416278770880F880F48
:106D5000880F90917806977C982B909378064091B5
:106D60008406443008F044E022E06CEF7FE088E1E4
:106D70000E941627843008F087E08093840693E011
:106D8000E9120BC0CD2DC06444E661E0809182061B
:106D90000E943B168093820601C0C0E440918206A7
:106DA00050E02C2F60E286E60E94186AE4E0EE12C2
:106DB0000AC0CD2DC06465E0809183060E943E1616
:106DC0008093830601C0C0E44091830650E00BEE3F
:106DD0001FE02C2F68E286E60E94BB2680917B068E
:106DE00025E04BE45AE160E3869581700E942827F4
:106DF00090917B0680FB91F990937B06DFC58CEC2C
:106E000097E10E94B5268AE08093E708F5E0FE1539
:106E100008F4BCC00E943D2A6FEA7FE088E00E942F
:106E200015688091920640E068E081700E942127F9
:106E30009091920680FB90F990939206C0917B0608
:106E4000C17041E060E18C2F0E94212781709091F8
:106E50007B0680FB90F990937B068C130E94831B2A
:106E60008091810642E068E185FB882780F90E94D5
:106E700021279091810680FB95F99093810683E00C
:106E8000E812D12CE0917E06F0E0EF59FC4FD4914E
:106E9000CCE6ED2FE370F0E0EF54F64E44912D2D4B
:106EA00060E28C2F0E942D67D695D695C650C435CA
:106EB00081F7DD2039F067E180917E060E943E1661
:106EC00080937E0614E2C0E0D0E02C2F4BE758E11F
:106ED00068E2812F0E94EC662091930630E00C2E30
:106EE00002C0359527950A94E2F720FF06C020E0FE
:106EF00042E168E2812F0E9451682196185E1438A1
:106F000021F7E4E0EE120FC08091CC0180FF65C54F
:106F10006FE0809193060E943E16809393068091C5
:106F2000550D86FF5AC580917906F5E0EF1213C022
:106F300090910D08992389F063E00E943E1690918C
:106F40007906891761F0909181069F779093810669
:106F50008093790604C020E003C021E001C022E054
:106F600041E3480F60E382E10E942D67D4E2C0E074
:106F70008C2F0E941F1220E0482F60E38D2F0E946B
:106F80004A12CF5FD85EC43099F718C589E08E15D4
:106F900040F4E0914901F0E0E65BFE4F808389E038
:106FA000E82E83E08093E508C4E9D6E010E008E02D
:106FB000F02E00E0212F4CED52E06F2D8EE10E946B
:106FC000DE6701E086E0810FE81200E024E0AE0118
:106FD0006F2D8091E4070E94732E98E0F90E1F5FD9
:106FE0002496143031F7EAC485ED97E10E94B52666
:106FF00086E08093E7086DE57FE088E00E941568F1
:10700000E1100BC0CD2DC06448E768E280916406B2
:107010000E943B168093640601C0C0E42C2F40916F
:10702000640668E086E60E94266AE1E0EE1209C086
:107030004EE666EF80917A060E943B1680937A06B0
:1070400001C0D12C40917A06552747FD5095465FE7
:107050005F4F2D2D60E180E70E94186A80917806CD
:1070600042E068E181700E9443279091780680FB9E
:1070700090F99093780643E060E291FB882780F9CD
:107080000E9443279091780680FB91F990937806AF
:1070900044E068E292FB882780F90E9443279091A0
:1070A000780680FB92F99093780697FB882780F901
:1070B00025E04FE45FE060E30E9439279091780675
:1070C00080FB97F99093780679C485EE97E10E944A
:1070D000B52687E08093E708E11003C089E080933C
:1070E000E50801E0E11000E02AE046E856E068E04B
:1070F0008091E4070E94732E80917B0621E04CE38F
:107100005AE160E182FB882780F90E94282790914C
:107110007B0680FB92F990937B0622E045E35FE0DB
:1071200068E194FB882780F90E94392790917B06BB
:1071300080FB94F990937B068091810643E060E2A6
:10714000829581700E9443279091810680FB94F97B
:107150009093810680917B0624E04BE25FE068E239
:1071600085FB882780F90E94392790917B0680FB58
:1071700095F990937B068091810687FB882780F99B
:1071800025E04FE15FE060E30E94282790918106AF
:1071900080FB97F9909381068091920687FB882760
:1071A00080F926E04EE05FE068E30E942827909196
:1071B000920680FB97F99093920600C48DEE97E1BA
:1071C0000E94B52663E877E080E1E2C089E09FE0B5
:1071D0000E94B526D0E0C0E04C2F6D2F80E372DC1A
:1071E000CF5FD85FC730C1F767EE7EE080E10E94D5
:1071F0001568D8E3C0E08C2F0E940D6C482F6D2FCE
:1072000080E29ED9CF5FD850C630A9F74FED5EE03F
:1072100068E184E50E942B6816E0C0E2D0E02D2FE3
:107220004BE758E16C2F84E50E94EC66812F0E94A9
:107230000D6C482F6C2F8CE683D981E0810F0E9462
:107240000D6C482F6C2F88E77BD9DF5FC85F1E5F0E
:10725000D43029F78091A40686FF0CC06AED7EE049
:1072600088E00E9415688BE20E94291B482F68E085
:1072700088E766D98091A40687FFA0C365ED7EE00C
:1072800080E10E9415688CE20E94291B482F60E172
:1072900088E756D993C381ED9EE00E94B52681E030
:1072A0008093E70810925A01D0E0C0E019E10D2D5B
:1072B000006241E46D2F88E10E94B86741E34C0F02
:1072C0006D2F8EE10E94B8678C2F0E941718AC01B9
:1072D0006D2F8AE20E942D68C43028F48C2F0E9402
:1072E0001F12815003C0C730D9F08C2FE82FF0E077
:1072F000EE0FFF1FE15DF74F20813181129FF001FA
:10730000139FF00D1124F7FF02C0E150FF4F5F2FD4
:10731000550F550B4F2F6D2F8AE50E94466A05C009
:10732000402F6D2F8AE50E943A6ACF5FD85FC83040
:1073300009F0BFCF6DEC7EE088E20E9415684091B5
:1073400000015091010160E388E70E94466A81E0F4
:107350008093090880910D08882309F42FC34FE713
:1073600061E8809165060E943B168093650626C3FE
:1073700085EF97E10E94B52686E08093E70880902C
:10738000E4078091630081FF06C066EC7EE088E13F
:107390000E94156813C366EB7EE088E00E941568C2
:1073A000CFE6D6E0A12CF0E1CF2EA3E07A2E9924EF
:1073B00093949A0C20E0492D6C2D80E00E944A1293
:1073C000B12CEA1004C07092E5088B1419F020E08B
:1073D00010E002C01D2D22E0F2E0BF16D1F183E0E3
:1073E000B81609F44DC091E0B91689F0498142956B
:1073F00046954695437069EA7EE08C2D0E94C8262A
:107400008295880F880F807C99819F731FC00981A6
:10741000000F000F059505958DE00802F00111247D
:10742000F7FD3396AF015595479555954795212F13
:107430006C2D82E40E94186A11FF3AC04FE161EEA0
:10744000802F0E943B168F739981907C982B998393
:107450002FC06880962D9770692E20E1290F012F8B
:1074600042E45CE16C2D88E40E94DE6711FF20C0DD
:1074700063E0862D0E943E1687709881987F16C023
:107480000881059505950595212F402F6C2D8AE5DE
:107490000E94391311FF0CC04FE061EF802F0E9452
:1074A0003B16880F880F880F98819770982B9883C8
:1074B000B394E4E0BE1285CFF8E0CF0E22969E167C
:1074C00011F0A92C74CF84E0E8120BC0CD2DC0625E
:1074D00048E266EF80917F060E943B1680937F060C
:1074E00001C0C0E240917F06552747FD5095465F99
:1074F0005F4F0EE91EE02C2F60E38EE40E94BB2656
:1075000004E211E0C7E6D6E070E3D72EF80141911E
:1075100051918F0129913991421B530B440F551FF3
:1075200020E268E38D2D0E94186AF8E1DF0E80E901
:10753000D812ECCF95E0E91215C0E0E6FE1214C0B7
:1075400010920D0888E0E4E2F1E0A7E6B6E00190D1
:107550000D928A95E1F781E00E94096187E10E941E
:10756000E07702C020E001C021E04AE95EE068E384
:1075700080E00E94F06722C28CED97E10E94B52660
:1075800089E08093E708F1E0FE1580F10E943D2A32
:1075900080917B0620E042E95EE068E086FB882778
:1075A00080F90E94392790917B0680FB96F9909391
:1075B0007B06C0919206C6FBCC27C0F921E043E8C8
:1075C0005EE060E18C2F0E9428279091920680FB5C
:1075D00096F990939206C81709F4F0C1882319F020
:1075E0000E94C36DEBC110929A00E8C188E08E152D
:1075F00008F487C068E37EE00E941568C0E008E0F8
:1076000022E02C0FF090A406C23051F0C33069F094
:107610004091A506C13079F442954F7010E10DC03C
:107620004091A7064F7010E408C04091A70642950C
:107630004F7010E802C04F7014E064E17EE0802FCC
:107640000E941627D82F812F80958F21D11103C03A
:107650008093A40603C0182B1093A4068091A4065F
:10766000F8120E947E12C23051F0C33069F0C1306E
:10767000A1F4D295D07F9091A5069F7012C0DF70C3
:107680009091A706907F05C0D295D07F9091A706D4
:107690009F709D2B9093A70607C0DF709091A50661
:1076A000907F9D2B9093A506085FCF5F083209F06D
:1076B000A7CF8091A80646E068E281700E9421274A
:1076C0009091A80680FB90F99093A80647E060E3AC
:1076D00091FB882780F90E9421279091A80680FBC2
:1076E00091F99093A80648E068E392FB882780F917
:1076F0000E9421279091A80680FB92F99093A806FA
:107700005DC18091A9068F7099E0E91205C06FE014
:107710000E943E162D2D01C020E0C82FD0E002E0CF
:107720001EE0AE0168E088E70E94BB266091A906D2
:107730007091AA06607F6C2B7D2B7093AA066093D4
:10774000A906FB01E07FFF2734E0F695E7953A951F
:10775000E1F78E2F9AE0E91205C06FE00E943E1615
:107760002D2D01C020E0C82FD0E000EF1DE0AE01BC
:1077700060E188E70E94BB26AE0124E0440F551F5C
:107780002A95E1F78091A9069091AA068F70482B5F
:10779000592B5093AA064093A90644275F70852F62
:1077A000EBE0EE1205C06FE00E943E162D2D01C0E9
:1077B00020E0C82FD0E00EED1DE0AE0168E188E7C3
:1077C0000E94BB269C2F88272091A9063091AA06EB
:1077D000307F822B932B9093AA068093A906892F42
:1077E00082958F70FCE0EF1204C06FE00E943E169D
:1077F00001C0D12CC82FD0E00CEC1DE02D2DAE0126
:1078000060E288E70E94BB26AE01542F44275295C0
:10781000507F8091A9069091AA069F70482B592B02
:107820005093AA064093A906C9C080EC97E10E9434
:10783000B52681E08093E708E0914901F0E0E65B3E
:10784000FE4F1082CAE6D8E010E0812F0E94171880
:107850002E853F85821793070CF49C013F872E8766
:107860004C8D5D8D481759070CF4AC015D8F4C8F22
:10787000143060F02E853F85240F351F37FF02C07E
:107880002F5F3F4F35952795398328831F5F2296B9
:107890001730D9F6809194088093090890E2F91680
:1078A00021F0EFEBFE120EC00BC08F5F80939408A7
:1078B000833041F487E10E94E07781E00E94096112
:1078C0001092940880919408813089F050F08230B1
:1078D00009F072C010925A01E8E7F8E0C6E3D6E07A
:1078E0001FC06BEB7DE088E10E94156865C0CAE6A9
:1078F000D8E0D12C18E9E12E1AE3F12E08E615ECB8
:10790000FF86EE861D8F0C8F8D2D0E941718899390
:107910009993D394F7E0DF12F3CF6DEA7DE043C093
:1079200061917191848595859B01281B390B37FFE7
:1079300003C0319521953109233331053CF1DF0135
:1079400050974D915C91598348839A01261B370BC0
:10795000B90137FF02C0615C7F4FB6E0759567954E
:10796000BA95E1F7261B370B3F872E87841B950BB3
:107970009C0197FF02C0215C3F4FA6E035952795FB
:10798000AA95E1F7821B930B9D8F8C8F229688E03E
:10799000E638F80729F60E94C65F90936106809347
:1079A00060066BE97DE080E10E9415684EE058E1D9
:1079B00068E182E10E942B680E94F829DF91CF9153
:1079C0001F910F91FF90EF90DF90CF90BF90AF90FD
:1079D0009F908F907F906F90089529E04CE567E22B
:1079E00083E20E94BC6A9FCACF93DF93C82FD62F31
:1079F000462F60E267D841E04D0F68E28C2F62D8D5
:107A000042E04D0F60E38C2F5DD8D1110DC089E0AD
:107A10000E94291B882341F020E042E160E28C2F84
:107A2000DF91CF910C945168DF91CF9108951F930E
:107A3000CF93DF93EC01862F11E0683008F410E05B
:107A40000E942022FC019E013C5F37FD0DC02115E4
:107A500088E0380784F0112319F048E050E002C0B4
:107A600044E050E0E40FF51F8081992787FD909551
:107A7000982F882723C0832F112321F03327220F2B
:107A8000331F02C086953170482F50E0E40FF51F78
:107A9000608140E052E0421B530B559547956403CB
:107AA000C001659F900D1124618135952795620372
:107AB000A001639F500D1124840F951F69E170E0B0
:107AC0000E94447ACB01DF91CF911F910895BF921C
:107AD000CF92DF92EF92FF920F931F93CF93DF939A
:107AE000182F7B010E948F26C82E812F0E94051A15
:107AF000811104C001E01E141F040CF400E08EE0AC
:107B0000189FE0011124C550DC4F84E0C89E60013D
:107B10001124F601E00FF11DEC0FFD1FB080812F45
:107B20000E94051A8823A1F08B2D0E94021A682F4B
:107B3000772767FD7095C7019C5F97FD0196959526
:107B400087950E94E42D7C01EE0CFF1C00E00BC029
:107B50008B2D0E94021A682F772767FD7095C70149
:107B60000E94E42D7C01CC0DDD1DC00FD11D8A814A
:107B700044E660E08C590E94EC199701A82FBB27BE
:107B8000A7FDB0950E94DD7924E630E040E050E0AA
:107B90000E94797AE901812F0E94051A8111D4503F
:107BA000CE01DF91CF911F910F91FF90EF90DF9069
:107BB000CF90BF900895DF92EF92FF920F931F93A3
:107BC000CF93DF93D62EB0EEFB2EF80EC0E0DCEFA5
:107BD0000FE710E2E12ED11005C06091E408CE015C
:107BE00026DF04C0BE018091E30871DF97FD4F9648
:107BF0009C01A5E035952795AA95E1F7122F0F373F
:107C000009F4022F412F552747FD5095401B51097C
:107C100007FD539557FF03C05195419551094230D7
:107C200030F46E2D611B8F2D0E947D680CC00117F2
:107C30001CF09FEF940F01C090E06E2D611B691B3B
:107C40008F2D0E94CB68112321F060E28F2D0E94BE
:107C50007D68F394A096C03284E0D80711F0012F1C
:107C6000BACFDF91CF911F910F91FF90EF90DF90EE
:107C70000895DF92EF92FF920F931F93CF93DF93BC
:107C8000D82E8091E408EE24E394883008F4E12CA7
:107C90000E942022EC0140E460E08CE50E94CB6869
:107CA000F12C0CE91FEF2F2D30E0EE2019F049E008
:107CB00050E002C045E050E0241735075CF5C901EB
:107CC00045E0880F991F4A95E1F7EE2019F064E02E
:107CD00070E002C062E070E00E94447AE62FDE01AC
:107CE000A20FB31F2C9130E22302C0011124B8016E
:107CF0000E94447ADF1005C0625E25E045E08AE319
:107D000004C0615E23E043E08BE38E0F0E94BC6AF7
:107D1000F394C9CF60E08CE5DF91CF911F910F9173
:107D2000FF90EF90DF9047CF5F926F927F928F929C
:107D30009F92AF92BF92CF92DF92EF92FF920F93FA
:107D40001F93CF93DF93882ECC24C3948091E408B3
:107D5000883008F4C12C85ED99E10E94B526CC202D
:107D600011F069E001C065E0882D0E946D27D82ED2
:107D70008FEB881202C01092DD084091E40850E0B9
:107D80004F5F5F4F21E060E08AE20E94186A8091B5
:107D9000E4080E942022EC0160900708CC2019F032
:107DA000F9E07F2E02C0E5E07E2E5C2E0C2F1D2F09
:107DB00065E0E62EF12C70E1972EAD2CB12C802FD2
:107DC0008519D81611F020E001C0262DF801419147
:107DD0008F01552747FD5095692D88E10E94186A4B
:107DE000CC20A1F0F9E0EF1689F0AE14BF0411F039
:107DF00020E001C0262DFE01EE0DFF1D408155271C
:107E000047FD5095692D80E30E94186A88E0980E1E
:107E1000EFEFEE1AFE0AF8E39F12D1CFD71411F05C
:107E200020E001C0262D4AE254E168E38CE00E9484
:107E3000F067D7103AC080910D088823F1F1809245
:107E400011021091DD0820E044E06CEF812F0E94C8
:107E50003116082F8093DD08811779F1CC2011F0BD
:107E600024E001C022E0122F119530E059E1F52EF7
:107E7000E12FFF27E7FDF0952E173F0794F0EC0F59
:107E8000FD1FE20FF31F1002A0011124F49EC00198
:107E9000F59E900D1124B9010E94447A60831F5F02
:107EA000E7CF82E00E94096108C0CD0DD11D44E6F4
:107EB0006CE988810E943B1688838D2DDF91CF91DC
:107EC0001F910F91FF90EF90DF90CF90BF90AF90F8
:107ED0009F908F907F906F905F90CBCEEF92FF92AC
:107EE0000F931F93CF93DF93C82F0E941718D0E0F2
:107EF000FE01EE0FFF1FEB5CF94F21813281821BE7
:107F0000930B9C01BC01882777FD8095982F0AE090
:107F1000660F771F881F991F0A95D1F7121613064F
:107F20001CF4258D368D02C0278530892436310515
:107F300014F424E630E0442737FD4095542F0E9486
:107F4000797A790121308CEF380744F0211584E0EB
:107F500038073CF0E12CA4E0FA2E03C0E12CBCEF82
:107F6000FB2E0E944012882379F080917906082F19
:107F7000017010E082E090E0801B910BC817D907D8
:107F800019F4F194E194F108C701DF91CF911F91A9
:107F90000F91FF90EF9008952F923F924F925F9232
:107FA0006F927F928F929F92AF92BF92CF92DF9209
:107FB000EF92FF920F931F93CF93DF93CDB7DEB76E
:107FC000A0970FB6F894DEBF0FBECDBF8F879B87FB
:107FD0006D8B80917906880F880F9E012F5F3F4F30
:107FE0004901E12CF12C1C8E1B8E1A8E212C682E3F
:107FF000712CA30144535D4F3A0160726E8B5D8911
:1080000051705D876D896270562E3E2C8E2D66DF15
:108010008C0173E07E1570F054E0959587955A9524
:10802000E1F7F701E35CF74F8083F301EE0DFF1DED
:10803000449001C04E2CC42CD12CC601880F991F2E
:108040009A878987FC01E15DF74F11830083C8019E
:1080500017FD0F9634E0959587953A95E1F7282F0F
:1080600087FD219522307CF481E090E00C2C01C04A
:10807000880F0A94EAF7211102C0982F03C090914B
:10808000D6079823292A93E0931508F473C0AD8589
:10809000A11158C080915D0281FF54C05601AA0C05
:1080A000BB1CF501E159F94F5F018181807C09F426
:1080B00049C080818595859585950E94291B8823D7
:1080C00009F440C080911B028823E1F1D501EC91B5
:1080D000E770F0E0DF01AA0FBB1FAC5DBE4FEE0FF3
:1080E000FF1FE959F94F8D919C9120813181821BAD
:1080F000930B97FD0196AC0155954795F5012181AC
:10810000322F330F330F359535953403C001359F2A
:10811000900D11246FE170E00E94447A660F771F82
:10812000660F771F2295269526952370213009F03A
:108130009CC4060F171FF2E04F1204C07B8F6A8F9A
:1081400021E02C8F3E89332339F0F601EE0FFF1F1B
:10815000E253F84F11830083B801842DB8DC8C0101
:10816000632D809111070E942815880F991FD40153
:108170008D939C93BE89BB2339F0F601EE0FFF1F50
:10818000EA54F84F118300835520E1F0E3E0E31552
:10819000C8F0F2E04F16B1F0065F1F4F0531110530
:1081A00038F0F601EE0FFF1FEA54F84F11821082EB
:1081B000E1E0F0E0EC0FFD1F29853A85E20FF31FA7
:1081C000118210823FEFE31AF30A42E0840E911C01
:1081D00057E0E516F10409F018CF8091620280FFA4
:1081E00027C062E0809111070E942815182F0E9475
:1081F0004012012F81110195202F332727FD309543
:10820000432F532F23583F4F4F4F5F4FA0E0B4E011
:108210008091BA079091BB07A81BB90B0E94027A04
:1082200020E034E040E050E00E94797A3E832D83E4
:108230006E89662309F435C110916602122180917E
:10824000D6078095812319F088E10E94E07710938A
:10825000D60706EB17E0D8018D0180E094E0FD0120
:1082600097878687918B808B40916902442309F41C
:1082700058C0A281B381E680F7809D010E94DD791C
:108280004B015C019701D7010E94DD79860E971E94
:10829000A81EB91E842F0E940F1A7C019C01DC01CC
:1082A0000E94DD79681579058A059B05D0F580E186
:1082B000C82ED12C40E050E8E0E0F0E89A01DA0165
:1082C0000E94E37986169706A806B90610F44E2791
:1082D0005F27F695E79521E0C21AD108C114D104B1
:1082E000E9F4F801228133814A01A12CB12CD70194
:1082F0000E94DD79A50194010E94797AF801338307
:10830000228326813781D7010E94DD79A50194015E
:108310000E94797AF8013783268303C04E2B5F2BA6
:10832000CDCF60916702862F807E09F4BAC05110CC
:108330000EC0F801228133818B819C81280F391F67
:10834000868197814F815885840F951F04C080E0F6
:1083500090E020E030E040916802442379F0415001
:10836000E42FF0E0EE0FFF1F443118F4E00FF11F8F
:1083700002C0E951F84F4081518102C040E050E015
:1083800062FF03C031952195310963FF03C09195C8
:108390008195910964FF03C05195419551096295FA
:1083A00066956770633009F463C0643009F469C08E
:1083B000623059F1BC0197FF02C0695F7F4FF3E063
:1083C00075956795FA95E1F7DC01A61BB70BBC0123
:1083D00097FF02C061587F4F660F672F661F770BAC
:1083E000A61BB70B97FF02C081509C4F892F990F96
:1083F000990B85958595A81BB90B7A01E21AF30AAA
:1084000037FF2CC02F5F3F4F29C0B90137FF02C093
:10841000695F7F4FF3E075956795FA95E1F7D901AC
:10842000A61BB70BB90137FF02C061587F4F660F1B
:10843000672F661F770BA61BB70B37FF02C02150B3
:108440003C4F232F330F330B25952595A21BB30BE0
:108450007A01E81AF90A97FD01969C01359527954E
:10846000240F351FB9016A0F7B1F2A1B3B0B12C05B
:108470007A01E21AF30A240F351FB901680F791F38
:1084800007C07A01E21AF30ABA01680F791F9A014C
:10849000281B390BF801F38AE28A758B648B378BC2
:1084A000268BFF85FA8B2B852B8B4BEA53E0598F5C
:1084B000488F1A8619861BE6212E12E0312E1C8A5F
:1084C000598558A3B101665F7F4F7E876D87C12CA8
:1084D000D12C7601D1018C9190E00197E985FA8544
:1084E0008E179F0709F06BC17C89672F70E0788B2E
:1084F0006F875B01B3E0B594A794BA95E1F7EC8977
:10850000E770F0E0EA5DFC4D8490ED85FE853897DC
:1085100080810E94021A898BF501EE54F84F9080F9
:10852000982040E061E00D851E8507501109D801B3
:108530008C910E94241AF8019081992359F0ED85BD
:10854000FE85399790819D50983020F490911B02C0
:10855000992399F0882391F0F10181858F7190E042
:108560000090110702C0959587950A94E2F78170F3
:108570009927F1E08F27817001C080E02D853E852D
:10858000295031093F8F2E8FD9011C91811134C0A0
:10859000782C7094F501EE54F84F8080872080820B
:1085A0001D32C9F4EF85F889EE0FFF1F2F8538893A
:1085B000E20FF31FEE5AF84FAFE8B2E0A7019601C1
:1085C0000E94F879BB2797FDBA95A92F982F872F7E
:1085D00080839183A28388EF810F823008F0E2C00C
:1085E000F10187818670843009F4DCC0193009F408
:1085F0000DC400E010E00CC481E0911080E0982EE2
:108600002FEF210F2C30B0F4822F90E0DC01AA0F65
:10861000BB1FAA54B84F0D911C91243008F06DC0B7
:10862000F101278126FF69C0FC01EE0FFF1FE25315
:10863000F84F29C02431C0F483EF810FE82FF0E018
:10864000DF01AA0FBB1FAC5DBE4F0D911C918430A2
:1086500040F4EE0FFF1FE959F94F80819181081B0B
:10866000190B000F111F49C0243280F4F1018781DA
:10867000E22FF0E0EE0FFF1F86FF03C0E354F84F38
:1086800002C0E951F84F0081118137C0243279F4DA
:10869000F10181858295869587700E9495238823B4
:1086A00051F1813009F0E6C100E010E026C02C3223
:1086B00060F4E22FF0E0EE0FFF1FE254FB4F008169
:1086C000F8E00F028001112418C02C3251F4C701C8
:1086D000B60124E630E040E050E00E94797A89015A
:1086E0000CC040E050E060E070E082ED810F0E943D
:1086F000E5238C0102C000E01CEFF501EE54F84FB9
:10870000808188298083F101878183FFB6C1F101CF
:10871000F681FD8FF111C1C1F10185818111BDC1CA
:10872000F1018781ED85FE85369787FFF1C2808153
:108730000E94021AA82FBB27A7FDB0951A161B0688
:108740000CF4CDC2109709F0D2C2F101478140FF6D
:1087500028C39801E989AE2FBB27A7FDB0950E94D9
:10876000DD794B015C0143FD30C3F10187818695C2
:108770008370813009F040C3C501B40124E630E0C4
:1087800040E050E00E94797ACA01B901A701960140
:108790000E94087A20E034E040E050E00E94797ABC
:1087A00069017A01FAE02F0E311C2C892F5F2C8B86
:1087B0004D855E85465F5F4F5E874D878BCE1092FD
:1087C00042088091C206882309F441C08F01000F3E
:1087D000111F000F111FF801EE53F94F8784908885
:1087E000A188B288FE89FF2319F0812C912C5401B5
:1087F000C701B60124E630E040E050E00E94797AFB
:10880000E0911107F0E0EE0FFF1FEE53F94FA58145
:10881000B6810E94F879680D791D8A1D9B1DF801AB
:10882000EE53F94F6787708B818B928B2D8926FFD2
:10883000EFC02091C5063091C60640E050E00E948E
:10884000797AA4E6B0E00E94F8796B017C01098591
:108850001A85000F111F015F174FC701B60124E6EB
:1088600030E040E050E00E94797AD8012D933C93AB
:10887000688C798CF3013F0183819481809001059C
:10888000912C49845A84440C551C881699063CF056
:10889000919481949108881699060CF44C01F30187
:1088A00021818401FAE02F02000D111D1124D30152
:1088B0002C91F4014AE02402E00DF11D11249F01E6
:1088C000285E334008511C4F033E54E0150714F056
:1088D00002EE14E049012E316BEF360724F42EE14D
:1088E000822E2BEF922E302F212F8017910714F418
:1088F000382F292FA32EB22EA814B9040CF454013A
:10890000C114D104E104F104A9F0F7FE04C0D501BB
:10891000A819B90903C0D801AA19BB09A701960172
:108920000E94027A20EA36E841E050E00E94797A1B
:1089300069017A01C5010E94D6195C01AC0CBD1C0D
:10894000C8010E94D6198A159B050CF45C01C4016C
:108950000E94D619A816B9060CF45C01F3018281B5
:10896000882319F0B194A194B1089091CD049F711E
:1089700080E1891BF8A1F81708F044C0C2018253B6
:108980009B4FDC012D018C91982F9F77D9F1880F97
:1089900085950E94291BF201908197FF27C08823AB
:1089A00019F01092D4081BC09091C2052091330891
:1089B0003091340895FF06C02D5E3F4F27323105B8
:1089C00020F00DC024313C4F54F47C8D772309F402
:1089D00025C22A8D3B8D24313C4F0CF41FC290914F
:1089E000D408911101C081E080934208882351F09E
:1089F000E985FA85EE0FFF1FE153FB4F80810E944E
:108A00000F1A5C01F894AA89BB89AD92BC92789444
:108A1000E985FA853196FA87E9872A893B892E5FAD
:108A20003F4F3B8B2A8B488D598D4B5F5F4F598F42
:108A3000488F709709F044CDA0960FB6F894DEBF2A
:108A40000FBECDBFDF91CF911F910F91FF90EF909F
:108A5000DF90CF90BF90AF909F908F907F906F905E
:108A60005F904F903F902F900895223009F063CB94
:108A70008B0161CB00E014E040CEED85FE8532979E
:108A80008081882309F443CE4DE763E80E94EC1906
:108A90000E940F1A080F191F3ACE8091620283FFBD
:108AA00003C0F4E1FF8B02C024E62F8B4F85588969
:108AB000440F551FDA01AE5EB84F3C91FD01218194
:108AC000EF85F889E40FF51FEE5AF84F8081918108
:108AD000A281AC016A2F772767FD70952A013B01BF
:108AE000BB2777FDBA95A72F962F852FB801681B56
:108AF000790BCB01AB01465F5F4F4531510550F01B
:108B0000A32EB22EA114B10439F4F1012581211153
:108B100008C002C0A12CB12C911003C09C878B8788
:108B200037C0F101878186708430D9F4E081F0E0AC
:108B3000EE0FFF1FE35FF74FA081B18120E034E625
:108B40000E94F2792B013C01F989FF2351F02F2F6C
:108B5000332727FD3095432F532F0E94797A29011F
:108B60003A01BB2777FCBA95A72D962D852D980144
:108B7000281B390B3C872B872115310549F0F10162
:108B8000858137FF82958F70FF89F89F50011124EE
:108B90001A141B04B4F48091B301882331F021E04E
:108BA000A21AB108A114B10449F0332777FC3A9511
:108BB000272D162D052D1C861B8603C0AA24AA94DA
:108BC000BA2CEF85F889EE0FFF1FEE5EF84FB182E9
:108BD000A0824B855C85452B09F473C04801AA240B
:108BE00097FCA094BA2C5D8D552309F466C0809142
:108BF000B301882309F440C06989662379F0262FE0
:108C000027FD219530E040E050E060E070E080E238
:108C100093E00E94797ACA01B90104C060E070E073
:108C200080E293E0F10126814B855C8514161506E0
:108C300044F090958095709561957F4F8F4F9F4F31
:108C400022952F7030E02115310591F0AF89A29F58
:108C5000A001A39F500D11249A01442737FD409590
:108C6000542F0E94797A420E531E641E751E04C052
:108C70004424582C692C7A2CBB2777FCBA95A72D55
:108C8000962D852DEB85FC851E161F0634F488165F
:108C90009906AA06BB0634F009C088159905AA05ED
:108CA000BB0524F44424582C692C7A2C332777FCF8
:108CB0003A95272D162D052D04C04424582C692CD7
:108CC0007A2CEF85F889EE0FFF1F2F853889E20F88
:108CD000F31FEE5AF84F40825182628221CD17FF76
:108CE00034CD24E630E02A1B3B0BD90106C0101618
:108CF00011060CF02ACDAC59BF4F98010E94DD79C6
:108D000024E630E040E050E00E94797A89011DCDF0
:108D100060818BE1860F873340F06058772767FDCD
:108D20007095C8010E94E42D34C0862F992787FDD5
:108D30009095A92FB92F87309105F8F4FC01E758D9
:108D4000FF4F0C94957A17FF00CD10C01016110636
:108D50006CF0FBCC17FFF9CC119501951109F5CCFE
:108D600010161106C4F002C017FD18C000E010E094
:108D7000ECCC101611067CF011C067FF06C01195EF
:108D80000195110936E0361B632F6750C8010E9418
:108D9000173D8C01DACC00E014E0D7CC00E01CEFEA
:108DA000D4CCAE8DBF8D8C919FEF980F943008F08E
:108DB000D0CCFE013196E80FF11DE80FF11D32977E
:108DC00080819181080F191FC4CCED85FE853297F3
:108DD0008081882309F4C9CC4DE763E80E94EC192F
:108DE0000E940F1A24E630E0DC010E94F279860E20
:108DF000971EA81EB91EB9CC823029F0C80CD91C08
:108E0000EA1CFB1CCFCC75016401CCCC00E01CEF4C
:108E1000F501EE54F84F8720808275CC91E0909355
:108E2000D408DDCDFF920F931F93CF93DF930E9461
:108E30000A1C182F8093110763E68AE698E0ACD8E5
:108E400061E68AE898E0A8D8CAE6D8E0EDEAF3E05F
:108E500021813281499159918E8D9F8D481B590BEB
:108E60008081811103C0519541955109240F351F0F
:108E7000293E83E038073CF428318CEF38072CF486
:108E800028E13CEF02C028EE33E03283218335969F
:108E900028E0CA38D207E1F600E0023071F40F5F33
:108EA0000430D9F786E00E94096181E0DF91CF911B
:108EB0001F910F91FF900C94E077602F812F0E94FB
:108EC0002815EC01F12C602F8F2D0E94E814853FAE
:108ED00021E092073CF4AC014C1B5D0B602F8F2D01
:108EE0000E943A15F39484E0F812EDCFD8CFEF92B8
:108EF000FF920F931F93CF93DF9390917706192FD3
:108F00001F7010925A012091660821119DC0907720
:108F1000813809F483C088F4843209F441C038F4FC
:108F2000823209F461C0833209F452C08DC08532A7
:108F300009F440C0803809F187C0843841F160F4F9
:108F4000823809F45EC0833809F07EC08DEC92E36C
:108F50000E946E1B83E85AC08E3879F08F3B09F46B
:108F600065C0853809F070C081E0809309088BE9FD
:108F700095E30E946E1B85E828C092E090936608F6
:108F8000109267080E94196D109211025DC081E075
:108F9000809309088FE49CE20E946E1B84E815C050
:108FA000123009F051C08091DF088F5F833054F098
:108FB00080E008C0123009F047C08091DF0881507E
:108FC00087FD82E08093DF083FC00E94196D3CC09E
:108FD0001F5F143008F010E0912B9093770681EA20
:108FE0000E94096183E11FC0112311F0115001C0DB
:108FF00013E0912B9093770681EA0E94096184E146
:1090000012C08DEC92E30E946E1B82E8DF91CF913B
:109010001F910F91FF90EF900C94196D0E94843373
:109020000E948A3387E10E94E0770EC081E00E94AF
:10903000196D83E00E94196D82E00E94196D81E034
:109040008093D6081092DF08809165020E94291B48
:10905000C82F882329F08091D608811101C0E2DE53
:10906000C093D60890913C0180916406981710F443
:10907000C6E001C0C4E080E00E9457354C2F406834
:1090800060E185E20E943A6A46E568E186E20E9474
:10909000B86724E040E060E18FE50E945F2520E0B2
:1090A00040E068E183E30E9489130E940A1C882340
:1090B00021F1282F30E02150310996E0929FB00134
:1090C000939F700D1124FB01E458FA4F9081903268
:1090D00041F0AF0100E126E060E186E20E94BA675C
:1090E00005C0482F60E186E20E94EF2F29E046E2AA
:1090F0006FE085E20E94BC6A09C000E02091630233
:1091000048E551E160E186E20E94DE67D0E0BFE120
:10911000EB2E8D2F0E941F12E82FF0E0ED5AFE4E2D
:10912000C4916D2F809111070E942815AC0197FF03
:1091300002C04D5F5F4F5595479555954795411135
:1091400008C01816190614F441E003C0492F440F53
:10915000440B443E0CF444EE042F4D310CF00CE172
:109160008FEF8D0F46E38230C8F464E08C2F0E94AD
:10917000CB68D13021F08091620280FD0CC043E0C9
:109180006EE18FEF8C0F0E94CB6843E06EE181E0CF
:109190008C0F0E94CB686E2D601B14C06BE385EEB4
:1091A0008C0F0E94C968FF24FA94FC0E43E06AE326
:1091B0008F2D0E94C96843E06CE38F2D0E94C9681F
:1091C000C00F6BE3635027E047E08DEF8C0F0E94E8
:1091D0009C6ADF5FD43009F09CCF123008F040C0A9
:1091E000C5EED7E000E0FBE1FF2E49915991902FA9
:1091F0009370113029F19F9D802D1124043010F4BB
:1092000068E201C060E39A0157FF02C0215E3F4F50
:10921000E5E035952795EA95E1F7FA01E21BF30BB6
:109220009F0157FF02C041585F4F440F452F441F15
:10923000550B420F531F20E28F5D0E94186A0CC02D
:10924000043010F482E201C08EE5692F660F660FCC
:10925000690F6A5D0E9461240F5F083031F623C0F8
:109260001230A9F40E94F829C091DF08CC2329F01C
:109270008C2F880FC80FCC0FCC5F6C2F8AE00E9418
:10928000F43C63E06C0F84E60E94F43C0CC024E0E4
:1092900041E068E289E30E945F2520E840E060E366
:1092A0008FE00E94891380916608882399F14EE02F
:1092B0006FE182E09AE10E94BA2B1092650881303A
:1092C00049F590916808911103C08FE49CE220C099
:1092D000913039F4909309081092440886E593E59B
:1092E00017C0923061F480936508E0914901F0E085
:1092F000EE0FFF1FEF5AFE4F8081918109C093301E
:1093000019F48BE995E304C0943021F48DEC92E3D9
:109310000E946E1BDF91CF911F910F91FF90EF90F4
:109320000895AF92BF92CF92DF92EF92FF920F9388
:109330001F93CF93DF936C01162FC2ECD6E00E94EF
:109340000A1CF82E4091D5088417E1F1442361F0FE
:10935000EFEFE40F8AE0E89FF0011124E15EFA4F9D
:10936000808182958F7001C080E0FF2061F0EFEF77
:10937000EF0D9AE0E99FF0011124E15EFA4F908130
:109380009F70891718F08823D9F001C0892F682FA2
:1093900070E080E092E00E94447A7A83698381E001
:1093A00090E09C01042E01C0220F0A94EAF7388154
:1093B000322B0F2C01C0880F0A94EAF7382B388320
:1093C000F092D5081062E12E8881882329F11C8251
:1093D0001B828E01B12CAA24A39488818A21A1F03A
:1093E000BF1491F0B09211078B819C81F801258107
:1093F0003681820F931F9C838B836E2DC6010E9442
:10940000CC3FFE2DFF7DEF2EAA0CB3940E5F1F4FB5
:1094100085E0B812E2CF09C0FE01EF0DF11DEF0D9E
:10942000F11D80E094E696838583FE01EF0DF11D2A
:10943000EF0DF11D8B819C8125813681820F931F59
:109440009C838B83F09211076E2D6064C6010E948D
:10945000CC3F8881882309F43EC08091B3018823E2
:10946000D1F1FE01B0E0A1E080E094E625813681F3
:1094700018814A2F412331F10091B30169817A812A
:10948000069FA001079F500D1124BF1559F04217E8
:10949000530718F4241B350B17C02A2F20952123BE
:1094A000288310C0BC01621B730B4617570718F4C2
:1094B000240F351F09C02A2F20952123288320E05F
:1094C00034E602C020E030E036832583AA0FBF5F78
:1094D0003296B53059F6DF91CF911F910F91FF90E1
:1094E000EF90DF90CF90BF90AF900895FF920F93D1
:1094F0001F93CF93DF93F82ED62FC42F122F043152
:1095000061F190F4053001F138F4013009F446C0FE
:10951000023009F05BC021C00D3009F442C00E30AA
:10952000E1F00630E9F052C00432B9F028F4083115
:10953000A1F00B31F1F04AC0063379F00F3369F036
:10954000063209F043C009C02CEF240F2930F0F592
:10955000012F4EE251E188EE0AC067E271E138C0A6
:109560004230A0F5022F242F49E151E18CED8F0DFF
:1095700025C047FF06C065E171E18D2F0E94156887
:10958000CF77C73418F56FE071E18D2F0E94156811
:109590008C2F880F880FC80FCE5C1DC067E071E16B
:1095A00017C0423098F46FEF70E18D2F0E9415685C
:1095B000012F2C2F4BEF50E16D2F88E70E94DE67C3
:1095C000DF91CF911F910F91FF90089563EF70E1AC
:1095D0008D2F0E9415684C2F552747FD5095212F40
:1095E0006D2F8F2DDF91CF911F910F91FF900C94D4
:1095F000186A0F939CEF940F9D3138F450E042505D
:1096000051098E5E0F910C94186A413208F04D5149
:10961000022F242F40E85AE10E94DE670F9108953F
:10962000CF92DF92EF92FF920F931F93CF93DF932E
:10963000C82E8FE89DE00E94B526C091E6084C2F09
:1096400050E089E0C89FE0011124C653DA4F4F5F14
:109650005F4F60E084E50E94466A8C81877011F05C
:109660006AE001C069E08C2D0E946D27F82EE5E0CC
:10967000E8171CF066E67DE002C061E47DE088E06A
:109680000E94156810910708F5E0FF150CF4ADC0B5
:109690000E943D2AF11007C06EE288810E943E16AA
:1096A0008883212F01C020E0488168E080E60E9485
:1096B0004A1288818823D9F081500E94D9136C0105
:1096C0006CE37DE088E00E9415684881453250F0E7
:1096D000455222E0E22E00E0960168E088E40E9414
:1096E0006D2505C0A60168E088E40E94466A81E015
:1096F000F81207C066E089810E943E168983012F17
:1097000001C000E02981253018F446E95AE103C080
:1097100025504CE25DE060E18EE40E94DE67E2E00D
:10972000FE1210C084E680933D0122E040E05DE738
:1097300060E073E88D819E810E946C159E838D830D
:10974000212F01C020E048816D817E81453250F09B
:10975000455292E8E92E022F9B0168E188E70E94BA
:109760006D2505C0AB0168E188E70E94186AF3E047
:10977000FF120AC040915C01642F61958A810E94AA
:109780003B168A83212F01C020E04A8160E280E6F7
:109790000E94391384E0F81206C061E28B810E94B6
:1097A0003E168B8301C010E0212F4B8168E280E6DA
:1097B00020DF4C81469546954695437025E06CE048
:1097C0007DE080E30E9416278370880F880F880F42
:1097D0009C81977E982B9C83DF91CF911F910F9155
:1097E000FF90EF90DF90CF9008954C814295469581
:1097F000437026E06DE279E188E00E9416278370CD
:109800008295880F807E4C814F79482B4C8347FB93
:10981000442740F927E06EE979E180E10E941627AC
:109820004C8180FB47F94C83042F077028E0402FC0
:1098300068E179E188E10E94162787709C81987F12
:10984000982B9C83801711F018861F828C8187705B
:1098500009F467C061E07DE080E20E9415688C81B8
:109860008770813009F042C0E9E0FE120DC022E0AD
:109870004FEF51E060E070E08F8198850E946C1599
:1098800098878F83012F01C000E04F8158854C3F9E
:10989000F1E05F077CF0202F46EC58E160E28CE6B7
:1098A0000E94F0674F814B5C202F60E288E70E94A6
:1098B0002D6733C0453F81E058073CF0445F202FBF
:1098C00060E28CE60E94282628C0202F60E288E70C
:1098D0000E94186A002309F1E0E8CE1204C08F81CB
:1098E00098850E947E1610920D0817C08230A9F448
:1098F000F9E0FF120AC06FE08F810E943E16282F08
:1099000030E038872F83012F01C000E02F814DE028
:109910005BE160E28AE50E94DE678AE0D82E08E219
:1099200003C009E0D02E00E26AEF7CE0802F0E94A5
:1099300015684D2D50E0EF2DFF27E7FDF095E4175A
:10994000F507A9F480E8C81213C089E0FE0111925E
:109950008A95E9F710920D08FAE0FF1209C0E0912C
:109960004901F0E0E65BFE4F88E0808301C010E033
:10997000212F40EF5CE0602F88E4DF91CF911F91B1
:109980000F91FF90EF90DF90CF900C94F067CF9302
:10999000C62F20E04EE1682F80E00E945168809140
:1099A0001102803831F4C0938D0D87E492E20E9459
:1099B0006E1B10920D08CF9108951F93CF93DF93E4
:1099C000D82F162F237021F0223021F4C1E803C0D4
:1099D000C0E801C0CDE2612F8D2F0E94B8674C2FE7
:1099E000612F86E08D0FDF91CF911F910C94B867A6
:1099F00090910E08282F291B181644F4273014F0D4
:109A0000865005C027FD03C0892F01C080E08093E8
:109A10000E080895CF92DF92EF92FF920F931F935B
:109A2000CF93DF93C82F8BED99E10E94B5266FE0AD
:109A30008C2F0E946D27F82EDBDFD82ECE3211F04E
:109A4000C03669F4F7FC0BC0F092E4088C2F0E943A
:109A5000196D1092110284E99EE30E946E1B38E09A
:109A6000E32E0F2D112707FD1095CD2DD0E0CC242E
:109A7000C3940C171D0709F0C12C2C2D47E254E1AB
:109A80006E2D80E00E94F067AE014F5F5F4F88E06F
:109A90008D1510F486E101C081E12C2D6E2D0E9400
:109AA000186A88E0E80ED39480E4E812DECFF7FC71
:109AB00005C0F092E40884E60E94393EDF91CF9120
:109AC0001F910F91FF90EF90DF90CF9008956F92CC
:109AD0007F928F929F92AF92BF92EF920F931F93BC
:109AE000CF93DF9368E00E946D27A82E66EC78E1A3
:109AF00080E00E941568C091E60841E34C0F60E0E9
:109B00008CE00E94B8678A2D73DF782E45E24C0FF7
:109B100052E0E52E00E020E030E060E080E30E94CB
:109B20006D2540910E0863EE73E188E00E941A688B
:109B300018E0BB24A7FCB0948BE0C89FE00111247F
:109B4000CC56DA4F4E0187E0880E911C63E0662EFA
:109B5000872D90E0A816B90619F40091070801C0F6
:109B600000E0872D90E08930910508F090C0FC015D
:109B7000E058FF4F0C94957A202F4881612F82E4A2
:109B80000E944A12002309F482C06EE288810E947A
:109B90003E1688837CC001116092E50824E0A40190
:109BA000612F8091E4070E94732E71C049815A8110
:109BB000202F612F8EE40E94186A002309F467C0E9
:109BC00022E040E05DE760E073E889819A810E94CD
:109BD0006C159A8389835BC0402F6B81812F0E9413
:109BE000612A8B8354C0402F6C81812F0E94612A8F
:109BF0008C834DC0002329F067E08D810E943E16C2
:109C00008D832D814CEC58E1612F88E40E94DE6742
:109C10003EC0002349F08E8161E081700E943E16B3
:109C20009E8180FB90F99E838E8180FF02C04DE271
:109C300001C04BE2202F612F88E40E942D6727C0CE
:109C4000002361F08E81869562E083700E943E164B
:109C50008370880F9E81997F982B9E83EE81E69575
:109C6000E3704E2F50E0202F612F84E50E94186A88
:109C70000EC04E8143FB442740F928E061E979E1B9
:109C8000812F0E9416279E8180FB93F99E837394F7
:109C9000185F103409F05CCFDF91CF911F910F91C5
:109CA000EF90BF90AF909F908F907F906F900895AE
:109CB000DF92EF92FF920F931F93CF93DF93C82F02
:109CC00080ED93E10E94B52668E08C2F0E946D27FD
:109CD000082F8EDED82FC03861F480E80E94196DFD
:109CE00089E180930B08802F0E94AA6E81E00E9478
:109CF000E0774D2FE8E0FE2E112707FD1095493043
:109D000051F1C42FD0E0EE24E3940C171D0709F0A5
:109D1000E12CDD24D394D40E2E2D4D2D6F2D82E118
:109D20000E94486A80910B08882311F020E001C04E
:109D30002E2DFE01EE0FFF1FEB54FC4D459154916B
:109D40006F2D88E10E94F06788E0F80E80E4F81635
:109D500011F04D2DD4CFDF91CF911F910F91FF9036
:109D6000EF90DF9008957F928F929F92AF92BF9273
:109D7000CF92DF92EF92FF920F931F93CF93DF93D7
:109D8000C82E8091E2080E943912EC016EE08C2D01
:109D90000E946D27B82E83EC93E10E94B52620E047
:109DA000488160E08A5F0E9478128B2D21DED82ED8
:109DB00040910E0866E473E188E00E941A68F8E0BA
:109DC000FF2EA4E0AA2EB0E89B2EBD1003C0E090A9
:109DD000070801C0E12C0D2D10E00F30110508F02F
:109DE0006CC1F801E757FF4F0C94957A19812E2D1D
:109DF000AE016F2D84E50E94D32A153231F4198506
:109E00001295169517701B5D03C0163208F01A5F85
:109E1000EE2009F452C147E361E0812F0E943B1616
:109E2000853268F08C3210F0865009C085528295D8
:109E3000880F807E99859F71982B998785E2898309
:109E40003CC12E2D4A816F2D80E60E9486268A8392
:109E500034C12E2D48856F2D80E60E948626888786
:109E60002CC18F8143E06F2D83FB882780F90E94EE
:109E700021279F8180FB93F918C099818F819530AC
:109E800040F444E06F2D86FB882780F90E94432729
:109E900009C024E047E353E16F2D86FB882780F952
:109EA0000E9428279F8180FB96F99F8306C18F819E
:109EB00045E06F2D81700E9443279F8180FB90F9C0
:109EC000F4CF8F8187FD08C08C81855E863340F496
:109ED00010E045ED59E107C011E04BE253E103C04A
:109EE00012E041E353E12E2D6F2D86E00E94F067D2
:109EF000EE2009F4E2C062E0812F0E943E1618179E
:109F000009F4DBC0823011F49C8201C01C829F8165
:109F100080FB97F9CACF8F8187FF09C004E62CE93F
:109F20004C816F2D88E40E9440268C83C6C04C81F2
:109F30008BE1840F8733B8F010E8140F2E2D2064C6
:109F4000412F552747FD50956F2D86E60E94186AD0
:109F5000EE2031F044E66CE9812F0E943B16182F69
:109F600010581C83AAC02E2D6F2D8CE00E94432A0E
:109F7000EE2009F4A2C046E160EF8C810E943B16FE
:109F80008C8390E6C91299C087303CF0875080934B
:109F9000E40884E99EE30E946E1B8C8187FF8DC0DC
:109FA00080958093E40884E99EE30E946E1B85C03F
:109FB00001E0E11001C000E02E2D4B816F2D8EE4F9
:109FC0000E947E2A8B8379C0E110A092E5080FE3FE
:109FD00010E08824839477247A947F0C99859F716C
:109FE000982121E009F020E040E3410F6F2D802F00
:109FF0000E942D67EE20E9F08091E407811319C0DB
:10A0000029E048E0672D8FEF800F0E94BC6A80E254
:10A01000C81619F09EE2C9120CC08985982D9827A0
:10A020009F71807E892B898782E00E94096110924E
:10A030000D08880C1F5F095F153081F63EC04F8107
:10A04000469543702AE06FE073E18F2D0E9416273A
:10A050008370880F9F81997F982B27CF4D814F70F8
:10A060006E2D8F2D0E9468228F709D81907F0BC076
:10A070004D8142954F706E2D8F2D0E9468228295E2
:10A08000807F9D819F70982B9D8317C04E81429544
:10A090004F706E2D8F2D0E9468228295807F9E8149
:10A0A0009F7009C04E814F706E2D8F2D0E946822C7
:10A0B0008F709E81907F982B9E83D39488E0F80EBA
:10A0C00090E4F91282CEDF91CF911F910F91FF9012
:10A0D000EF90DF90CF90BF90AF909F908F907F9048
:10A0E00008952F923F924F925F926F927F928F923C
:10A0F0009F92AF92BF92CF92DF92EF92FF920F9317
:10A100001F93CF93DF93A82E85E099E10E94B52697
:10A11000E0914901F0E0E65BFE4F90808091E0071E
:10A12000882311F10E94A926882321F04CF0D2E661
:10A13000AD2E0AC0911008C083E6A81205C011C058
:10A14000992079F0C3E6AC2E292D30E08091E2070A
:10A15000992787FD90952817390721F4E2E6AE127A
:10A1600001C0A12CA092110280916608811106C045
:10A170006091E2078A2D0E946D27982E809111022E
:10A18000803641F08F3B19F08E32D1F403C010922B
:10A19000E00716C09091E007992339F01092E0078C
:10A1A00010920D08109244080BC09091660891110E
:10A1B00007C00E94196D109211027724739401C098
:10A1C000712C892D15DC582E809166088111109212
:10A1D00011028091E0078823E1F0809111029EE94D
:10A1E000980F9230B0F401E0823609F000E010914F
:10A1F000E208812F0E943912EC011111A2C1011154
:10A20000AAC18881823010F08150888382E00E9448
:10A21000096166246394B12C812CC52CD12C882D26
:10A220000E943912EC01B51488F06B2D70E06C19A6
:10A230007D096730710554F46F5F7F4F660F660FBD
:10A24000660F20E0462D81E00E947812FFE1F815AC
:10A2500008F4BEC028802610BBC02A96482C7E0178
:10A260008AE0E81AF108B51408F4A5C08B2D90E037
:10A270008C199D09873091050CF08BC00196382E02
:10A28000330C330C330C8091E007811112C09B100A
:10A2900010C04092E2082092E008772031F010923E
:10A2A0006708E1E0E0936608A12C11E08091660860
:10A2B000811110E0841459F0F7012781269523704D
:10A2C00000E04FE559E1632D83E10E94DE6720E065
:10A2D000A701632D80E30E94D32A212F8E0108500D
:10A2E0001109F8014081632D8DE20E948626F80154
:10A2F0008083FE0137974081442329F020E0632DBD
:10A3000088E40E943913FE01369740814423A9F066
:10A31000F701878187FF02C044E60BC08BE1840F01
:10A32000873330F420E0632D80E60E94432A05C085
:10A3300045E4632D80E60E94B867F70186818111AC
:10A3400002C040E201C043E5F7018581882329F07E
:10A35000433511F44AE201C044E4632D89E70E94C9
:10A36000B8678091E007882331F18091E10884117A
:10A3700022C020E046E6632D88E10E9451684092A9
:10A38000E208E0914901F0E0E65BFE4FB0829B2CD1
:10A3900012C0079781F48091E007882361F08091D3
:10A3A000E108841108C0E0914901F0E0E65BFE4F4E
:10A3B00080818F5F8083B3944394F0E24F1671F1F4
:10A3C0002A96FE013A978081821509F448CF26C06B
:10A3D0009B1022C06092E0088092E208692D6C19FF
:10A3E000660F660F660F695F29E049E180E00E9411
:10A3F000BC6A772089F00E94FF2A81110DC060E0BD
:10A400008091E2080E9487221092E00783EB9EE48D
:10A410000E946E1BB92C08C0B394482C639481E150
:10A42000681611F0842CFBCEB51428F18B2D90E02A
:10A43000851991090797FCF461E972E188E30E94AC
:10A440001568292D30E08091E207992787FD9095C6
:10A450002817390781F420E04EE768E380E00E9486
:10A460005168E0E6AE1619F0FEE2AF1204C088E5CE
:10A470009EE40E946E1B80916608882309F44CC0FC
:10A48000A09211024BE06FE384E598E10E94BA2BA1
:10A49000909168088130D1F5913079F40E94FF2ABB
:10A4A00081110DC08091E2088F5F8093E20860E027
:10A4B0000E9487221092E00702C0923018F483EBCA
:10A4C0009EE40EC0943079F48091E2088093E10715
:10A4D000809111020E94196D1092110283E39BE298
:10A4E0000E946E1B11C0953011F48FEFEFCF9230A8
:10A4F00041F48091E2088F5F8093E20861E00E945E
:10A50000872281E08093E007109266088091E2083C
:10A510008093E10810920D08B092E207DF91CF918D
:10A520001F910F91FF90EF90DF90CF90BF90AF9071
:10A530009F908F907F906F905F904F903F902F9063
:10A540000895113208F065CE103219F4002329F075
:10A5500060CE002311F01F5F01C01150812F0E94B7
:10A560003912FC0198818FEF890F803108F051CEAC
:10A570002081213108F04DCE291302C08BE009C0A3
:10A58000002309F442CE903108F040CE9F5F9883BB
:10A590003DCE815029F09081288121939993F9CF64
:10A5A0001093E10833CE9F92AF92BF92CF92DF9289
:10A5B000EF92FF920F931F93CF93DF93D82F8AEEE2
:10A5C0009CE00E94B52667E08D2F0E946D27C82F62
:10A5D0000FDAA82EDE3211F0D03659F4C8304CF420
:10A5E000C093E6088D2F0E94196D80E19BE40E94C4
:10A5F0006E1B18E0B12ECC2EDD24C7FCD09409E0F0
:10A60000902EEA2CF12C9E9CE0019F9CD00D1124F1
:10A61000C653DA4FA7014F5F5F4F07EE1CE020E003
:10A620006B2D81E10E94BB2620E048816B2D8EE1DD
:10A630000E944A1220E04A816B2D86E30E94391362
:10A6400020E04B816B2D8EE40E94F94A9C8197702B
:10A65000913021F0923039F441E401C043E26B2D96
:10A6600082E70E94B8678C81887129F048E46B2DDD
:10A6700088E70E94B867CE14DF0431F420E048E791
:10A680006B2D80E00E94516888E0B80EA39480E4AE
:10A69000B812B7CFDF91CF911F910F91FF90EF903C
:10A6A000DF90CF90BF90AF909F9008953F924F92D0
:10A6B0005F926F927F928F929F92AF92BF92CF9252
:10A6C000DF92EF92FF920F931F93CF93DF9392E06D
:10A6D0009093060867E00E942523E82E6091E70822
:10A6E00061500E946D27809163088630A1F038F494
:10A6F000813071F08530C9F483E090E314C08A3072
:10A7000069F08B3071F0883081F488E59EE40BC0ED
:10A7100081E790E508C08AE09DE405C088EF98E2F3
:10A7200002C083ED92E50E946E1BF0904B01D09029
:10A7300007080091630810E00F30110510F00C9429
:10A740008E5FF801E856FF4F0C94957A8FE09AE1FE
:10A750000E94B5268EE08093E70841E04F0D67E048
:10A760008BEC9CE00E94C5220C948E5F85EE97E1F5
:10A770000E94B5262AE02F1510F00E943D2A80E1A4
:10A780008093E70885E08F1508F4AEC0F11003C090
:10A7900089E08093E50801E0F11000E02AE041E55E
:10A7A00052E068E08091E4070E94732E91E0F91274
:10A7B00010C0E0E6EE1204C080915B020E94941685
:10A7C00061E380915B020E943E1680935B022D2D17
:10A7D00001C020E040915B0250E04C5F5E4F0AEB0D
:10A7E0001CE060E188E50E94BB2667E87CE088E128
:10A7F0000E94156808E028E0822E28E1922EC8E029
:10A80000D8E116E3AC2EA818FE01449168E1812F2F
:10A810000E94B8678A2D0E94AB14E82FF0E0EB5F2E
:10A82000F74E449168E186E0810F0E94B867145F9B
:10A8300021961E3739F7015011F7F2E0FF121AC0C6
:10A8400029E04AE467E185E30E94BC6A20E6E2165B
:10A8500019F08EE2E8120EC08E2D0E94196D0E9432
:10A860006B14809300059093120610920D0882E0FD
:10A870000E9409618091C20543E060E28295817087
:10A880000E9421279091C20580FB94F99093C20504
:10A8900094E0F9120AC0CD2DC06264E680910105F2
:10A8A0000E943E168093010501C0C0E2409101055F
:10A8B00050E02C2F68E288E70E94186A4091CD048E
:10A8C00042954695477025E06BE67CE080E30E9468
:10A8D00016278295880F807E9091CD049F71982BCA
:10A8E0009093CD040C948E5FEAE0EF1508F477C0E6
:10A8F00064E27CE088E00E9415688091670246E08F
:10A9000068E0869581700E9421279091670280FB04
:10A9100091F99093670291FF18C0C091C205C5FBE1
:10A92000CC27C0F927E04C2F64E17CE080E10E9455
:10A93000162781709091C20580FB95F99093C2050E
:10A940008C1791F00E94831B0FC0EBEAF3E080812B
:10A9500087FD1082818118160CF41182359623E050
:10A96000EB3FF207A0F3D9CFC091C205C6FBCC27BD
:10A97000C0F948E068E18C2F0E94212781709091F6
:10A98000C20580FB96F99093C2058C130E94831B2D
:10A990000E944012882311F041E801C040E860E2C3
:10A9A00080E60E94B8678091620249E068E28170A7
:10A9B0000E9421279091620280FB90F9909362029D
:10A9C0004AE060E394FB882780F90E942127909158
:10A9D000620280FB94F9909362020C948E5F60EEA9
:10A9E0007BE088E00E9415682BE0409163026EEBEB
:10A9F0007BE088E00E941627809363028CE0F812C7
:10AA000004C001E0D11003C001C0D12C00E02D2D05
:10AA10004091650260E186E60E947E2A809365028D
:10AA2000809162024DE068E183FB882780F90E94F3
:10AA300021279091620280FB93F9909362028091AA
:10AA40005D024EE060E2869581700E942127909120
:10AA50005D0280FB91F990935D0286EBC82E8BE03E
:10AA6000D82EE6011FE301E096E0B92EAC2EAC181B
:10AA7000FE01449180916602802321E009F420E0E8
:10AA800068E2812F0E942D67FFE0FF121DC0B09287
:10AA9000E5088091E4078A1117C029E048E067E2E1
:10AAA0008FEF810F0E94BC6A20E2E21619F08EE25D
:10AAB000E8120AC08091660280278093660282E0D5
:10AAC0000E94096110920D08000F2196195F10373E
:10AAD00069F60C948E5F8FE69BE10E94B5268AE0B2
:10AAE0008093E70894E09F1528F00E943D2AE12C0E
:10AAF00010E003C0EE24E39415E0E5E0EE9EE001F3
:10AB00001124CA5FDD4FD09007086EE478E088E03A
:10AB10000E94156841E34E0D68E08EE10E94B8671F
:10AB2000F11202C02D2D01C020E048815981022F71
:10AB300068E087E40E94566AF11214C08CE38093A7
:10AB40003D014CE364EC80E00E943B164881598152
:10AB5000480F511D87FD5A955983488357FF02C0FE
:10AB60001982188281E0810FF81207C063E18A819F
:10AB70000E943E168A8341E001C040E0E11002C01D
:10AB800021E001C021E860E18CE30E94891382E0AA
:10AB9000810FF81205C0DD2019F02D2D03E002C051
:10ABA00020E002E04B8168E18AE50E947E2A8B83E7
:10ABB00023E0210F4C8166E378E080E20E941627B3
:10ABC0008C831C5FF112D12CE11003C04091C005B1
:10ABD00002C04091C105DD2011F003E001C002E098
:10ABE0002D2D68E28FE40E947E2AE11003C080933D
:10ABF000C00502C08093C105E6E0F2E0808191814A
:10AC000090935F0280935E02828180935C028381D5
:10AC10008093CC0480915D02948190FB80F98093B5
:10AC20005D02858196819093FD048093FC04878169
:10AC30008093FE0480858093FF048091C2059185F6
:10AC400090FB87F98093C2050C948E5F80EF99E1A9
:10AC50000E94B52686E08093E708C09107086BE65E
:10AC60007BE088E00E941568409167024295469516
:10AC7000477020E063E57BE088E00E94162782951C
:10AC8000880F807E909167029F71982B9093670246
:10AC9000F1E0FF1209C064E2809168020E943E1652
:10ACA000809368022C2F01C020E04091680260E18F
:10ACB00086E60E944A1222E0F21208C064E6809101
:10ACC00069020E943E168093690201C0C0E0409173
:10ACD000690250E02C2F68E184E50E94632741E07F
:10ACE00083E0F81240E08091670260E282FB8827EF
:10ACF00080F90E944D279091670280FB92F9909312
:10AD0000670241E094E0F91240E08091670268E256
:10AD100083FB882780F90E944D279091670280FB72
:10AD200093F99093670241E0E5E0FE1240E08091E4
:10AD3000670260E3829581700E944D2790916702BF
:10AD400080FB94F9909367020C948E5F88EE99E1F2
:10AD50000E94B52685E08093E70810925A01D091B1
:10AD6000E30820E0F11009C043E060E08D2F0E946D
:10AD70003116D82F8093E30821E041E04D0F68E0C1
:10AD800080E00E944A128D2F0E948F26182F00E02B
:10AD9000282F47E45BE068E08AE20E94DE6767E212
:10ADA0007BE088E00E941568ED2FF0E0EE0FFF1FBA
:10ADB000E15DF74F40815181453651052CF44C3906
:10ADC0005F4F24F0C2E003C0C0E001C0C1E08D2F9E
:10ADD0000E94051A811106C0CC2329F081E0F812E7
:10ADE00002C002C0C0E080E0EE24E39400E0212F26
:10ADF00048E168E10E94112EC13011F081E0F812A3
:10AE000080E0E12C00E0212F48E160E30E94112E58
:10AE1000CC2319F081E022E0F21280E0EE24E394EA
:10AE200001E0212F48E268E10E94112EC13019F0A3
:10AE300081E092E0F91280E0E12C01E0212F48E26C
:10AE400060E30E94112E81E0E3E0FE1280E0E12C3D
:10AE500000E023E640E36EE10E94112E81E0F4E081
:10AE6000FF1280E0E12C00E022E648E36EE10E9460
:10AE7000112E8091E3080E94051A882311F08CE3BB
:10AE800001C08CE540E460E00E94CB6881E08093E3
:10AE9000410961E08CE50E94DB3D8091E308E82FE9
:10AEA000F0E0EE0FFF1FE15DF74FC081D181BE01E1
:10AEB0000E94673D8C0189E18C9F90018D9F300D30
:10AEC000112437FF02C021503F4F532F550F550B10
:10AED000432F60E382E70E94466A89E1809F9001E8
:10AEE000819F300D112437FF02C021503F4F532F57
:10AEF000550F550B432F68E084E50E94466ACE014A
:10AF0000409697FF02C0CE018F967C01C5E0F59474
:10AF1000E794CA95E1F7E8016096D7FF02C0E8011F
:10AF2000AF96B5E0D595C795BA95E1F7D195C1959E
:10AF3000D1096C2F635E47E08CE58E0D0E94CB68D3
:10AF40006C2F605E47E089E58E0D0E94C968109203
:10AF50004109E4C7D0916002DF70CD2FD13041F0BC
:10AF6000D23021F0D53021F014E003C013E001C04D
:10AF700017E086EB99E10E94B5261093E708D09080
:10AF80000708E090E40767E17BE080E00E94156835
:10AF9000F11013C08091620267E0829586958770F8
:10AFA0000E943E168295880F807E909162029F716A
:10AFB000982B9093620221E001C020E04091620250
:10AFC0004295469547704F5C60E082E70E942D678E
:10AFD000DD2349F08DE08D0F8F70CC24C394823037
:10AFE00020F0C12C02C0CC24C39421E0F21202C094
:10AFF000EE2011F000E001C00D2D2D2F4BEE5AE098
:10B0000068E084E20E94DE67CC2081F167EE7AE09E
:10B0100088E00E94156881E0F81202C0E81611F07D
:10B0200000E001C00D2D209161022E5F49EC5AE035
:10B0300068E088E40E94DE6791E0F91203C0E2E074
:10B04000EE1611F020E001C02D2D40916402F2E3D4
:10B050004F02A0011124445D5E4F68E080E70E942A
:10B06000186A21E0F21279C082E01AC040916102B0
:10B07000D53009F44F7081E0F81202C0E81611F0E3
:10B0800020E001C02D2D552747FD509502EC1AE018
:10B0900068E08EE70E94BB2691E0F9127FC081E054
:10B0A0008093E50880910C08882309F463C0E1E0EF
:10B0B000EE1661F0EE1620F0F2E0EF1689F13AC0DC
:10B0C00066E08D2F0E943E16C82F34C0CC2019F0A8
:10B0D00044E06EEF1EC0D530D1F490914E059073D0
:10B0E000809161028F706FE3892B0E943E16982F2A
:10B0F0009F7020916102207F920F90936102807374
:10B1000090914E059F7C982B90934E0513C04FE372
:10B1100060E0809161020E943B16809361020AC048
:10B12000CC2041F04AE06CEF809164020E943B1613
:10B130008093640280916002982F9F70807F2C2FF3
:10B140002F70822B809360029C1310926102809179
:10B150005D028B7F80935D020DC022E0F2120CC075
:10B1600044E16CEE80916A020E943B1680936A0271
:10B1700021E203C0CC2091F020E240916A0285E0F8
:10B180004802A00111244F515F4F03EB1AE060E128
:10B190008CE40E94BB26D3E018E105C0C63009F05C
:10B1A000CFC6D2E010E16AEA7AE0812F0E941568EA
:10B1B0004091670241702D2F60EA7AE0812F0E9452
:10B1C00016279091670280FB90F990936702185FB1
:10B1D000CC24C394CD0EC53009F050C280914108F3
:10B1E000811102C010926A0889E18093410864E7E6
:10B1F0007AE0812F0E94156820914E05237090E41B
:10B20000299F90011124B0904205EB2DEF73BE2EC3
:10B21000B22AFC1007C06FE78B2D0E943E16982EB5
:10B220002D2D02C09B2C20E0C92DD0E0F3E4F915B0
:10B2300048F0022F292D4AED58E0612F8CE30E943F
:10B24000DE6707C0AE014F5F5F4F612F8EE70E9440
:10B25000186A892D8F7390914205907C890F809395
:10B260004205A6E0D595C795AA95E1F72C2F237046
:10B2700090914E059C7F922B90934E05A090610279
:10B280009B100BC04A2D50E0F4E055954795FA9578
:10B29000E1F7242F2770B22E01C0B12C78E0972E51
:10B2A000910E91E09C0DE6E0CC0FDD1FEA95E1F7F1
:10B2B0008F738C2B09F478C0833009F478C0813007
:10B2C00009F478C0853009F478C0873009F478C073
:10B2D000883009F478C0893009F478C08A3009F4DC
:10B2E00078C08B3009F478C08C3009F478C08D3088
:10B2F00009F478C08E3009F478C0803109F478C040
:10B30000813109F478C0833109F478C0893109F4B6
:10B3100078C08B3109F478C08C3109F478C08D3154
:10B3200009F478C08E3109F478C0813209F478C00C
:10B33000833209F478C0843209F478C0863209F483
:10B3400078C0893209F478C08C3209F478C08D3223
:10B3500009F478C08E3209F478C0813309F478C0DA
:10B36000823309F478C0833309F478C0843309F454
:10B3700078C0863309F478C0893309F478C08D33F6
:10B3800009F478C08E3309F478C08F3309F478C09B
:10B39000803409F478C0813409F478C0823409F02B
:10B3A00078C0C2E6D4E177C0C1E7D7E174C0C7E591
:10B3B000D7E171C0C3E6D7E16EC0C9E3D7E16BC086
:10B3C000C4E1D7E168C0C6E0D7E165C0C6EFD6E109
:10B3D00062C0CAEED6E15FC0C7EBD6E15CC0C6EA88
:10B3E000D6E159C0C8E9D6E156C0C2E8D6E153C09B
:10B3F000C7E6D6E150C0C7E4D6E14DC0CBE3D6E105
:10B400004AC0C1E2D6E147C0C3E0D6E144C0C5EFBF
:10B41000D5E141C0CFECD5E13EC0C5EBD5E13BC0A5
:10B42000C2E8D5E138C0C4E6D5E135C0C0E5D5E114
:10B4300032C0CCE3D5E12FC0CAE2D5E12CC0C9E1CE
:10B44000D5E129C0CDE0D5E126C0C1E0D5E123C0DA
:10B45000C7EFD4E120C0C2EFD4E11DC0CDEED4E1EE
:10B460001AC0C5EED4E117C0C5EDD4E114C0C0EDDB
:10B47000D4E111C0C6ECD4E10EC0C4EBD4E10BC0E2
:10B48000C4E9D4E108C0CAE7D4E105C0C4E7D4E107
:10B4900002C0C3EDD8E0F91207C067E08B2D0E940F
:10B4A0003E16B82E2D2D01C020E0FE0184918B1593
:10B4B00050F0AE014F5F5F4F022F2B2D692D8CE3B3
:10B4C0000E94DE6706C04B2D50E0692D82E40E9489
:10B4D000186A8A2D8F78F0E1BF9E800D1124809329
:10B4E000610260E1B62EB10EC2E0CC0DDA2DDD1F97
:10B4F000DD27DD1FFC1202C0EE2011F000E001C0CC
:10B500000D2D2D2F49EC58E06B2D84E20E94DE6753
:10B5100040914E05437020E4429FA0011124009108
:10B5200042050F73042BFC1203C081E0E81611F0F2
:10B5300020E001C02D2D409143056B2D8EE70E9428
:10B54000764AFC1223C081E08093E508E1100FC029
:10B5500080910C088823D1F061E08D2F0E943E1667
:10B560009A2D9F7781119068909361020FC091E0AE
:10B57000E9120CC080910C08882341F04FE760E885
:10B58000809143050E943B168093430548E1B42E09
:10B59000B10E53E0A52EAC0CC0914205C6FBDD27D1
:10B5A000D0F9FA1003C0E1E0EE1611F000E001C09E
:10B5B0000D2D2D2F45E159E16B2D88E70E94DE67A7
:10B5C000FA101BC081E08093E508E11005C061E03E
:10B5D0008B2D0E94C74C11C0F1E0EF120EC080917C
:10B5E0000C08882351F061E08D2F0E943E169C2F9D
:10B5F0009F7B8111906490934205105EC4E0CC0D56
:10B6000080916A0880FF35C048E2612F80E20E9485
:10B61000B86749E2612F8FE40E94B8674EE2612F5C
:10B6200089E20E94B8674EE2612F83E30E94B86707
:10B630004EE2612F81E40E94B86740916C08405D42
:10B64000612F84E20E94B86740916D08405D612FD0
:10B650008EE20E94B86740916E0850E0612F81E44D
:10B660000E94466A40916F0850E0612F8FE40E946B
:10B67000466AFC1253C460E2812F8DC0C23081F44F
:10B6800060EC78E0812F0E9415682C2D40914205D6
:10B6900061EA78E0812F0E941627809342053EC41C
:10B6A000C13009F03BC460E878E0812F0E94156842
:10B6B00080914205833049F569E778E0812F0E9447
:10B6C0001568FC1004C0C093E50821E0E21220E0F8
:10B6D00090914D05492F429543708091600280738F
:10B6E000803229F4907C19F466E779E102C063E6C0
:10B6F00079E1812F0E94C82683708295807F909186
:10B700004D059F7C982B90934D05FC1002C021E0C5
:10B71000E11020E04091420567E474E1812F0E942E
:10B72000C8268093420540915D0242FB442740F9C0
:10B7300021E02C0D60E474E188E0810F0E9416275F
:10B7400090915D0280FB92F990935D0240916002BE
:10B750004295437022E02C0D66E574E180E1810F93
:10B760000E94162783708295807F909160029F7C53
:10B77000982B9093600283E08C0DF81205C061E075
:10B7800088E1810F0E94C74C84E08C0DF812C6C37B
:10B7900060E280E2810F0E94C74CC0C385E298E05E
:10B7A0000E94B5268CE08093E70883E08093E5084B
:10B7B000B090E4078F2D0E94F84C982E38E0D32EDD
:10B7C000F91003C08090070801C0812C4CE46D2D56
:10B7D00080E00E94B86728E0291510F448E301C012
:10B7E00041E3490D6D2D85E00E94B86781E0B816F0
:10B7F00029F092E0B91629F0712C01C0782CA12C07
:10B8000002C0A82C712C492D50E0EA01CC0FDD1F9D
:10B81000C40FD51FC955DB4FBB2011F000E001C09C
:10B82000082D2A812F7046E95AE16D2D8DE00E9486
:10B83000DE678A818F700E943312C82E81111CC06E
:10B84000188115327CF015526981812F0E94BB242A
:10B850009C0192E8E92E0A2D412F6D2D84E60E946D
:10B860006D2523C04981552747FD50952A2D6D2D03
:10B8700083E60E94186A19C0E1E08E130DC0272DDF
:10B8800048816D2D86E30E9439132A2D49816D2D43
:10B890008DE40E94391334C0F2E08F130DC02A2DBD
:10B8A00049816D2D80E50E944A12272D48816D2D1A
:10B8B00086E30E944A1224C0488147FF04C0409595
:10B8C000272D2062722E552747FD50954F5F5F4F01
:10B8D00001E218E0272D6D2D89E40E94BB264981E5
:10B8E00047FF04C040958A2D8062A82E552747FD4A
:10B8F00050954F5F5F4F2A2D6D2D8BE60E94186A81
:10B900004A8142954F7049300CF04F5F93E0B91671
:10B9100011F020E001C0282D6D2D88E60E9439131A
:10B9200080910C08882309F462C0882009F45FC064
:10B93000E1E0BE1631F1BE1698F0F2E0BF16D9F183
:10B9400023E0B21254C08A816FE082958F700E940A
:10B950003E168295807F9A819F70982B9A8347C06C
:10B960008A816EE08F700E943E168F709A81907F60
:10B97000982B9A830E943312C816C9F11882198233
:10B9800036C081E0C81659F0C81690F092E0C9168A
:10B9900079F0E3E0CE122BC043E66EEC04C0409198
:10B9A0005C01642F619588810E943B1688831FC0CB
:10B9B0004EE260E0F8CFF1E0CF1671F0CF1648F01C
:10B9C00022E0C21671F083E0C81211C043E66EECAB
:10B9D0000AC04DE763E807C040915C01642F6195A0
:10B9E00002C04EE260E089810E943B1689839394F5
:10B9F00098E0D90EE0E4DE12E3CE90C28BEF99E13D
:10BA00000E94B52681E18093E70883E08093E508F2
:10BA1000A090E4078F2D0E94F84C982EFFE0FF15B0
:10BA2000A0F0EF2DF0E0EE0FFF1FEB51F84F40813B
:10BA3000518157FF02C04F5F5F4F55954795445264
:10BA40005A4F60E08EE40E94466A8091110280386D
:10BA500019F52FE02F1540F14F2D50E0FA01E919AB
:10BA6000F109EE0FFF1FEB51F84F20813181A1103A
:10BA700013C085E0849FF001859FF00D1124E555EA
:10BA8000FC4F8281882319F0319521953109348347
:10BA9000238382E0BED3B9D4B8E0EB2EC5E05C2EA0
:10BAA000DAE0CD2ED12C8EC080E1F812F5CF89E1FD
:10BAB00080930B0880E80E94196D0E941247ECCF1A
:10BAC000E92DF0E05E9EE0015F9ED00D1124C5558A
:10BAD000DC4FEE0FFF1FEB51F84F808191814A81BF
:10BAE0002B813C81442319F0319521953109821B2A
:10BAF000930B833391050CF069C08E3C9F4F0CF47F
:10BB000068C01DE266246394690C20E0462D6E2D0A
:10BB100080E00E947812412F6E2D8BE40E94B8675E
:10BB20008091670281FF59C07DE7772EB12C472CA9
:10BB3000419433243A943E0CF91052C0AB1050C0DB
:10BB40002091070880910C08882309F44BC0222318
:10BB500009F448C010925A01822E80910105882371
:10BB600009F44EC00B811C810115110509F03CC080
:10BB7000C801B6010E94447AF1E0BF1609F449C039
:10BB8000BF1608F042C020624B815C816E2D8DE2B1
:10BB90000E94186A882059F022E048EE53E068E1DC
:10BBA0007CEF8B819C810E946C159C838B83B3946A
:10BBB000E4E0BE12C1CF88E08E0D803409F482C06B
:10BBC000E82E962C90E199127BCF6EC0411103C0F4
:10BBD000BBC14111B9C11FE795CF64E6762EA6CF50
:10BBE00020E0B0CF812CB9CF90E0801791075CF0B6
:10BBF000919581959109081719070CF0B9CF03C0E9
:10BC000000E010E0B5CF8C01B3CF82E0B816E9F0C8
:10BC100040C018811456AB01410F511D17FD5A95B4
:10BC200043389FEF590714F443E85FEF6E2D88E423
:10BC30000E94186A882009F4BACF49E1642D812F47
:10BC40000E943B168C598883B2CF89818C59AB01F5
:10BC5000480F511D87FD5A954E37510514F04DE799
:10BC600050E06E2D86E60E94186A012B31F029E023
:10BC700048E3632D82E30E94BC6A882009F497CFD1
:10BC80008981472D67EE8C590E943B168456898323
:10BC90008ECF422F6E2D8A810E944D2791E0811117
:10BCA00001C090E09A8383CF21E0F0E1FF1220E011
:10BCB00080910B0881114AC140E158E06E2D82E16C
:10BCC0000E94F0672BC180E098E00E94B52689E1D0
:10BCD0008093E708C090E4078F2D0E94F84CD82E7F
:10BCE00038E0E32E40E1B42E52E0A52E8091CD0441
:10BCF000D11021C0F11010C01092E508C0910708C2
:10BD000060E18F710E943E168F719091CD04907EFC
:10BD1000982B9093CD0401C0C0E04091CD044F71A9
:10BD200050E0485F5F4F00EF17E02C2F6E2D8CE640
:10BD30000E94BB26EDC08F719B2C981ACD2DD0E0B0
:10BD4000FD1002C0A092E508C131D1052CF4CC0F42
:10BD5000DD1FC453DB4F04C0CC0FDD1FC05DDA4FC5
:10BD6000812CFD1008C0C81006C0009107080023F0
:10BD700019F012E002C000E010E09D1408F444C085
:10BD8000811014C020E04D2D6E2D80E00E947812AD
:10BD9000488147FB442740F9212F6AEE77E08E2D3A
:10BDA0000E94C826988180FB97F91DC0F1E08F1290
:10BDB0001CC070905C014881440F4595202F6E2D6A
:10BDC00085E40E943913112309F49EC060915C013F
:10BDD00061958881880F472D85950E943B168F7746
:10BDE00098819078982B98838FC04981552747FD7B
:10BDF0005095202F6E2D88E70E94186A112309F4B0
:10BE000083C04DE763E876C0811022C067EE77E01B
:10BE10008E2D0E94156820E04D2D6E2D86E10E942A
:10BE2000486A112369F040915C014150888160E0CB
:10BE30008F730E943B168F739881907C982B988308
:10BE400048814F73202F6E2D89E10E9439135CC009
:10BE5000488121E0821211C0429546954695437073
:10BE6000212F6BEC77E08E2D0E94C8268295880FDB
:10BE7000880F807C98819F73B5CF842F829586959B
:10BE80008695837049818330D9F4403F24F049304E
:10BE90001CF049E001C040EF498347FF09C0242F4F
:10BEA00020954DE05BE16E2D8BE50E94DE6706C0BC
:10BEB0004F5F202F6E2D80E60E94AE2349E010C018
:10BEC0004B3F38F450E0202F6E2D86E60E94186A12
:10BED00006C0485F202F6E2D84E50E9428264FEF74
:10BEE000112391F0888182958695869583708330A1
:10BEF00029F460EF89810E943B1605C08981642F77
:10BF000090E00E9443168983839483E0881229CFAE
:10BF1000D39498E0E90EE0E4EE12E8CEDF91CF9101
:10BF20001F910F91FF90EF90DF90CF90BF90AF9057
:10BF30009F908F907F906F905F904F903F9008956B
:10BF400082E0C82E10E147C91EE7DCCD20E0B4CE68
:10BF50001F93CF93DF93EC011AE088810E94592E42
:10BF60000E94692E89931150C1F7DF91CF911F91E3
:10BF700008959C01265F3F4FFB014491DC014D93E6
:10BF8000CD013196A217B307C1F70895E6E3F6E0B5
:10BF900080E090E021913191820F931F26E0EE34F2
:10BFA000F207C1F7089587E7E5E3F6E0DF011D92A8
:10BFB0008A95E9F78BE08093350689E180936306E3
:10BFC0008AE58093640681E0809379068091780603
:10BFD000877C88608093780686E180936606E6E336
:10BFE000F6E020E034E080E093E021933193958700
:10BFF0008487938F828FB6E0E434FB07B1F76CE45B
:10C000007DE186E896E0B5DFC1DF9093610680931D
:10C0100060060895EF920F931F9361E0680F88EC1C
:10C02000E82E04EE13E021E532E042E082EF98E0F2
:10C0300048D621E0843E934009F020E0822F1F91F2
:10C040000F91EF900895CF93C82FE1E5F2E01192A0
:10C0500086E0E533F807D9F761E47DE181E592E018
:10C0600088DF8C2F90E06AE070E001960E94447AAD
:10C07000605D60935602805D8093570284E08093F8
:10C08000410582E08093630280E00E94AA6E809165
:10C090007B06806280937B068C2FCF91BBCF0F9362
:10C0A0001F93CF93DF93EB01042F803120F561E0E4
:10C0B000680F82EF98E056D410E0A80160E270E0CB
:10C0C000CE010E94B57A4AE050E0BE0182EF98E0CE
:10C0D000CCD40A9781F482EF98E036D4C00FD11FF8
:10C0E000009749F06AE070E00E94447A805D8A938C
:10C0F000862F972FF5CFDF91CF911F910F91089544
:10C100008F5FDAC361E0680F82EF98E02BD484EE92
:10C1100093E0E1E5F2E0DF019C011D922150304007
:10C12000E1F744EE53E0BF0182EF98E09EC4FF9236
:10C130000F931F93CF93DF93CDB7DEB768970FB6FA
:10C14000F894DEBF0FBECDBF01E0080F102F1031F5
:10C15000B0F4FF24F394F10E8F2DAED381110DC0F6
:10C16000602F82EF98E0FED361E0610F28E532E0B6
:10C1700042E0CE01409655D506C01F2DE8CF1031C4
:10C1800079F780E017C04FE050E0BE016F5F7F4F4E
:10C1900082EF98E004D4882349F0482FBE016F5FF6
:10C1A0007F4FCE014096C4D4A895EDCFCE014096E6
:10C1B0005ED581E068960FB6F894DEBF0FBECDBFA6
:10C1C000DF91CF911F910F91FF900895EF920F9300
:10C1D0001F9389E09DE10E94491B87EF9CE10E942B
:10C1E00048142ED398ECE92E07E710E025E336E05B
:10C1F00041E060E082EF98E064D58737910521F057
:10C2000088EE9CE10E94491B80E01F910F91EF9006
:10C210001ACFCF93C82F8770A1F09091FD08982B6B
:10C220009093FD080E942C129093FC088093FB08C9
:10C230008C2F90E024E0959587952A95E1F78093DF
:10C24000FE08CF910895CF93DF931CD3811102C0D4
:10C2500080E02EC095D287FDFBCF60E082EF98E0B2
:10C2600081D387E7E5E3F6E0DF011D928A95E9F7E0
:10C2700047E750E0BF0182EF98E0F7D386E896E009
:10C2800067DE809135068B3040F481E08093CD01EC
:10C290008BE08093350681E0BCDFC0916006D091D1
:10C2A000610674DE21E0C817D90709F020E0822F6B
:10C2B000DF91CF910895EF920F931F93CF93DF9368
:10C2C00010924009C091FD08CC2309F498C09091C8
:10C2D000FE089F5C9093400981111CC00E942C12A3
:10C2E0002091FB083091FC08821B930B883C910540
:10C2F00008F485C08091FE08882361F08150809306
:10C30000FE08882339F00E942C129093FC08809339
:10C31000FB0875C01092FE088091E80881116FC07B
:10C32000DC2FD470C2FD02C081E001C083E08093A5
:10C33000E808C0FF2CC082E3809340098091FD088B
:10C340008E7F8093FD0844E1E42E07E710E025E3AB
:10C3500036E041E061E189EE98E0B3D4873791059A
:10C3600019F461E180E02FC08091EF08823051F430
:10C370008091FD08816030C08091EF08823029F102
:10C38000D1113BC087E59DE10E94491B36C0C1FF2A
:10C3900034C083E3809340098091FD08897F8093B6
:10C3A000FD0834E1E32E04EE13E021E532E042E043
:10C3B00061E189EE98E085D4843E9340E9F680916E
:10C3C000620661E18F5F86D218C08091FD08D111AD
:10C3D00002C0826001C086608093FD080E942C121A
:10C3E000885C91099093FC088093FB0880918F0DE5
:10C3F000833019F4A89510928F0D1092E808DF9100
:10C40000CF911F910F91EF9008958091FD0888239F
:10C4100051F081E050DF80918F0D8330B1F7A89506
:10C4200010928F0DF2CF0895EF92FF920F931F930A
:10C43000CF93DF93C82F803108F0BFC063DE8F3FFA
:10C44000910509F010F48C2FFEDD81E592E080DD8E
:10C450008091F904811107C08091620286958370F2
:10C460008E5F8093F90480916002982F9295969543
:10C4700096959370933029F090934205806C809349
:10C48000600280914105823008F062C010E0812F87
:10C490000E943912EC0189818150843018F40E9485
:10C4A0001F1289831F5F103291F7C7EAD4E000E0C2
:10C4B00010E08A818F700E943312882389F08230C5
:10C4C000C1F4C80188559B4F7C01FC018081882301
:10C4D00039F085302CF481500E941F12F7018083BF
:10C4E0008881882331F0853024F481500E941F1206
:10C4F000888323960D5F1F4F04321105D1F688E320
:10C50000EBEFF3E0AAE6B8E001900D928A95E1F72F
:10C51000CAE6D8E010E00EE0812F0E941F12815081
:10C52000089FD0011124A550BC4FFE01802F01901F
:10C530000D928A95E1F71F5F2E96143069F78CE211
:10C540009DE10E94491B82E08093410562DE5DDF30
:10C55000809141058330F8F480E090E0FC01E955DA
:10C56000FB4F2281322F3F703C3019F4207F2A602C
:10C5700022832281322F3F703D3019F4207F2B60BF
:10C58000228303968432910549F783E08093410525
:10C5900082E03FDE3ADF80914105843070F4809183
:10C5A00090068093000589E19DE10E94491B84E08B
:10C5B0008093410582E02DDE28DFE6E0F2E0809105
:10C5C0005C0282838091CC04838380915E0290918F
:10C5D0005F029183808380915D028170848380916A
:10C5E000FE0487838091FF0480878091FC049091F2
:10C5F000FD04968385838091C20587FB882780F997
:10C60000818780914105853008F044C09091CD0428
:10C610009F7180E1891BEEECF4E020E0281789F19E
:10C620003081932F929596959695937071F09330F3
:10C6300059F43068932F990F990F959595959F7799
:10C640003078392B308301C010822F5F3296E6CFCD
:10C65000E82FF0E0EE0FFF1F8031B0F0EE5CFA4FF4
:10C660009081929596959770933008F093E0292FDA
:10C670002295220F220F207C90819F71922B908314
:10C680008F5F883128F303C0E253FB4FE9CF86E088
:10C69000809341050E9484330E948A33DF91CF91B9
:10C6A0001F910F91FF90EF90089540E450E060E0FB
:10C6B00070E08FEF98E00C94716B41E050E062E025
:10C6C00070E081E099E00C94716BCF93DF931F923F
:10C6D000CDB7DEB7698390E1899FB001112441E0B5
:10C6E00050E0CE010196FDD70F90DF91CF910895D4
:10C6F000CF93DF931F92CDB7DEB790E1899FB00152
:10C70000112441E050E0CE0101960E94BC7A89815B
:10C710000F90DF91CF910895CF93DF93D82FC82F3B
:10C720008C2FE6DF882321F08C2FE2DFC82FF8CF93
:10C73000609101098C2FC9DFD0930109DF91CF915E
:10C74000BCCFCF93C0910109CC2341F08C2FD0DF17
:10C7500080930109B2DF60E08C2FB7DF8C2FCF917F
:10C760000895CF93DF9380910109C0E0D0E0882342
:10C7700019F02F96BDDFFBCFCE01DF91CF91089549
:10C78000DF92EF92FF920F931F93CF93DF9380E896
:10C79000E1E5F2E0DF011D928A95E9F7C3E0D9E017
:10C7A000F12CB4E1FB1205C08091010901E019E010
:10C7B00002C08E01888190E0E12CDD24D394DF0C4F
:10C7C0000097E9F09C01245031092C37310530F4F1
:10C7D000FC01EF5AFD4F2081222361F0EE2021F071
:10C7E00060E08E2D72DF03C0F80110825EDF80E012
:10C7F00090E0E6CFD082E82E7BDF90E0E1CFF394AB
:10C800002396F5E1FF12CDCFC4E0D0E0FE01EF5A50
:10C81000FD4F8081811107C0609101098C2F55DF88
:10C82000C09301094ADF2196C038D10579F780E02D
:10C83000DF91CF911F910F91FF90EF90DF900895BE
:10C84000CF9380E4EFEFF8E0DF01982F1D929A95E7
:10C85000E9F794E09093FF088093000980E18093CA
:10C86000020984E0C1E0C80F6C2F2FDFCF3711F031
:10C870008C2FF8CF60E08FE728DF84E080930109F8
:10C88000CF9113CF40E450E060E070E08FEF98E08C
:10C890000E94BC7A80910009811103C080E48093DA
:10C8A00000098091FF08843029F481E0909100090B
:10C8B000903409F080E0089590E0FC01EE0FFF1F36
:10C8C000E80FF91FE150F74F81E09481911101C009
:10C8D00080E00895CF93DF9390E0EC01CC0FDD1F53
:10C8E000C80FD91FC150D74F8C819D81AE8170E098
:10C8F000FB01EE0FFF1FE60FF71FE150F74F2481FA
:10C90000358146812C833D834E8384839583A68322
:10C91000DF91CF91CACECF9390E09C01220F331FBD
:10C92000280F391FF901E150F74FC481F901ED5F7C
:10C93000F64F108211821282B8DECC2319F08C2FB0
:10C94000CF91EACECF910895FC01808190E0FC0167
:10C95000EE0FFF1FE80FF91FEC5FF64F918180810A
:10C960009F700895CF93DF93FC0160831282118240
:10C9700070E0CB01880F991F860F971FEC01C15003
:10C98000D74F2C812383148215821682FC01EB5F22
:10C99000F64F808182958F70DF91CF910895AF928D
:10C9A000BF92CF92DF92EF92FF920F931F93CF939C
:10C9B000DF931F92CDB7DEB78C01FC01808190E040
:10C9C000FC01EE0FFF1FE80FF91FEC5FF64F8081AF
:10C9D0002181922F9F70F80121813281821B930B5C
:10C9E0007A018417950708F47C015B016701C11483
:10C9F000D10421F1F8018381882301F164816F5F03
:10CA0000648370E0F0E18F9F600D711D112441E09F
:10CA100050E0CE0101960E94BC7A8981F501819394
:10CA20005F01F80184818F3028F01482838160DEF9
:10CA3000F8018383F1E0CF1AD108D9CFF8018181C1
:10CA400092818E0D9F1D8C199D09928381838E2D5D
:10CA50008C190F90DF91CF911F910F91FF90EF9064
:10CA6000DF90CF90BF90AF9008957F928F929F926A
:10CA7000AF92BF92CF92DF92EF92FF920F931F93EC
:10CA8000CF93DF934C016B018A01C0E0D0E05C01E1
:10CA900025E0A20EB11CC017D107D8F5F40185819D
:10CAA0008F7781F0F4014581F42FFF777F2E2F2FB0
:10CAB00030E0C8018C1B9D0B8217930758F4702E31
:10CAC0007C1A08C041E050E0B501C40168DF813044
:10CAD00049F31FC0E72CF12CC6018C0F9D1F47FFA7
:10CAE00006C0A70160E070E00E94B57A0BC0A70104
:10CAF000BC01C40154DF871529F0FE01E80FF11DC8
:10CB0000CF0108C0CE0DDF1DF40185818719858313
:10CB1000C2CFCE01DF91CF911F910F91FF90EF9087
:10CB2000DF90CF90BF90AF909F908F907F900895AF
:10CB3000AF92BF92CF92DF92EF92FF920F931F932B
:10CB4000CF93DF93EC018B01D42E8B81811110C028
:10CB500089819A81892B61F4E880F12CF2DD8B8345
:10CB6000F701EE0FFF1FEE0DFF1DE150F74F84831D
:10CB7000CD2C8FE0A82ECC2009F43CC0EF80F884A7
:10CB80000E942C12E81AF90AF7FE02C082E004C0E3
:10CB90008B81811103C081E08E832CC09C819F30EA
:10CBA00058F01C82A5DD811104C0CBDD682F8B817C
:10CBB0008CDD8B819DDD8B838B81882361F36C8180
:10CBC0009A2D961BBC2C9C1508F4B92EEB2CF12C3D
:10CBD00070E090E1899F600D711D11246F5F7F4FA0
:10CBE000A701C8017ED50E0D1F1D8C818B0D8C8376
:10CBF000CB18C1CF6D2D70E06C19710929813A8174
:10CC0000260F371F3A8329838D2D8C19DF91CF9101
:10CC10001F910F91FF90EF90DF90CF90BF90AF905A
:10CC20000895EF92FF920F931F93CF93DF93EC0140
:10CC3000F62EE42E890196DE6F2D70E0FB01EE0FDB
:10CC4000FF1FE60FF71FEC5FF64F1082E29430EF04
:10CC5000E322E1820E942C12800F911F98878F831C
:10CC6000DF91CF911F910F91FF90EF9008951F9347
:10CC7000CF93DF93EC01888190E0FC01EE0FFF1F62
:10CC8000E80FF91FEC5FF64F898180839A819F70CE
:10CC90008181807F892B81838B81882321F028DD0E
:10CCA000182F81110AC010E000DD112311F0812F2F
:10CCB00033DDDF91CF911F91089560E08B8105DD19
:10CCC000F3CF7F928F929F92AF92BF92CF92DF92DB
:10CCD000EF92FF920F931F93CF93DF931F92CDB7E5
:10CCE000DEB76C0159012E2D30E09BDF1982450122
:10CCF000E12CF12C77247394F40181914F019981F7
:10CD0000811108C071104CC08081811105C0772449
:10CD100073941BC071100AC080E09F3718F4E016AE
:10CD2000F10661F5772081F0782E01C0712C9923EE
:10CD300029F19068998341E0BE016F5F7F4FC60182
:10CD4000F7DE8130D1F026C0782E9923B9F041E08A
:10CD5000BE016F5F7F4FC601EBDE8130D9F44981A0
:10CD6000B701641B71096A0D7B1DC601E1DE998163
:10CD7000891719F0981B99830DC0198289818F5FDB
:10CD80008983A895FFEFEF1AFF0A0E151F0508F01B
:10CD9000B3CF08C089818F778701081B110902C0B2
:10CDA000872DBBCFC60163DFC8010F90DF91CF9104
:10CDB0001F910F91FF90EF90DF90CF90BF90AF90B9
:10CDC0009F908F907F900895E2E4F9E011928DE0BA
:10CDD000E234F807D9F70895FF920F931F93CF938A
:10CDE000DF93FA01149131967491795F7695769577
:10CDF0007695DA011396FA0132964491249FA00D9C
:10CE0000B11D112466956695669590E0F0E86F9FD8
:10CE1000800D911D112420E030E060E08E5B964F84
:10CE2000412F50E0671799F00A2FEC01C20FD31F72
:10CE3000FD01FE2EF01AF11620F4F490F9923196CD
:10CE4000F8CFA40FB51F6F5F20583F4FEBCFDF9196
:10CE5000CF911F910F91FF900895CF93DF93382FBB
:10CE6000463128F4842F880F840F880F7EC086E017
:10CE7000830F20FD08C021FD02C090E005C0909105
:10CE8000550D96FFFACF91E0687FA32FB0E050E1F7
:10CE9000659FA00DB11D1124AE5BB64F22FF3DC0B2
:10CEA0004E3211F088E0830F24ED240F2F3010F460
:10CEB0004B5211C02FEB240F2A3110F441530BC0F9
:10CEC0002FE9240F2A3110F4465305C04F3511F4D1
:10CED0004AE201C040E06EE0469FA00111244F5895
:10CEE000524E27E0FA0134913796E491211102C0A5
:10CEF000E0E030E04F5F5F4F992311F03095E0950F
:10CF0000FCE0A13CBF0730F43C93ED01C058DF4F7B
:10CF1000E8831196215030F728C023FF07C0892FDE
:10CF200081958D9385E0830F31E001C030E025E0ED
:10CF3000429FF0011124E956FF4D25E0449133232F
:10CF400011F0243041F05DE0A234B50718F49111DE
:10CF500040954C931196215031962111EFCF6DE001
:10CF6000A234B60710F491959C93DF91CF91089568
:10CF700020E073CFEF92FF920F931F93CF93DF9335
:10CF8000F62E122F902F9071E92EFA01112379F0CD
:10CF9000EE2011F0408101C04491EF01219644231D
:10CFA00031F0202F6F2D59DF1150FE01EFCFDF91AF
:10CFB000CF911F910F91FF90EF9008950F93FA0179
:10CFC00094914F5F5F4F929F400D511D1124292F67
:10CFD000D1DF0F9108950F9300E0CCDF0F910895FA
:10CFE000FF920F931F93CF93DF93162F022F922F51
:10CFF0009071F92EEA01FF2011F0488102C0FE0174
:10D000004491442361F04F3131F4185F103438F407
:10D0100080E02196F0CF202F612F1FDFFACFDF9124
:10D02000CF911F910F91FF900895AB0120E0682FE1
:10D0300080E0D6CFFB01442341F09491992351F035
:10D040009F3109F441503196F6CF20E0AF01682FAF
:10D0500080E0C6CF089520E0C3CFFF920F931F93C7
:10D06000CF93DF93082FF62EEA0114E1180F155025
:10D070004C2F4F704A301CF0495C28E002C0405DE4
:10D0800020E06F2D812FE9DE84E0D695C7958A9543
:10D09000E1F71013ECCFDF91CF911F910F91FF902B
:10D0A0000895222321F09091550D96FD0895480F83
:10D0B000687FE82FF0E090E1699FE00DF11D1124F9
:10D0C000EE5BF64F8E1B982F9E0F941720F49081E5
:10D0D00090959193F8CF08952DE08234920760F4F3
:10D0E000FC01208130914109332319F0262B313086
:10D0F00009F02627FC0120830895262F287F6770DA
:10D10000E62FF0E0EA5DFC4D649190E030E1239F72
:10D11000800D911D11248E5B964FDECFEF92FF9212
:10D120000F931F93CF93DF93F42E47FF02C0840F1A
:10D13000F194962F987FC82FD0E080E1989FC00D82
:10D14000D11D1124CE5BD64F6770E62FF0E0EA5D6B
:10D15000FC4DE490FF20B1F08DE0C234D80790F48C
:10D16000022F10E020FF08C06E2DCE01B5DF15950F
:10D170000795202F206803C015950795202FFA9456
:10D180002196E8CFDF91CF911F910F91FF90EF9003
:10D1900008952FEFC3CF1F93CF93DF93142F47FF33
:10D1A00002C0640F1195962F987FC82FD0E080E1C0
:10D1B000989FC00DD11D1124CE5BD64F862F87704E
:10D1C00099F0E82FF0E0EA5DFC4D64916195180F4D
:10D1D000185017FF0DC0E12FFF27E7FDF095E25D26
:10D1E000FC4DE4916E0F04C018303CF018506FEF06
:10D1F000CE0172DFC058DF4FF7CF111654F4E12F84
:10D20000FF27E7FDF095EA5DFC4D64916150CE018A
:10D2100063DFDF91CF911F9108953F924F925F920C
:10D220006F927F928F929F92AF92BF92CF92DF9236
:10D23000EF92FF920F931F93CF93DF93182FB62E89
:10D24000802F05FF04C004FF04C002E003C000E01B
:10D2500001C001E0982F9F77C92EE7FE04C0E1943A
:10D260006624639401C0612C57FF0AC05095409515
:10D27000309521953F4F4F4F5F4F7724739401C0F6
:10D28000712C82FF06C098E09093420DE8E0DE2EFC
:10D2900005C096E09093420D75E0D72E86FF28C01A
:10D2A00071101D0D283E83E038074105510514F02B
:10D2B0001D0D05C0243631054105510514F01D0D25
:10D2C00005C02A303105410551050CF01D0D002324
:10D2D00081F0023031F424363105410551054CF41A
:10D2E0001D0D2A303105410551051CF41D0D01C0ED
:10D2F0001D198091420D810F8093420D023011F46F
:10D3000090EFC90E8824839452E0A52E912CFF241F
:10D31000E7FCF09466E0562E5B0CE82DF0E0EE168C
:10D32000FF060CF45DC06AE070E0C9010E94447A17
:10D33000382EEB0140E3442E480E2C2D442D6B2D4E
:10D34000812F8BDD08112FC0C2FE1AC08FEF830D15
:10D35000833008F4A394CE016AE070E00E94447A1E
:10D36000823011F08430D9F484E3481204C0992447
:10D370009394910E15C099249A94910EA39410C081
:10D380003EEF432E410E8FEF810FC0FE04C047E0F9
:10D390006B2D01DF02C0652DB0DE142D01C0912E72
:10D3A000209709F000E09E01442737FD4095542F57
:10D3B000211531054105510581F4002331F002307A
:10D3C00059F491E0981540F008C0C4FE09C06110FE
:10D3D00004C080EFC80E01C000E01D1983949DCFEA
:10D3E000992059F09A944A2D6CE06B0D892DD1DE6D
:10D3F0004A2D6DE06B0D892DCCDE772031F02C2D80
:10D400004DE26B2D812F8D1928DD80E0DF91CF91CA
:10D410001F910F91FF90EF90DF90CF90BF90AF9052
:10D420009F908F907F906F905F904F903F90089566
:10D43000EF920F93022F9A01442737FD4095542F06
:10D44000F5E0EF2EEADE0F91EF900895CF93DF9392
:10D45000D62FC22F206250E0EBDFC7FD08C02C2F73
:10D4600046E76D2F8091420DDF91CF91F6CCDF9191
:10D47000CF91089590913C0120916406921710F489
:10D4800022E001C020E0242B492FE0CF20E0D0CFC4
:10D49000EF920F93022F005F242F30E040E050E026
:10D4A000A2E0EA2EBADE0F91EF900895DF92EF929C
:10D4B000FF920F931F93CF93DF93182FE62EEA016D
:10D4C000F22E822F8470D82E22FF05C01D5F57FFD9
:10D4D0000FC087E103C057FF0BC08FE02F2D4DE237
:10D4E0006E2D912F981B892FB8DCD195C195D1094C
:10D4F0002F2D20234AE36E2D812FAFDC6CE370E0EB
:10D50000CE010E94447A462FC82FD1101E5F2F2DC6
:10D510006E2D812FBDDFDD2011F085E101C08FE090
:10D52000810F202F4C2F6E2DDF91CF911F910F91E6
:10D53000FF90EF90DF90ACCF0F931F93CF93DF93CB
:10D54000C82FD62F142F022F422F25DE123030F095
:10D55000402F6D2F8FEF810F8C0F1DDE6FEF6D0F42
:10D56000600F412F8C2F15DE412F6D2F8C2FDF91F7
:10D57000CF911F910F910DCECF93C091410991E0B2
:10D5800090934109D9DFC0934109CF9108950F933A
:10D590001F93CF93DF93182FC62FD22FE42FF0E0E5
:10D5A0003297053608F004E60E9FC0010F9F900DDC
:10D5B000112464E670E00E94447A062F2D2F6C2F10
:10D5C000812FDADF002361F0D150DC0FCF5F1F5FC6
:10D5D000CD1730F4402F6C2F812FDBDDCF5FF8CFDC
:10D5E000DF91CF911F910F910895A998AB988BBBB4
:10D5F000AD9AAD98AB9AA99A0895CF93C82F81E0C0
:10D6000080933F0981E8F1DF8C2FEFDF10923F0913
:10D61000CF91089580916306F0CFCF93DF9381E09F
:10D6200080933F09AA982AE02A95F1F700C0AA9AA8
:10D630008CED95E0E5E0EA95F1F7000001970097A1
:10D64000C9F7AC98C7E6DDE1FE018491CEDF2196F3
:10D65000FDE1C137DF07C1F7DF91CF91DBCF1F932A
:10D66000CF93DF9340914009442321F08091550DE1
:10D6700086FD32C081E080933F0910EBC2E4D9E01F
:10D6800084E0B3DF80E1B1DF812FAFDFA998AB9AEF
:10D69000FE019E0120583F4F80818BBBAD9AAD9813
:10D6A00081818BBBAD9AAD9882818BBBAD9AAD98D1
:10D6B00083818BBBAD9AAD983496E217F30761F77F
:10D6C000EF01AB9AA99A1F5F183BD1F610923F0960
:10D6D000DF91CF911F9108954A5260E080E059DDBB
:10D6E000C9CFBF92CF92DF92EF92FF920F931F9319
:10D6F000CF93DF937B018A01080F191FEC01E81A11
:10D70000F90A6701CC0EDD1EC017D107C1F0B99030
:10D710008091E8088270E19B05C08823E1F30E94B4
:10D72000951DF6CFDFBACEBAE09A8DB3B81649F39D
:10D73000BDBA8FB7F894E29AE19A8FBFE2CFDF913A
:10D74000CF911F910F91FF90EF90DF90CF90BF90FE
:10D750000895FC0180818F70880F611181608F7046
:10D760009081907F982B908381818F5F81838281CC
:10D77000882351F09F7041F4833621F0842F80621A
:10D780008093860D118212828281883061F140F48B
:10D79000813079F180F0823031F18430E9F523C0B5
:10D7A0008F35C1F018F48031F1F00895813649F0D9
:10D7B000823661F1089580818F708F3069F581E63E
:10D7C00029C040664093860D1092360110923501B3
:10D7D0008FE520C08181803211F4406814C0883206
:10D7E000D9F480E117C09181903318F08695828337
:10D7F0001182828190E00197218130E0822393237E
:10D80000892B51F440644093860D089581818034C2
:10D8100018F088E08283118208955091630041B12D
:10D82000282F30E02F3031056CF4F901EE0FFF1F87
:10D83000E20FF31FE75AF24F90819F7081E09F3013
:10D8400051F52AC090E0FC013F97E930F10518F549
:10D85000E955FF4F0C94957A942F947019C091B1AB
:10D86000927016C0952F10C0952F9095987010C08B
:10D8700053FF11C091B102C0942F9095907408C0CD
:10D88000942F907105C0942F917002C0942F9072C4
:10D8900081E0911101C080E008958D3208F0A3C0AD
:10D8A0009FEF980F993010F4825FB7CF51EE580F69
:10D8B0005330D8F491B1909594705523C9F04091AC
:10D8C000A5064F70415021E030E0042E01C0220F28
:10D8D0000A94EAF73091580D3223523041F0932BDD
:10D8E00021E009F020E0922F03C090E001C0932FC7
:10D8F0005EED580F5330E0F4409163004095417065
:10D900005523A9F09091A6069F70915021E030E038
:10D9100001C0220F9A95EAF79091580D9223523048
:10D9200039F0942B21E009F020E0922F01C0942FD0
:10D930005BED580F5330F8F491B19695917021E05A
:10D9400092275523C1F04091A50642954F70415052
:10D9500021E030E0042E01C0220F0A94EAF7309152
:10D96000580D3223523031F0932B21E009F020E0A2
:10D97000922F01C0932F88528330E0F491B190959B
:10D980009071882369F14091A60642954F704150ED
:10D9900021E030E0042E01C0220F0A94EAF7309112
:10D9A000580D3223823009F1932B81E009F080E099
:10D9B000982F16C0833019F42091A70605C0843033
:10D9C00079F42091A70622952F70215081E090E0F4
:10D9D000022E01C0880F0A94EAF79091580D9823FF
:10D9E00081E0911104C080E00895932FF9CF08954C
:10D9F000CF93C82F52DF811107C081E08C0F4DDF1C
:10DA0000882321F081E003C080E001C082E0CF9153
:10DA100008958F7090E08F30910551F0FC01EE0F6A
:10DA2000FF1FE80FF91FE75AF24F82E68283118247
:10DA300008958F7090E08F30910549F0FC01EE0F52
:10DA4000FF1FE80FF91FE75AF24F83E6828308951C
:10DA5000EF92FF920F931F93CF93DF938091560D18
:10DA60009091570D01969093570D8093560D80938A
:10DA7000550D96B390958091870D882321F0282F1E
:10DA80002877292349F4892F807609F07AC093FDFD
:10DA900074C094FF74C080E1182F1660192380931E
:10DAA000870DC9E5DDE000E011FB662760F9402F36
:10DAB000CE014FDE0F5F169523960630A9F78091B1
:10DAC000100281110EC0F0B2F0948091920686FF90
:10DAD00009C08F2D837FF82E80915E0E8C70F82AFE
:10DAE00001C0F12CCEE2D3E200E010E046E0E42EEB
:10DAF000EC1AFE0184914C2F4E0D8F2161E009F448
:10DB000060E0C8018559924F24DE21960D5F1F4FBA
:10DB10000831110571F78091160261E0C82FC072BB
:10DB200085FF60E04EE083E89DE013DE86B38095DC
:10DB30008E778C2B19F089E08093590180915E0ECD
:10DB400086FD02C0817402C0817082609091630082
:10DB500092FF88609091630095FF8062989B84603B
:10DB60009C9B8064B79B80618093580DDF91CF911F
:10DB70001F910F91FF90EF90089588E08DCF80E086
:10DB80008BCF80E689CF929A1092980089E180939A
:10DB9000990080919B008D7F80939B0086E080930D
:10DBA0009D0080919B0087FF03C080919C00F9CF6E
:10DBB00088E980939A00089581E080938B0D80938B
:10DBC00010028091920686FFDECF08958091920622
:10DBD00086FF10929A001092100283C790919B00CA
:10DBE00095FFFCCF80939C000895E3E4FDE09189CC
:10DBF0008089891749F0DF01A90FB11D8C919F5FC2
:10DC00009F70918B90E008958FEF9FEF08951F9282
:10DC10000F920FB60F9211242F938F939F93EF9330
:10DC2000FF9380919A008F7780939A007894E09187
:10DC3000530D81E08E0F8F7090919C002091540DB8
:10DC4000821731F0F0E0ED5BF24F90838093530D3B
:10DC5000F89480919A00806880939A00FF91EF91E8
:10DC60009F918F912F910F900FBE0F901F9018953D
:10DC700095E0899FD0011124A95CBB4FCB0105968B
:10DC8000FB0124912D933196E817F907D1F70895F8
:10DC90000F931F93CF93DF93182FCBE6D2E090E042
:10DCA0008881181738F0882329F0903201F19F5F9E
:10DCB0002A96F6CF9032D9F02FE130E0291B3109B6
:10DCC0000AE0029FA001039F500D1124BE01CE0166
:10DCD0000A960E94A47AFE0111920A95E9F7188328
:10DCE00084E68A838F8188608F83CE0102C08BE6B1
:10DCF00092E0DF91CF911F910F910895EBE6F2E052
:10DD0000119283E0EB3AF807D9F7089588E2E7E348
:10DD1000F4E0DF011D928A95E9F788E4EFE5F4E08D
:10DD2000DF011D928A95E9F7089590E00197FC01C3
:10DD3000EE0FFF1FE80FF91FE955FB4F6F7062836D
:10DD4000408321830895CF93C62FA2DFFC01C183B6
:10DD5000CF9108959F92AF92BF92CF92DF92EF92B0
:10DD6000FF920F931F93CF93DF9300D000D0CDB7D6
:10DD7000DEB7182FE0917E06F0E0EF59FC4FE491FA
:10DD800084E09E2F9370A1E0B0E0AC0FBD1FA90FFF
:10DD9000B11D8C93E695E695815099F7111108C055
:10DDA000ADDF61E08981CFDF62E08A81CCDF3AC0FC
:10DDB000113041F4EB81F0E0EE0FFF1FE453FB4F15
:10DDC00081E009C0123089F4EB81F0E0EE0FFF1F13
:10DDD000E453FB4F81E880838091C20585FF02C038
:10DDE00080E001C08CE9818309C1133009F586DF29
:10DDF0000981802F4DDFFC01EE24E394E1821EECCB
:10DE00001283802F45DF02E0FC0101831283FA8038
:10DE10008F2D3EDFFC01E18212838F2D39DFFC0163
:10DE20000183128363E08B818EDF64E08C8121C0EB
:10DE3000143009F563DFFA808F2D2ADFFC0122E020
:10DE4000E22EE1820EEC02838F2D22DFFC01118392
:10DE50000283FC808F2D1CDFFC01E18202838F2D69
:10DE600017DFFC011183028361E089816CDF63E0CD
:10DE70008B8169DFC3C0153009F092C03FDF46DFF8
:10DE800081E006DF4AE0C42EFC01C18282E000DFAF
:10DE90005BE0D52EFC01D18283E0FADE6CE0F62E49
:10DEA000FC01F18261E084E04EDF85E0F1DEFC01FF
:10DEB00003E0018374E0B72EB38287E08483878117
:10DEC0008160878385E0E4DEFC0101831383A8E0A1
:10DED0009A2E948287818160878385E0D9DEFC0158
:10DEE0000183B6E0EB2EE38289E0A82EA48287812D
:10DEF0008160878385E0CCDEFC0191828CE982839E
:10DF000081E083838781897F8460878386E0C0DEA8
:10DF1000FC01A1828EE1828388EF83838BE0B8DEEF
:10DF2000FC01018396E4A92EA282B382C482878178
:10DF3000816087838BE0ACDEFC010183A2821383C6
:10DF4000D4828781816087838BE0A2DEFC0101831C
:10DF5000A282E382F4828781816087838091670255
:10DF60008F718062809367028FE1809368026AE418
:10DF700073E280E07DDE65E473E281E079DE60E4F7
:10DF800073E282E075DE6BE373E283E071DE66E3E9
:10DF900073E284E06DDE66E373E285E069DE2EC045
:10DFA000163099F486E074DEFC01118382E38283EB
:10DFB00098EF9383808786E06BDEFC0111838EEC03
:10DFC000828398E09383808719C0173021F018303E
:10DFD000A9F488E001C080E15BDEFC0189E0818377
:10DFE00084E6828384E1838387E786838EE080935F
:10DFF000C70488E08093C5048093C60482E00E9431
:10E0000009610F900F900F900F90DF91CF911F91AA
:10E010000F91FF90EF90DF90CF90BF90AF909F90C7
:10E020000C94056280E49CE99BBD8ABD87B7806142
:10E0300087BF1FBC8AE08EBD08950F931F93CF93B7
:10E04000DF9310916202129516951770882331F0B4
:10E05000A1EEBDE0833021F420E103C0A9E9BDE0D9
:10E0600028E090916102990F910F920F60916402E4
:10E0700024E66202B0011124685A7D4F00916A02C1
:10E0800048EE53E004039001059F300D11242853FE
:10E090003045261B370BFD0132966D937C934091E2
:10E0A000670241FF03C040E055E002C040E054E099
:10E0B000833011F418EF190FCC27DD27C41BD50BC3
:10E0C0001917F0F4A12FB0E0AA0FBB1FAB51B84F46
:10E0D0000D90BC91A02D4A175B070CF4DA01AC1728
:10E0E000BD070CF4DE01A854B44F2A1B3B0BA61B42
:10E0F000B70BB183A083738362831F5F3496E0CF35
:10E10000283293E2390710F428E233E23183208386
:10E11000882331F0285E33403093890D2093880D99
:10E1200013821282DF91CF911F910F9108951F9258
:10E130000F920FB60F9211242F933F938F939F93BB
:10E14000EF93FF9388B391E0892788BBE0910E019C
:10E15000F0910F013081832F8F708F3039F0209133
:10E160002B0E829F202D1124215001C02FEF822FD2
:10E1700090E097BD86BD832F82958F7031F43196E4
:10E18000F0930F01E0930E0101C08083293C60F001
:10E19000809160028F70863031F48091670280FD3B
:10E1A00002C0C09801C0C09A80918F0D8160809399
:10E1B0008F0DFF91EF919F918F913F912F910F9034
:10E1C0000FBE0F901F9018951F920F920FB60F92CF
:10E1D00011242F938F939F93EF93FF9388B391E034
:10E1E000892788BBE0911001F0911101208188B549
:10E1F00099B520FD02C0809601C0409699BD88BDAA
:10E20000822F869569F4CF01019690931101809336
:10E2100010018181811105C087B7877F87BF01C049
:10E22000808380918F0D816080938F0DFF91EF919E
:10E230009F918F912F910F900FBE0F901F90189567
:10E24000EDE7F0E08081857E808317981F9AAAE829
:10E25000B0E01C9210928B0082E88C9380818062E7
:10E2600080830895EDE7F0E080818F7D8083179AA9
:10E27000AAE8B0E01C9210928B008AE08C93808117
:10E280008861808308951F920F920FB60F92112418
:10E290008F939F93EF93FF938091290E882321F012
:10E2A0001F9A1092290E04C01F9881E08093290EB6
:10E2B000E0910A01F0910B01808191819093870098
:10E2C000809386008091880D9091890D90938500B0
:10E2D0008093840082819381892B11F0329608C04B
:10E2E00080916702809581708093290EE1EEFDE0B8
:10E2F000F0930B01E0930A0180918F0D8160809370
:10E300008F0DFF91EF919F918F910F900FBE0F9006
:10E310001F901895E0E9FDE09081969596952781EC
:10E32000222311F096959695982B908321812F5F4B
:10E3300021838085281750F0A281B3819D012F5F32
:10E340003F4F338322839C93108211820895FF9262
:10E350000F931F93CF93DF93C82F809160028F702C
:10E36000823069F09C2F88E0D0E0292F2078D20FEE
:10E37000990F8150D1F7D07899E0F92E03C088E049
:10E38000F82ED0E810E080E190E00C2F017090139F
:10E3900002C0805F02C0BEDF80E1C695CD2B1F5F4B
:10E3A000F11618F0D0E8902FF0CF805FDF91CF9179
:10E3B0001F910F91FF90AECF882339F08091960D79
:10E3C0008F5F8093960D80E803C01092960D80ECCD
:10E3D000A1DF8091960D8530C0F70895CF93DF932C
:10E3E000C82F8091950D8C27E82FEF70F0E0EE0F8D
:10E3F000FF1FE953FC4D6591749182958F7041E840
:10E4000050E1849F9001859F300D11245091940D0F
:10E4100040E024273527262737273093950D209372
:10E42000940DD8E08C2F8078C7DFCC0FD150D1F776
:10E43000DF91CF910895CF9380EC6CDFC6E080E848
:10E4400069DFC150E1F780ECCF9164CF8031E0F417
:10E45000E82FF0E0EE0FFF1FEB51F84F20813181E4
:10E46000C901880F991F820F931F97FD03969595F9
:10E470008795959587959C5F1816190644F48E3FED
:10E4800027E092073CF4089580E094E0089581E04D
:10E4900090E008958EEF97E008954F925F927F92FB
:10E4A0008F929F92AF92BF92CF92DF92EF92FF92A4
:10E4B0000F931F93CF93DF931F92CDB7DEB7809159
:10E4C0004E05837020E4829FC0011124F090420524
:10E4D000EF2DEF73FE2EF82AF3948F2D8F7390E0BB
:10E4E000809714F084E501C085E590E9492E9DE010
:10E4F000592EF2012F0129E93DE033832283108256
:10E5000011821582148291E0978392E09087109196
:10E510008A0D009160020F70023009F057C080E14F
:10E5200080932B0E16FF0CC080914205882321F0AA
:10E53000813021F410E906C010E804C018E902C0D7
:10E5400017FF05C087E169D9882309F4F8C017FDD2
:10E55000F8C085E10E94291B882309F4F2C01062EB
:10E56000812FF5DE10938A0D80916102F0DE05EEB9
:10E5700017E0F12C8DE0D82EF801819191918F0157
:10E58000D89E9001D99E300D1124B5E03595279580
:10E59000BA95E1F73E5F37FD07C02F3FF3E03F0735
:10E5A00034F4E22E832F06C0E12C80E003C0EE2479
:10E5B000EA9483E09F2D990F990F892BC8DE8E2D49
:10E5C000C6DEF39426E0F212D7CF95C094E1909383
:10E5D0002B0E063011F48FE014C0B9DE1091420505
:10E5E0001F5F1F7580918D0D80FD106885FD106285
:10E5F000812FADDE10938A0D80916102A8DE80919B
:10E600004305A5DE8090620282948694E7E08E2224
:10E6100010E0C12CD12CE12C912CF5E0AF2EB12CC7
:10E62000A8EF7A2EE12FE80DF0E0EE0FFF1FEB517F
:10E63000F84F80819181880F991F880F991F1816B4
:10E6400019061CF424E030E002C02CEF3FEF820FEB
:10E65000931FB50119D79B01053011F43C5F02C02F
:10E6600020523C4F37FD07C0211588E038072CF0B9
:10E670002FEF37E002C020E030E0442737FD40951F
:10E68000092C03C0220F331F441F0A94DAF7C22A51
:10E69000D32AE42AEBE0E90DE9838C2D58DECD2C5A
:10E6A000DE2CEE24F981F850F983F830B0F793E0CE
:10E6B000990D892F869586958695992E879D900C24
:10E6C00011241F5F103109F0ADCF063021F480E036
:10E6D0003EDE80E00FC09091920697FB992790F95B
:10E6E000990F990F990F80914E058073892B9F2D5B
:10E6F000907C892B2CDEF2018181A281B381882359
:10E7000019F08FE08C9304C0FD018291806F8083AB
:10E7100089E99DE090930F0180930E010F90DF91A6
:10E72000CF911F910F91FF90EF90DF90CF90BF900E
:10E73000AF909F908F907F905F904F9008951F773C
:10E7400006CF1F7D0DCFCF92DF92EF92FF920F93F6
:10E750001F93CF93DF93C0916002CF7080918106A9
:10E7600085FF04C080914D028111C4E080918B0D22
:10E770008111CFEF80918E0D8C1709F467C0C09383
:10E780008E0D1EBC1DBC1CBC87B7837C87BF8091CF
:10E790007D008E7F80937D008CE386BF8FE3809326
:10E7A0007C008C2F90E08730910508F04FC0FC0171
:10E7B000E055FF4FBAC644DD35DC19C141DD88E5BF
:10E7C0009BE199BD88BD80EA9FE09093790080939A
:10E7D000780087B7886087BF80917D0081608093D3
:10E7E0007D001FBC82E08EBD48C02ADD88EC90E031
:10E7F00090937900809378008CE291E09DBD8CBD70
:10E8000080EE9BEA97BD86BD87B7806287BF809107
:10E810007D00816080937D001FBC8AE18EBD16C0A3
:10E82000C43021F484E009DCC09803C0FBDB83E042
:10E8300004DC80E593EC909387008093860088E861
:10E8400093E190938500809384000CDDC33009F43C
:10E85000CEC028F4C13089F008F4C9C0C5C0C530A5
:10E8600008F4C7C0C73008F4BFC0CF3F09F0C1C02B
:10E8700088B391E0892788BBBCC07894F0902B0EB8
:10E8800087B7877F87BF80917D008E7F80937D00D3
:10E89000E0E9FDE089E99DE090931101809310018A
:10E8A0008AE99DE09383828315821482108211820B
:10E8B0001682178284E080878FEF8093990DBBDDED
:10E8C000809161028BDD40918D0D8091420540FF6A
:10E8D0000CC090E489029001112480916002869519
:10E8E000869586958670822B04C020E48202C00142
:10E8F0001124842B73DD80E071DDE0906202E294EC
:10E90000E69447E0E4228F2D8170D82EF0FE02C0FD
:10E9100098E0E90E38E0C32ECE0C8E2D97DD8C01E9
:10E92000D110185F802F5ADD81E08E0D8FDDEC0154
:10E93000D110D85FE394E3949C2F9295907F812F20
:10E940008F70892B4BDDCE0124E0969587952A9513
:10E95000E1F744DDEC10E1CF80914205833029F4EA
:10E9600080914D058695887101C080E037DDC091AA
:10E97000940D8091950D32DD8C2F30DD5CDD809122
:10E98000910D882319F080E0C5DCF9CFE091920D5C
:10E99000F091930D1082E8E7F0E0808191819C0175
:10E9A0002854344F39BD28BD805B994B91838083B7
:10E9B000C09A88E086BF81E080937C0087B788603A
:10E9C00087BF80917D00816080937D0080914205AA
:10E9D000813031F080915D0282FD02C0F39401C06C
:10E9E000F12CF0922B0E05C0789457DD02C080E028
:10E9F00024DBDF91CF911F910F91FF90EF90DF907B
:10EA0000CF9008951F920F920FB60F9211242F935B
:10EA10003F934F935F936F937F938F939F93AF93A6
:10EA2000BF93CF93DF93EF93FF938CB59DB5209168
:10EA30002A0E222321F0C09A10922A0E04C0C098F8
:10EA400021E020932A0EC0910C01D0910D01FE010E
:10EA5000219131913BBD2ABDF0930D01E0930C0152
:10EA6000E6E0F1E0282F3181381708F48183308106
:10EA7000231708F480838A819B81892BD1F489E94B
:10EA80009DE090930D0180930C0180916702809529
:10EA9000817080932A0E87B78F7E87BF54DE809166
:10EAA00060028F7011F0833021F487B7806187BFD7
:10EAB000789480918F0D816080938F0DFF91EF91FD
:10EAC000DF91CF91BF91AF919F918F917F916F9186
:10EAD0005F914F913F912F910F900FBE0F901F901C
:10EAE0001895809167028095817080932A0E80939B
:10EAF000290E811101C0C09A809160028F70865FDB
:10EB000080938E0D10928B0D1ECE1F920F920FB61A
:10EB10000F9211242F933F934F935F936F937F93A3
:10EB20008F939F93AF93BF93EF93FF938091600276
:10EB30008F70813011F1863029F0853031F080E41A
:10EB400092EA05C080E89EE302C080E99DE397BD9C
:10EB500086BD20917800309179002F3F310538F43F
:10EB600088589341909379008093780007C088EC8F
:10EB700090E09093790080937800E5DDFF91EF912C
:10EB8000BF91AF919F918F917F916F915F914F91C5
:10EB90003F912F910F900FBE0F901F9018951F92CD
:10EBA0000F920FB60F9211242F933F934F935F93C1
:10EBB0006F937F938F939F93AF93BF93EF93FF9345
:10EBC000809160028F70789490918E0D981769F003
:10EBD000943059F480914D02882321F08091810670
:10EBE00085FD02C0B0DD02C084E027DAFF91EF911D
:10EBF000BF91AF919F918F917F916F915F914F9155
:10EC00003F912F910F900FBE0F901F9018958091FC
:10EC1000A80680FD05C0809165008B7F809365000C
:10EC20000895F5CFF4CF21E0FC018481811101C06A
:10EC300020E0822F0895FC0121818081281B27700C
:10EC400098E0921B81E0933008F480E00895CF9320
:10EC5000DF93EC018C818823F1F081508C838A81D1
:10EC60009B81890F8A838EA58823D1F18FA59FEF81
:10EC7000980F9FA7882351F08091A80680FD30C08F
:10EC8000809165008460809365002AC0C0DF809118
:10EC900083068FA725C01B98BADF8D81882319F0C2
:10ECA00081508D831DC0888199818917C9F090E0BA
:10ECB000FE01E80FF91F26812A8326892C832685E9
:10ECC0002B83268D2D8320A92EA71FA626A13FEFDB
:10ECD000320F36A3211104C00196877099278883CB
:10ECE000DF91CF910895EF92FF920F931F93CF93EF
:10ECF000DF93EC01F62E142FE22E9DDF882309F41A
:10ED000053C08091CC0181FD4FC0809178068873FB
:10ED100009F44AC0302F3295369536953370402F1E
:10ED20004F70333009F43FEFFF2021F090918206BD
:10ED3000965FF90E803129F48BEA189F112D11246A
:10ED400002C0883111F4169509C0883211F4110FF0
:10ED500005C0803319F4812F880F180F288104FF14
:10ED60000DC0FA821C83ED8205FB882780F98EA7EF
:10ED70001FA63B8329834423B9F001C04F5FE9817B
:10ED8000F0E0CF01019687709927281769F0EC0F02
:10ED9000FD1FF682168BE68E05FB002700F900ABFF
:10EDA000415046A336878983DF91CF911F910F9100
:10EDB000FF90EF9008950F931F93CF93DF93EC0193
:10EDC000062F642F809178068695869586958770A4
:10EDD000388129813213EFC010E00332110508F0A9
:10EDE000EAC0F801E954FF4FA0C300E326C000E3E6
:10EDF00021E0C0C002EA22E04AE064E6DAC00AE2AA
:10EE000022E045E06FE5CE016EDF01E22AE045E059
:10EE10006FE5CE0168DF0AE222E045E06FE5C9C098
:10EE200002EC23E04AE060E5CE015DDF02E423E08E
:10EE30004AE06CE3CE0157DF00E221E065C001E269
:10EE400021E045E066E4CE014EDF22E04FE062E3E0
:10EE5000CE0149DF22E04FE062C002E221E045E05E
:10EE60006EE6CE0140DF03E221E045E097C000E01E
:10EE700025E045E062E3CE0136DF25E045E06AE5C6
:10EE8000CE0131DF02E024E043E06EE692C003E20F
:10EE90002AE045E060E5CE0126DF01E224E145E01D
:10EEA00060E5CE0120DF03E22AE045E038C002E65B
:10EEB00025E044E16AE07DC002E22AE044E062E34A
:10EEC000CE0111DF01E224E148E066E4CE010BDF70
:10EED00002E22AE048E062E3CE0105DF01E224E13C
:10EEE00044E04DC00AE22AE002C002E222E345E02B
:10EEF0004BC001E203C002E201C003E22AE044E1A8
:10EF000060E057C002E122E04AE039C002E423E0B9
:10EF100044E16CE3CE01E7DE02EE23E044E160E58C
:10EF200048C000E321E048E22AC0813009F443C030
:10EF300000E121E04AE06BE43CC08130E1F100E116
:10EF400021E04AE061E435C000E121E046E031C063
:10EF500000E3D9CF813079F100E1D5CF00E112C0D3
:10EF600003E303C002E301C001E323E04FE00CC070
:10EF700001E329E144E103C000E321E04EE166E45E
:10EF800018C001E321E04AE068E713C002E321E092
:10EF90004AE06AE70EC003E321E04AE06CE709C0FB
:10EFA00000E520E04AE062E804C000ED20E04AE02D
:10EFB00062E3CE0198DEDF91CF911F910F9108950A
:10EFC00046E4682F8EEC91E0F6CE462F682F8EEC4B
:10EFD00091E0F1CE9091840691FF03C0862F0C94AE
:10EFE0009816EECFCF92DF92EF92FF920F931F937E
:10EFF000CF93DF93EC01062F142F47FF03C0842F1C
:10F000000E949816D7FF06C0D195C195D1098AE113
:10F010000E949816002369F0023019F464E670E04B
:10F0200002C06AE070E0CE012FD2262FC22FD72F68
:10F03000F82E64E670E0CE0127D29B01FB01EC01C3
:10F040006115710591F16A307105C4F06AE070E0F4
:10F05000C9011AD26B017C01653171051CF48EE681
:10F060008C0D05C08CE88C0D0E9494168EE60E94D3
:10F070009816F701309769F001E001C000E084E6DE
:10F080008E0F0E949816011104C0209741F18C2F19
:10F090000AC0209721F1CE016AE070E0F5D19E010F
:10F0A000281B390BC901845713C084570E9494163A
:10F0B0000023A9F0023079F46AE070E08F2D90E02F
:10F0C000E3D1C82F86E0860F0E9498168CE88C0F3B
:10F0D0000E94941604C086E08F0D0E9498161116A7
:10F0E0001CF4812F0E949816DF91CF911F910F91F0
:10F0F000FF90EF90DF90CF90089586B380958E7744
:10F1000008958FEF8ABB1BBA91E897BB9EE798BB27
:10F110009EE394BB91EC95BB11BA82BB98E092B987
:10F1200097EF93B9109261001092620094E190936E
:10F1300064009BEF9093650080938A0DD4B780E8BC
:10F1400084BF84BF80E487B985E886B987E083BF40
:10F150008CE981BF82E085BD83E487BF1FBC8AE064
:10F160008EBD10928B0082E880938A0080E28093AB
:10F170007D00789487E797E49093500180934F0146
:10F180000E942361882319F00E940D6B06C00E9423
:10F19000D35F0E940D6B0E94E66091E080B3809582
:10F1A000837C803419F49093CC01F8CF823849F4F1
:10F1B000F89466E072E088E00E9415680E942F6B68
:10F1C000FFCFD09062068D2D0E94146296DF982F9B
:10F1D0009670963031F48091CC0182608093CC019E
:10F1E00025C0C0E081FD05C08695CF5FC630D1F750
:10F1F0001DC08C2F0E9480608823C1F0C0936206DE
:10F200008C2F0E94146281E00E9409610E94E466D2
:10F2100024E04EEF51E060E086E10E94F06788E173
:10F220000E9457350E942F6B0E9411140E947E127B
:10F230008091920686FD0E94C36D81E08093390122
:10F240000E94EC1B1092390180919106895F0E9407
:10F250009A16D3FD76C080917B0684FF05C080910D
:10F26000780682FD47C03DC080918406882319F04E
:10F270006CE187E0AFDE0E942C1B0E94E46620E078
:10F2800040E853E060E080E00E94EC6680918106F7
:10F2900084FD08C000E12AE046E856E068E380E02B
:10F2A0000E94BA670E942F6B0E9411140E944E1890
:10F2B0000E943B188C010E942C12EC01C057DE4FBB
:10F2C0000E942F6B0E942C1B0E944E180E943B181C
:10F2D0007C0113DF8111C3CFE016F10609F463C08E
:10F2E000BECF0E94B163883C910520F48FEE91E07F
:10F2F0000E94491B0E944E18809121019091220189
:10F300006EE070E0ADD060933C010E94831B0E94D0
:10F310009E1B90917806987B21F48FED91E00E94DE
:10F32000491B8091CD01882331F084EB91E00E944C
:10F33000491B1092CD010E94111480915B020E9422
:10F340009416909105019260909305011092110717
:10F3500060E085EE97E00E949149C3DB8DE028E1F3
:10F3600030E00FB6F894A89521BD0FBE81BD2FE403
:10F370003CE2309352012093510180916206D816ED
:10F3800029F081E00E9409610E94056281E080937A
:10F390004E020E94951D8091B3018823D1F380E035
:10F3A0000E945B61F6CF0E942C12C817D90709F0A2
:10F3B00087CF55CF8EEC91E034CC05D0332312F4B7
:10F3C0008A1B9B0B10C0A29FB001B39FC001A39FDB
:10F3D000700D811D1124911DB29F700D811D11248E
:10F3E000911D0895F0DFB7FF0895821B930B0895D8
:10F3F000EADFA59F900DB49F900DA49F800D911DF5
:10F4000011240895B7FFF4CFF3DF821B930B089507
:10F41000DB018F939F93ECDFBF91AF91A29F800D93
:10F42000911DA39F900DB29F900D11240895991BDB
:10F4300079E004C0991F961708F0961B881F7A95EB
:10F44000C9F78095089587FB082E062687FD8195CC
:10F4500067FD6195ECDF0EF4919507FC81950895A9
:10F46000AA1BBB1B51E107C0AA1FBB1FA617B707EA
:10F4700010F0A61BB70B881F991F5A95A9F7809506
:10F480009095BC01CD01089597FB072E16F40094CA
:10F4900006D077FD08D0E4DF07FC05D03EF4909558
:10F4A00081959F4F0895709561957F4F0895A1E2D2
:10F4B0001A2EAA1BBB1BFD010DC0AA1FBB1FEE1FEE
:10F4C000FF1FA217B307E407F50720F0A21BB30B39
:10F4D000E40BF50B661F771F881F991F1A9469F7B5
:10F4E00060957095809590959B01AC01BD01CF0111
:10F4F0000895052E97FB16F400940FD057FD05D004
:10F50000D6DF07FC02D046F408C0509540953095F0
:10F5100021953F4F4F4F5F4F08959095809570957F
:10F5200061957F4F8F4F9F4F0895EE0FFF1F0590FE
:10F53000F491E02D0994FB01DC0102C001900D92D1
:10F5400041505040D8F708956817790768F4FB01D7
:10F55000DC01E40FF51FA40FB51F02C002900E924C
:10F5600041505040D8F70895E6CFDC0101C06D93BB
:10F5700041505040E0F70895DC01CB01FC01E199D6
:10F58000FECF06C0FFBBEEBBE09A31960DB20D92E6
:0CF5900041505040B8F70895F894FFCFA8
:10F59C00F00064000A02FF000000E10D990D990DC6
:02F5AC00990DB7
:00000001FF
